:100000001EC500004DC500004BC5000049C50000DD
:1000100047C5000045C5000043C5000041C50000BC
:100020003FC500003DC500003BC5000039C50000CC
:1000300037C5000035C5000033C500000C94951687
:100040002FC500002DC500002BC5000029C50000EC
:1000500027C5000025C5000023C500000C94C81466
:100060001FC500000C9463130C943A1319C50000CB
:1000700017C5000015C5000013C5000011C500001C
:100080000FC500000DC500000BC5000009C500002C
:100090000C94A2150C9412150C9459150C945B1E1B
:1000A000FFC40000FDC40000FBC40000F9C4000050
:1000B000F7C40000F5C40000F3C40000F1C4000060
:1000C000EFC40000EDC40000EBC400000C94111359
:1000D0000C94E812E5C40000E3C40000E1C4000091
:1000E000DFC400009C088D089608A5089C089C08A1
:1000F000A50896089C089C08ED08D408D408FF08B9
:10010000ED08FC08FF08FF08ED08ED08D109CD094E
:10011000CD09D409D109D109D409D409D109D1090A
:10012000290C2E0C330C3D0C470CC00C510C590CF7
:10013000610C6B0C750C7F0C8E0C980CC00CA20C17
:10014000AC0CB60CFC10FF10EE10F210F8103611CB
:10015000031107110D11111115111B111F1123117D
:10016000361129112D1131119D19AC198A19C9198E
:10017000C919C919C919C919C919C919C919C9196F
:10018000DA1754196A198319512554256C258325CA
:10019000CC25DE25FD25F729F729F729F729F429AC
:1001A000F429FB29FB29FB29FB29FB29FB29FB2936
:1001B000FB29F429F429FB29FB29FB29FB29FB292D
:1001C000F929F72907634236B79BD8A71A39685629
:1001D00018AEBAAB558C1D3CB7CC5763BD6DEDFD69
:1001E000753EF6177231BF000000803F0800000026
:1001F000BE922449123EABAAAA2ABECDCCCC4C3E1C
:1002000000000080BEABAAAAAA3E00000000BF000A
:100210000000803F0000000000084178D3BB438706
:10022000D1133D190E3CC3BD4282AD2B3E68EC821A
:1002300076BED98FE1A93E4C80EFFFBE01C4FF7F9F
:100240003F00000000006364696E6F70737578583A
:100250005B00203D0020543A00204974656D3A004F
:100260002056616C3D002053746F726520003A3D4A
:10027000003A003D3E003D00564323004D6F64624E
:100280007573206F70206661696C65640020636D12
:10029000643D003D0056435F6865617423003D0086
:1002A00050696E3A003D0050696E3A00573A00209E
:1002B00048616C74656400466F72636520576869B5
:1002C0007465003D00526573746F7265643A200076
:1002D0003A204E6F2073746F7265642076616C757E
:1002E0006573202D2064656661756C7400526573BA
:1002F000746F7265642066726F6D3A00436D643D81
:1003000000496E76616C6964204D41433A20736503
:10031000742064656661756C74000A4C617A796852
:100320006F6D652E7275204C696768744875622020
:10033000636F6E74726F6C6C65722076302E393517
:1003400000496E76616C696420636F6D6D616E64E7
:10035000003E3E2000312D7769726520636F756E17
:10036000743A200020416464723A00646576230088
:1003700020616C69766500204E6F64653A005365B4
:1003800061726368696E67004D6F64627573207097
:100390006F6F6C696E67206572726F723D004D6F92
:1003A000646275732056616C3A20004D6F6462750B
:1003B0007320706F6F6C696E67206572726F723D2B
:1003C000002D002050492056616C203A004D6F648A
:1003D00062757320706F6F6C696E67206572726FE3
:1003E000723D002D0020464D2056616C203A002FB2
:1003F0006D79686F6D652F735F6F75742F00202D99
:100400002D00204F464600204F4E00204F4646000C
:1004100020636D643A002043757274656D703A0014
:10042000205365743A002045787069726564000055
:10043000002100240027002A002D00300033000195
:10044000010000040107010A010000220025002824
:10045000002B002E003100340002010000050108CD
:10046000010B01000020002300260029002C002F92
:100470000032000001000003010601090105050525
:1004800005070508080808020202020A0A0808040B
:100490000404040101010101010101030303030339
:1004A000030303040707070C0C0C0C0C0C0C0C02C8
:1004B00002020206060606060606060B0B0B0B0BCF
:1004C0000B0B0B01021020200808102040102040C8
:1004D0008002010201080402010102040810204008
:1004E0008080402010080402018004020180402026
:1004F000100804020108040201010204081020404F
:1005000080010204081020408000000A0B02090C40
:100510000D0E0807030401000000000000000000A9
:1005200000000000000000000000000000000000CB
:100530000000000000121110000000000000000088
:100540000000000000000000000000000000005259
:100550006562696E642073756363657373004572C9
:10056000726F723A20726562696E64206661696CAE
:100570000052656E65776564207375636365737398
:10058000004572726F723A2072656E6577656420FD
:100590006661696C002074727920616761696E2000
:1005A000696E2035207365636F6E647300666169E0
:1005B0006C65642C2072633D00636F6E6E656374BE
:1005C00065642061732000202E2E2E002075736537
:1005D000723A003A00417474656D7074696E6720F8
:1005E0004D51545420636F6E6E656374696F6E2055
:1005F000746F20004661696C656420746F20636FBE
:100600006E6669677572652045746865726E65749B
:10061000207573696E6720444843500053746172BB
:1006200074696E67206C616E00005EBCE2613FDD44
:1006300083C29C7E20A3FD1F419DC3217FFCA2405D
:100640001E5F01E3BD3E6082DC237D9FC1421CFE34
:10065000A0E1BF5D0380DE3C62BEE0025CDF81633F
:100660003D7C22C09E1D43A1FF4618FAA427799B1A
:10067000C584DA3866E5BB5907DB856739BAE40615
:10068000581947A5FB7826C49A653BD987045AB800
:10069000E6A7F91B45C6987A24F8A6441A99C725F7
:1006A0007B3A6486D85B05E7B98CD2306EEDB351E6
:1006B0000F4E10F2AC2F7193CD114FADF3702ECCC5
:1006C00092D38D6F31B2EC0E50AFF1134DCE9072CC
:1006D0002C6D33D18F0C52B0EE326C8ED0530DEFA7
:1006E000B1F0AE4C1291CF2D73CA947628ABF517AA
:1006F000490856B4EA6937D58B5709EBB536688A8D
:10070000D495CB2977F4AA4816E9B7550B88D63487
:100710006A2B7597C94A14F6A8742AC896154BA96E
:10072000F7B6E80A54D7896B355573652074686548
:1007300020636F6D6D616E64733A202768656C701D
:1007400027202D207468697320746578740A2773D4
:1007500061766527202D207361766520636F6E6654
:10076000696720696E204E5652414D0A27676574AD
:1007700027202D2067657420636F6E666967206689
:10078000726F6D207072652D636F6E66696775722A
:1007900065642055524C0A276C6F616427202D2018
:1007A0006C6F616420636F6E6669672066726F6D3F
:1007B000204E5652414D0A276B696C6C27202D2024
:1007C00074657374207761746368646F6700444D67
:1007D00058696E2042756666657220616C6C6F6345
:1007E0002065727200496E697420696E2063683AF0
:1007F0000009526573657420646F6E650009436873
:1008000065636B696E6720666F7220312D57697260
:100810006520646576696365732E2E2E004453321D
:100820003438322D3130302070726573656E74004B
:1008300020416464723A006465762300312D776943
:10084000726520006D71747420006D6F6462757341
:100850002000696E7075747320006974656D732073
:1008600000436F6E666967757265643A00444D585F
:1008700020696E20737461727465642E2043686110
:100880006E6E656C733A00444D58206F757420731A
:100890007461727465642E204368616E6E656C735A
:1008A0003A2000436F6E6E2E2061626F7274656431
:1008B000004C6F61646564006C6F616420666169FF
:1008C0006C6564004E6F2073746F72656420636F93
:1008D0006E666967006C6F6164696E6720436F6E56
:1008E0006669670072657175657374204D51545463
:1008F00020436F6E666967005361766564005361DB
:1009000076696E6720636F6E6669672E2E00636F6F
:10091000756C64206E6F742070617273653A20008C
:1009200055706461746564006F6E006F66660048A0
:100930005454502F312E31202569002048545450F2
:100940002F312E310D0A486F73743A2025730D0A2A
:100950004163636570743A202A2F2A0D0A436F6E33
:100960006E656374696F6E3A20636C6F73650D0A10
:100970000025730020000D0A0047455400207472C2
:100980007920616761696E20696E20352073656327
:100990006F6E6473006661696C656420746F2063B8
:1009A0006F6E6E656374004552524F523A20536524
:1009B000727665722072657475726E65642000438C
:1009C0006F6E6669672070617273696E6720666119
:1009D000696C656400676F7420436F6E66696700B9
:1009E000687474703A2F2F00436F6E6669672055E4
:1009F00052493A20002D3E004F4F4D21005B002E02
:100A0000004D7920495020616464726573733A2007
:100A1000003A004D79206D616320616464726573F2
:100A2000733A20002F6D79686F6D652F735F6F7556
:100A3000742F004E6F742066696E64008A5811240A
:100A40001FBECFEFD1E2DEBFCDBF00E00CBF15E08F
:100A5000A0E0B2E0E6EFFEEC00E00BBF02C00790C2
:100A60000D92A232B107D9F72BE0A2E2B5E001C0A6
:100A70001D92AE39B207E1F715E0CFE1D5E000E015
:100A800006C021970109802FFE010E942766CE3102
:100A9000D10780E00807A9F70E946A4E0C94796795
:100AA000AFCAEF92FF920F931F93CF93DF937B0117
:100AB0008901C0E0D0E0CE15DF0559F0CC33D10577
:100AC00041F0F80161918F012196CE010E947E17BD
:100AD000F2CFDF91CF911F910F91FF90EF9008958A
:100AE0008F929F92AF92BF92CF92DF92EF92FF923E
:100AF0000F931F93CF93DF93E62EB72ED42EA52E00
:100B0000C22E932EF02E812EBC0180914A05909129
:100B10004B050E949143EC01892B09F453C0888551
:100B2000853009F04FC060E0CE010E9484438C0103
:100B300061E0CE010E948443DC011996CD91DC91E5
:100B40001A97D8011996ED91FC911A97E130F105A9
:100B500061F02CF4EF2BB1F56F2DCE0117C0E23010
:100B6000F10541F03797A9F02DC06F2DCE01039606
:100B70000E947E176E2DCE010E947E176D2DCE0134
:100B800001960E947E176C2DCE0102960E947E1760
:100B900019C00097B9F0FC018085853099F4C681B1
:100BA000D781209779F00F2D182D2C2D392D4D2D13
:100BB0005A2D6E2D7B2D89859A8592DF0A80DB81E7
:100BC000C02DEFCFDF91CF911F910F91FF90EF904C
:100BD000DF90CF90BF90AF909F908F900895CF926D
:100BE000DF92EF92FF920F931F93CF93DF93E091E9
:100BF000FE07F091FF07309789F09085953071F4EA
:100C000069017A01EB01682FCF010E9484439601AC
:100C1000A701BE01FC018185928562DFDF91CF9142
:100C20001F910F91FF90EF90DF90CF900895AF92BA
:100C3000BF92CF92DF92EF92FF920F931F93CF93C9
:100C4000DF93E1E0F0E0C0E0D0E0CC24C394D12C0D
:100C50004091260550912705B6010C2E02C0660F63
:100C6000771F0A94E2F77F0184E0E80EF11CCF01C0
:100C7000B12C9C01A0910402B0910502A817B907FC
:100C800020F42091040230910502A091B005B091AA
:100C9000B105A20FB31FAC90A091FA07B091FB076A
:100CA0009C0121503109A20FB31F0A2D10E02C9195
:100CB00030E00217130729F0462B572BAC92BB24C8
:100CC000B39401968E159F05A1F650932705409386
:100CD0002605BB2009F18091FA079091FB07E80FE8
:100CE000F91F028110E0218130E0408150E031970E
:100CF000608170E0CE0173DF0E94BC14DC01CB0187
:100D0000845D9E4FAF4FBF4F809322059093230584
:100D1000A0932405B09325052196F701C430D10591
:100D200009F096CFDF91CF911F910F91FF90EF9037
:100D3000DF90CF90BF90AF900895DC011296ED91B7
:100D4000FC911397309721F081E09085953009F060
:100D500080E00895CF92DF92EF92FF92CF93DF93DE
:100D6000DC011696ED91FC911797309721F12085C3
:100D7000223009F56A017B01EC0166E672E086EA41
:100D800098E00E948E1160E672E086EA98E00E9488
:100D90008E112AE030E0B701A60186EA98E00E94B1
:100DA0000F1286EA98E00E949F12EE81FF81C186B1
:100DB000D286E386F486DF91CF91FF90EF90DF90AB
:100DC000CF900895FC0186819781009789F0FC01FE
:100DD0002085223041F0253079F460E00E94844380
:100DE000009779F0FC01618572858385948508956B
:100DF0006FEF7FEFCB0108956EEF7FEF8FEF9FEFE7
:100E000008956DEF7FEF8FEF9FEF0895FC018481D0
:100E10009581009761F0FC012085223029F0253072
:100E200049F40E948443FC018185928508958FEFE7
:100E30009FEF08958EEF9FEF0895CF93C62F63E045
:100E4000FC01828193810E948443009749F04C2FDA
:100E500050E060E070E0FC0141875287638774874F
:100E6000CF91089563E0FC01828193810E948443C5
:100E7000009719F0FC01818508958FEF08958F92F6
:100E80009F92BF92CF92DF92EF92FF920F931F93A8
:100E9000CF93DF93EC0151DF882309F47EC08A8170
:100EA0009B810E94DD2A082F10E06801CC0CDD1C1C
:100EB000E12CF12C92E0B92E0430110504F5F70174
:100EC000EC0DFD1DEE5EFD4F808091800E941C2781
:100ED000009751F0FC01B086A401990C660B770BCA
:100EE0004187528763877487BC018A819B810E94F6
:100EF000CF430F5F1F4FF2E0EF0EF11CDDCF0A81F1
:100F00001B8160E0C8010E948443FC0181858887C1
:100F100061E0C8010E9484439D838C8362E0C80124
:100F20000E9484439F838E8369E572E086EA98E09D
:100F30000E948E11EA81FB816081718186EA98E0CE
:100F40000E94D71265E572E086EA98E00E948E1151
:100F5000488550E060E070E02AE086EA98E00E9470
:100F6000C71162E572E086EA98E00E948E1160E0A7
:100F700070E0CE014BDF4AE050E0BC0186EA98E029
:100F8000DF91CF911F910F91FF90EF90DF90CF9065
:100F9000BF909F908F900C94A212DF91CF911F91E0
:100FA0000F91FF90EF90DF90CF90BF909F908F9028
:100FB0000895CF93DF93EC018AE292E099838883CE
:100FC0006115710549F080914A0590914B050E9489
:100FD00091439B838A8302C01B821A82CE01DF91D8
:100FE000CF914DCF3F924F925F926F927F928F92AF
:100FF0009F92AF92BF92CF92DF92EF92FF920F93A8
:101000001F93CF93DF93CDB7DEB761970FB6F894F8
:10101000DEBF0FBECDBF6C015B012A017901302E0E
:101020006CEF72E086EA98E00E948E114AE050E090
:10103000B50186EA98E00E94A2121B861A861D86D8
:101040001C861F861E86E114F10421F47E012AE02D
:10105000E20EF11C60E070E0C601D8DE8C0133E0E6
:10106000A316B104C1F084E0A816B10481F5C6014D
:10107000F9DE823009F47BC038F4882309F477C0A4
:10108000813009F450C1C1C1853009F470C0893084
:1010900009F449C1BAC1D60118968C91873009F478
:1010A000B4C1C601DFDE853079F46DEE72E086EA08
:1010B00098E00E948E114AE050E065E070E086EA18
:1010C00098E00E94A21253C08DEF9FEF3EC6B1E0A0
:1010D000AB16B10409F44BC024F4A114B10461F0BF
:1010E00094C1F2E0AF16B10409F41DC125E0A216C7
:1010F000B10409F431C189C169E0C6019EDED6019F
:1011000018968C9190E08A309105F8F4FC018827BC
:10111000EE58FF4F8F4F0C942766F7018281938121
:10112000892B21F48FE7D60118968C93F701408123
:1011300051816281748107C0D7014D915C91052E68
:10114000000C660B770BC60105DE0E94BC14609391
:101150008E0B70938F0B8093900B9093910BF601F5
:101160008281938190932905809328054EC1C60101
:1011700079DE813009F49FC0C60124DEAB01BC01D9
:1011800014161506160617060CF043C0D60118965D
:101190008C9190E08A30910590F5FC018827E45805
:1011A000FF4F8F4F0C942766F70140835183862FA2
:1011B000660F990B93838283872F770F990B958303
:1011C0008483970143E050E060E070E0C6010E9434
:1011D000304A63E0A62EB12C43C0D7014D935C93F7
:1011E000970141E050E060E070E0C6010E94304AA3
:1011F000AA24A394B12C34C0F7015183408320E08A
:1012000030E040E050E061E070E0C6010E94304A0A
:1012100025C02AE030E086EA98E00E940F1260EDD7
:1012200072E086EA98E00E94C712D60118968C9167
:10123000883031F484E190E0F701918380830EC01F
:1012400084E690E0D70111969C938E9313961C929E
:101250001E92129715969C938E931497A12CB12CE5
:101260004701612C712C6A147B0409F165EC72E072
:1012700086EA98E00E948E114AE050E0B30186EAC7
:1012800098E00E94561263EC72E086EA98E00E94B1
:101290008E11F401619171914F014AE050E086EAAC
:1012A00098E00E94A212FFEF6F1A7F0ADCCF61E084
:1012B000C601C3DD28C0D60118968C91813019F57E
:1012C00067EB72E086EA98E00E94C7128FE7F601AA
:1012D0008087D70113961C921E92129784E690E0A5
:1012E00015969C938E9314974C9111965C9160E0A7
:1012F00074E6C6012FDD970143E050E060E070E046
:10130000C6010E94304AF6018085813009F076C01E
:10131000D70112968D919C911397892B09F06EC07D
:101320008FE780876BC0C6019DDD853009F46AC0F8
:10133000F70111821082138212821582148262E0F8
:10134000C6017BDD20E030E040E050E062E070E08C
:10135000C6010E94304A56C0C601EFDC882309F45A
:1013600054C0C6017FDD823009F44FC0853009F4D6
:101370004CC0813049F1C60125DD362F272FD6011B
:1013800018964C9150E04A30510570F4FA018827C4
:10139000EA57FF4F8F4F0C942766892E990F9908B3
:1013A00005C0832E922E02C0812C912C6EE672E035
:1013B00086EA98E0B3D74AE050E0B40186EA98E0C4
:1013C0000E94A212892809F1F7011182108213826A
:1013D00012821582148265E0C6012FDD20E030E024
:1013E00040E050E062E070E0C6010E94304A6FEADF
:1013F00072E086EA98E00E94C71207C0AA24A3946C
:10140000B12C03C032E0A32EB12CD60118968C91DA
:10141000843009F460C158F4813009F448C0B8F14F
:10142000823009F478C0833009F4ACC1E3C388305A
:1014300009F43DC338F4863009F480C1873009F4DB
:101440005BC1D8C3893009F4BBC28F3709F0D2C35E
:1014500060E0C8010E947E1760E0C80101960E940A
:101460007E1760E0C80102960E947E17F701A481F2
:10147000B5812FEF30E00E94366624E630E040E090
:1014800050E00E945962622FC801039621C1F70102
:10149000A081B1812FEF30E00E94366624E630E073
:1014A00040E050E00E945962622FC80111C1D7018B
:1014B00012962D913C91139784E690E0821B930B3A
:1014C00014962D913C911597829FD001839FB00D6A
:1014D000929FB00D11242FEF30E00E94366620E17C
:1014E00037E240E050E00E945962622FC801039643
:1014F000288B398B0E947E176CEA72E086EA98E0AE
:101500000DD74AE050E02889622F3989732F86EA87
:1015100098E00E94A212F701A481B5812FEF30E07C
:101520000E94366624E6422E512C612C712CA301B8
:1015300092010E945962C22EA22EF701A281B381AC
:101540002FEF30E00E943666A30192010E9459629B
:10155000D22EB22EF701A081B1812FEF30E00E9490
:1015600036662DE631E040E050E00E945962522F8D
:10157000422F4F71440F440F842F880F45E5682F89
:10158000649F060E60E0611D1124922F90742072FA
:1015900057FD21C091110BC0211104C0862F8095E9
:1015A000562F11C055E5560F40E06BEA33C02111AC
:1015B0000DC0482F5AEA459F040E40E0411D1124FA
:1015C0008BEA841B560F682F40E024C080E0562F22
:1015D0005095462F0EC0911111C021110CC0482FFB
:1015E0002AEA429F040E40E0411D11245BEA541B8D
:1015F0004B5A60E00FC0462F40950BC0211104C02C
:1016000085E5860F4BEA03C08AEA860F90E0461B09
:10161000682F50E0FFEFBF1609F426C0BB2009F188
:10162000662329F02D2D629F060E60E0611D552373
:1016300029F03D2D539F050E50E0511D442329F004
:101640002D2D429F040E40E0411D1124D0942D2DDC
:10165000229F020E20E0211D1124620F520F420F23
:1016600003C04FEF5FEF6FEF3FEFA31609F421C008
:1016700020E03C2D332321F0339F212D09F02F5FF3
:101680002223A1F0662321F0629F060E60E0611D17
:10169000552321F0529F050E50E0511D442321F0A7
:1016A000429F040E40E0411D112403C040E050E081
:1016B00060E0C801498B588B0E947E175889652FBE
:1016C000C80101960E947E174989642FC8010296BD
:1016D0000E947E178FC2D60114960D911C9115970A
:1016E000F8018085853009F085C2C8010E94DD2A95
:1016F000833009F07FC2F0C1D6011496ED91FC91C0
:1017000015978085853009F075C2C680D780C114D1
:10171000D10409F46FC2F60161857285CE0101968C
:1017200048DC032D9701A201B501CE0101965ADCD8
:10173000D6011296CD90DC901397E9CFE02E61E0B0
:10174000802F0E944814FF24F394AA94AB2809F038
:10175000F12C6F2D8E2D0E94191467EA72E086EA33
:1017600098E0DCD54AE050E0B80186EA98E09ED6E1
:1017700065EA72E086EA98E0D1D56F2D70E04AE024
:1017800050E01AC117FF07C0119501951109AA244D
:10179000A394B12C02C0A12CB12CD02E61E0802FDB
:1017A0000E9448148091A100887F8093A1008091BD
:1017B0009100887F809391008091A1008260809346
:1017C000A10080919100826080939100F701A08137
:1017D000B181AB2899F0CD01BB0FAA0BBB0B9C01CB
:1017E000AD012456310941095109AFEFB0E00E9423
:1017F00075622CE93FEF4FEF5FEF08C02FEF30E04D
:101800000E94366624E630E040E050E00E945962D3
:10181000790161E08D2D0E944814E114F10409F46E
:10182000B3C0FFEFEF16F10409F4B0C0F801FF27D1
:10183000E75FFA4FE4914E2F50E0FA013197E23121
:10184000F10508F09DC08827E057FF4F8F4F0C949B
:10185000276684B5806884BDE7BC9BC084B5806280
:1018600084BDE8BC96C08091800080688093800031
:10187000F0928900E09288008CC0809180008062A4
:1018800080938000F0928B00E0928A0082C0809169
:101890008000886080938000F0928D00E0928C0040
:1018A00078C08091B00080688093B000E092B3006F
:1018B00070C08091B00080628093B000E092B4006C
:1018C00068C080919000806880939000F0929900A9
:1018D000E09298005EC080919000806280939000BA
:1018E000F0929B00E0929A0054C080919000886032
:1018F00080939000F0929D00E0929C004AC08091FD
:10190000A00080688093A0008091A0008F7B8093CE
:10191000A000F092A900E092A8003BC08091A00036
:1019200080628093A000F092AB00E092AA0031C0E8
:101930008091A00088608093A000F092AD00E092BA
:10194000AC0027C080912001806880932001F09234
:101950002901E09228011DC08091200180628093BE
:101960002001F0922B01E0922A0113C08091200106
:10197000886080932001F0922D01E0922C0109C033
:1019800020E8E216F10414F460E001C061E08D2D5E
:1019900050D760EA72E086EA98E0C0D44AE050E0AE
:1019A000B80186EA98E082D56EE972E086EA98E0AE
:1019B000B5D44AE050E0B70186EA98E0C3D51AC131
:1019C000D7011C9160E070E0C60120DA082FF92EE3
:1019D00068E772E086EA98E0A1D44AE050E0602F20
:1019E0007F2D86EA98E062D566E772E086EA98E0A5
:1019F00095D4612F012E000C770B4AE050E086EA67
:101A000098E0A0D58091440590914505892B09F077
:101A100092C081E090E0909345058093440526E0D4
:101A200040E855E260E070E089E098E075D6009308
:101A3000FC0989E098E09093FB098093FA091092E1
:101A4000070B1092090B1092080B80ED97E0909312
:101A5000820A8093810A1092840A1092830A1123C9
:101A600039F085E090E09093860A8093850A04C05F
:101A70001092860A1092850A86E00E940C2862E382
:101A800070E080E090E040D782ED97E09093820A8A
:101A90008093810A1092840A1092830AB4E61B0292
:101AA000C00111249093860A8093850A9CC0D601B8
:101AB0001496ED91FC91159761857285CE01019682
:101AC00078DACE01019639D9882309F493C0898543
:101AD000893009F08FC093C060E0C8010E94844340
:101AE000FC015184752C628461E0C8010E9484432A
:101AF000DC0119968D909D90AD90BC901C9762E092
:101B0000C8010E948443FC0101851285F701A08170
:101B1000B1812FE330E00E94366624E630E040E0F9
:101B200050E00E94596269017A01809144059091C8
:101B30004505892B31F06CE772E086EA98E027D5FD
:101B400059C081E090E0909345058093440526E2DA
:101B500040E855E260E070E089E098E0DDD5509221
:101B6000FC0989E098E09093FB098093FA091092B0
:101B7000070B1092090B1092080B012B09F43BC0C4
:101B8000DC2CCC24CC24CA944AE050E0672D762D7E
:101B900086EA98E08BD463E772E086EA98E0BED3E9
:101BA000B501A4016627772720E186EA98E0EFD304
:101BB00061E772E086EA98E0B1D3A60160E070E0E8
:101BC00020E186EA98E0E3D386EA98E0B8D49092E0
:101BD000820A8092810A1092840A1092830AD0921B
:101BE000860AC092850A86E00E940C28109245055C
:101BF00010924405AAC0DD24DD24DA94C5CF0A2D55
:101C0000D7011C9160E070E0CE010196FFD8F82E5C
:101C1000E92E65E972E086EA98E080D34AE050E078
:101C20006F2D7E2D86EA98E041D463E972E086EA62
:101C300098E074D3612F012E000C770B4AE050E03E
:101C400086EA98E033D46DE872E086EA98E066D3DD
:101C50006A2DAA0C770B4AE050E086EA98E072D42D
:101C60008091440590914505892B09F064CF81E06E
:101C700090E0909345058093440526E040E855E2C6
:101C800060E070E089E098E047D5F092FC0989E0D7
:101C900098E09093FB098093FA091092070B109239
:101CA000090B1092080B0230A9F1053099F1612F50
:101CB000110F770B880B990B0E94986322E538EB84
:101CC00042E152E40E94956220E030E040E251E4BB
:101CD0000E944C642DEE3EE94CE35EE30E94FD62FF
:101CE0006B017C0120E030E0A9010E94486420E003
:101CF00030E040E05FE387FD05C0C701B6010E9408
:101D0000956204C0C701B6010E9494620E94656397
:101D10008B0102C000E010E0A80160E070E02AE062
:101D200086EA98E034D386EA98E009D483ED97E018
:101D30009093820A8093810A1092840A1092830AF7
:101D40001093860A0093850A4ECF61960FB6F894D9
:101D5000DEBF0FBECDBFDF91CF911F910F91FF90DE
:101D6000EF90DF90CF90BF90AF909F908F907F903B
:101D70006F905F904F903F900895CF93DF93EC0169
:101D80006BEA73E00E94A366892B41F16EEA73E06F
:101D9000CE010E94A366892B21F162EB73E0CE0194
:101DA0000E94A366892B01F167EB73E0CE010E94CC
:101DB000A366892BE1F06EEB73E0CE010E94A3666F
:101DC000892BC1F088818D32C1F090ED980F9A3047
:101DD000A0F08B37A9F48EEF9FEF14C081E090E064
:101DE00011C082E090E00EC083E090E00BC084E080
:101DF00090E008C085E090E005C080E090E002C07F
:101E00008FEF9FEFDF91CF910895EF92FF920F93A5
:101E10001F93CF93DF938091260590912705C4E00F
:101E2000D0E021E030E0A90148235923452B29F0D7
:101E3000A9014095509584239523220F331F2197A4
:101E400091F7909327058093260596D5009122055A
:101E50001091230520912405309125056017710705
:101E60008207930708F458C0012B022B032B09F4B7
:101E700053C010922205109223051092240510924F
:101E80002505E12CF12CE091FA07F091FB07EC0F0E
:101E9000FD1F038110E0228130E0418150E060812C
:101EA00070E0C7010E94EF058FEFE81AF80A249648
:101EB00084E0E816F10439F7C1E0D0E08091040233
:101EC000909105028C179D0728F48091040290914F
:101ED000050201C0CE012091B0053091B105F90194
:101EE000E80FF91F408150E060E070E02AE086EAE8
:101EF00098E04DD263EC73E086EA98E058D32196DF
:101F0000C131D105D9F686EA98E0DF91CF911F91D2
:101F10000F91FF90EF9013C3DF91CF911F910F911D
:101F2000FF90EF900895CF92DF92EF92FF920F9380
:101F30001F93CF93DF936C017A018B01C0E0D0E057
:101F4000CE15DF0589F0D8016D918D01D601ED9197
:101F5000FC910190F081E02DC6011995892B11F4B7
:101F60007E0102C02196ECCFC701DF91CF911F9176
:101F70000F91FF90EF90DF90CF900895FC01A08922
:101F8000B1898C91A689B78982FD0FC09C91818D02
:101F90008F5F8F73228D821749F0218DDF01A20F91
:101FA000B11D5D969C93818F08958C910895FC01DD
:101FB000538D448D252F30E0842F90E0821B930BAE
:101FC000541710F0CF96089501970895FC01918D54
:101FD000828D981761F0828DDF01A80FB11D5D968B
:101FE0008C91928D9F5F9F73928F90E008958FEFF9
:101FF0009FEF0895FC01918D828D981731F0828DAD
:10200000E80FF11D858D90E008958FEF9FEF089503
:10201000FC01918D228D892F90E0805C9F4F821B67
:1020200091098F739927089589E098E0F1DF21E005
:10203000892B09F420E0822F089586EA98E0E8DFF2
:1020400021E0892B09F420E0822F0895FC01848D82
:10205000DF01A80FB11DA35ABF4F2C91848D90E0D2
:1020600001968F739927848FA689B7892C93A089AD
:10207000B1898C9180648C93938D848D981306C064
:102080000288F389E02D80818F7D80830895EF920F
:10209000FF920F931F93CF93DF93EC0181E0888F22
:1020A0009B8D8C8D981305C0E889F989808185FD09
:1020B00023C0F62E0B8D10E00F5F1F4F0F731127FB
:1020C000E02E8C8DE8120BC00FB607FCFACFE88922
:1020D000F989808185FFF5CFCE01B8DFF2CF8B8DF6
:1020E000FE01E80FF11DE35AFF4FF0820B8FEA89E2
:1020F000FB898081806207C0EE89FF896083E8895F
:10210000F98980818064808381E090E0DF91CF91C4
:102110001F910F91FF90EF900895CF93DF93EC0103
:10212000888D8823C1F0EA89FB89808185FD05C0FF
:10213000A889B9898C9186FD0EC00FB607FCF5CF32
:10214000808185FFF2CFA889B9898C9185FFEDCF79
:10215000CE017CDFE8CFDF91CF91089580E090E061
:10216000892B19F06ADF811120C080E090E0892B73
:1021700041F080E090E0892B21F00E940000811165
:1021800017C080E090E0892B19F04EDF811113C059
:1021900080E090E0892BA1F080E090E0892B81F035
:1021A0000E94000081110AC008950E940000DDCF46
:1021B0000E940000E6CF0E940000EACF0C940000CD
:1021C000089590E0FC013197E231F10508F04EC02E
:1021D0008827EE55FF4F8F4F0C9427668091800023
:1021E0008F7703C0809180008F7D80938000089559
:1021F00080918000877FF9CF84B58F7702C084B546
:102200008F7D84BD08958091B0008F7703C0809149
:10221000B0008F7D8093B0000895809190008F77FB
:1022200007C0809190008F7D03C080919000877FD0
:102230008093900008958091A0008F7707C08091CF
:10224000A0008F7D03C08091A000877F8093A000B5
:102250000895809120018F7707C0809120018F7DA4
:1022600003C080912001877F8093200108953FB7AC
:10227000F8948091BE059091BF05A091C005B091E2
:10228000C10526B5A89B05C02F3F19F00196A11DD9
:10229000B11D3FBFBA2FA92F982F8827820F911DFC
:1022A000A11DB11DBC01CD0142E0660F771F881F43
:1022B000991F4A95D1F70895CF93DF931F92CDB719
:1022C000DEB789832091B2053981E091B305F091A1
:1022D000B405822F90E080959095F89400800822B4
:1022E00000824BE000C05DE000005A95E9F70080F5
:1022F00008220894379508F4022A00824A9599F733
:1023000078940F90DF91CF9108950E945066DC0180
:10231000ED91FC910190F081E02D1994EF92FF92E4
:102320000F931F93CF93DF938C017B01C0E0D0E02C
:10233000F701EC0FFD1F6491662361F0D801ED9168
:10234000FC910190F081E02DC8011995892B11F0C5
:102350002196EECFCE01DF91CF911F910F91FF908B
:10236000EF9008956115710579F0FB01019000204F
:10237000E9F73197AF01461B570BDC01ED91FC915A
:102380000280F381E02D199480E090E008954F924F
:102390005F926F927F92EF92FF920F931F93CF9372
:1023A000DF93CDB7DEB7A1970FB6F894DEBF0FBEAF
:1023B000CDBF7C01FA01CB0119A2223008F42AE03A
:1023C0008E010F5D1F4F422E512C612C712CBF01CD
:1023D000A30192010E943762F901CA01015011095B
:1023E0006A3014F4605D01C0695CD8016C93232BE2
:1023F000242B252B61F7B801C701B4DFA1960FB6D6
:10240000F894DEBF0FBECDBFDF91CF911F910F912A
:10241000FF90EF907F906F905F904F900895CF92D4
:10242000DF92EF92FF920F931F93CF93DF93EC0114
:102430006A017B012115310579F4E881F981019068
:10244000F081E02D642FDF91CF911F910F91FF90CC
:10245000EF90DF90CF9019942A303105D9F477FFAF
:1024600018C06DE254DF8C0144275527BA014C197E
:102470005D096E097F092AE0CE0189DF800F911F77
:10248000DF91CF911F910F91FF90EF90DF90CF9050
:1024900008952AE0B701A601CE01DF91CF911F91E7
:1024A0000F91FF90EF90DF90CF9071CF9A01AB0129
:1024B000770F660B770BB3CF8F929F92AF92BF923D
:1024C000CF92DF92EF92FF920F931F93CF93DF9300
:1024D0007C018B016C0182E0C80ED11C4701E5E054
:1024E0008E0E911CC0E0D0E0F60141916F0150E0EA
:1024F00060E070E02AE0C8014ADF5C016EE2C801DA
:1025000006DF8A0D9B1DC80FD91FC814D90461F7B7
:10251000F701458150E060E070E02AE0C80137DF54
:102520008C0F9D1FDF91CF911F910F91FF90EF9026
:10253000DF90CF90BF90AF909F908F90089565EE01
:1025400073E010CF0F931F93CF93DF93EC019A01A9
:10255000AB01770F660B770B62DF8C01CE01EFDFEB
:10256000800F911FDF91CF911F910F9108950F93CD
:102570001F93CF93DF93EC01F5DE8C01CE01DFDFFB
:10258000800F911FDF91CF911F910F9108950F93AD
:102590001F93CF93DF93EC01C1DE8C01CE01CFDF1F
:1025A000800F911FDF91CF911F910F910895DACE87
:1025B00023EA33E0FC0131832083FB014081518118
:1025C00062817381FC014283538364837583089520
:1025D0001F920F920FB60F9211240BB60F922F93EA
:1025E0003F934F935F936F937F938F939F93AF939B
:1025F000BF93EF93FF9389E098E028DDFF91EF917F
:10260000BF91AF919F918F917F916F915F914F910A
:102610003F912F910F900BBE0F900FBE0F901F9008
:1026200018951F920F920FB60F9211240BB60F92AE
:102630002F933F934F935F936F937F938F939F93CA
:10264000AF93BF93EF93FF9389E098E097DCFF91FE
:10265000EF91BF91AF919F918F917F916F915F911A
:102660004F913F912F910F900BBE0F900FBE0F9087
:102670001F9018951F920F920FB60F9211240BB650
:102680000F922F933F934F935F936F937F938F930B
:102690009F93AF93BF93EF93FF9386EA98E0D6DCC6
:1026A000FF91EF91BF91AF919F918F917F916F912A
:1026B0005F914F913F912F910F900BBE0F900FBEE6
:1026C0000F901F9018951F920F920FB60F92112422
:1026D0000BB60F922F933F934F935F936F937F931C
:1026E0008F939F93AF93BF93EF93FF9386EA98E006
:1026F00045DCFF91EF91BF91AF919F918F917F91B9
:102700006F915F914F913F912F910F900BBE0F9062
:102710000FBE0F901F901895CF92DF92EF92FF920D
:102720001F93CF93DF93EC016A017B01122FE8899D
:10273000F98982E080834115514E61057105B1F040
:1027400060E079E08DE390E0A70196010E94376296
:10275000DA01C9010197A109B109B695A795979525
:102760008795AC01411580E15807A8F0E889F989FF
:10277000108260E874E88EE190E0A70196010E9463
:102780003762BA01A9014150510961097109769571
:10279000679557954795EC85FD855083EE85FF85B8
:1027A0004083188EEC89FD891083EA89FB8980813A
:1027B00080618083EA89FB89808188608083EA89DF
:1027C000FB89808180688083EA89FB8980818F7D95
:1027D0008083DF91CF911F91FF90EF90DF90CF909A
:1027E0000895CF93DF93282F30E0F901E75FFA4F88
:1027F0008491F901ED53FB4FD491F901E358FB4F5C
:10280000C491CC2389F08111DCDCEC2FF0E0EE0FD9
:10281000FF1FED59FB4FA591B491EC91ED2381E0A1
:1028200090E021F480E002C080E090E0DF91CF9161
:1028300008951F93CF93DF93282F30E0F901E75FCE
:10284000FA4F8491F901ED53FB4FD491F901E3580C
:10285000FB4FC491CC23C1F0162F8111B2DCEC2FB9
:10286000F0E0EE0FFF1FE75BFB4FA591B4918FB730
:10287000F894111105C09C91ED2FE095E92302C059
:10288000EC91ED2BEC938FBFDF91CF911F910895C9
:10289000CF93DF9390E0FC01ED53FB4F2491FC01BB
:1028A000E358FB4F8491882361F190E0880F991FD2
:1028B000FC01E15DFB4FC591D491FC01E75BFB4F4F
:1028C000A591B491611109C09FB7F89488812095B2
:1028D00082238883EC912E230BC0623061F49FB772
:1028E000F8943881822F809583238883EC912E2B56
:1028F0002C939FBF06C08FB7F894E8812E2B2883B6
:102900008FBFDF91CF9108958F929F92AF92BF9228
:10291000CF92DF92EF92FF926B017C01A8DC4B011A
:102920005C01C114D104E104F104E9F0A0DCDC0194
:10293000CB0188199909AA09BB09883E9340A105D2
:10294000B10578F321E0C21AD108E108F10888EE58
:10295000880E83E0981EA11CB11CC114D104E104AF
:10296000F10421F7DECFFF90EF90DF90CF90BF9082
:10297000AF909F908F9008952FB7F8946091BA050B
:102980007091BB058091BC059091BD052FBF089546
:102990001F920F920FB60F9211242F933F938F9394
:1029A0009F93AF93BF938091BA059091BB05A0917F
:1029B000BC05B091BD053091B90523E0230F2D373B
:1029C00020F40196A11DB11D05C026E8230F029633
:1029D000A11DB11D2093B9058093BA059093BB0545
:1029E000A093BC05B093BD058091BE059091BF0535
:1029F000A091C005B091C1050196A11DB11D8093A4
:102A0000BE059093BF05A093C005B093C105BF91CB
:102A1000AF919F918F913F912F910F900FBE0F908B
:102A20001F9018951F920F920FB60F9211240BB69C
:102A30000F922F933F934F935F938F939F93EF93B7
:102A4000FF932091B0053091B1058091AE05909132
:102A5000AF05AC014F5F5F4F5093AF054093AE059C
:102A6000F901E80FF91F80818093CE008091040264
:102A7000909105022091AE053091AF058217930722
:102A800048F48FEF9FEF9093AF058093AE0588E4F5
:102A90008093C900FF91EF919F918F915F914F912A
:102AA0003F912F910F900BBE0F900FBE0F901F9074
:102AB00018951F920F920FB60F9211242F933F93E8
:102AC0008F939F932091AC053091AD058091AE0519
:102AD0009091AF0521303105A9F48F3F2FEF920778
:102AE00089F41092C8001092CD0089E08093CC0048
:102AF00086E28093CA001092CE001092AF05109229
:102B0000AE0517C0892BA9F41092C8001092CD0011
:102B100083E08093CC008EE08093CA0088E28093AB
:102B2000C9001092CE0081E090E09093AF058093B1
:102B3000AE059F918F913F912F910F900FBE0F90F7
:102B40001F9018951F920F920FB60F9211240BB67B
:102B50000F922F933F934F935F936F937F938F9336
:102B60009F93AF93BF93EF93FF932091C800809101
:102B7000CE009091AB0524FF08C081E08093AB05A7
:102B80008091B0059091B10554C0913091F48111BC
:102B90000DC082E08093AB05EFDE6093400570933B
:102BA000410580934205909343053EC01092AB05CA
:102BB00044C0923009F041C0E091A905F091AA0506
:102BC0009081981721F091E09093030280832091E7
:102BD000A9053091AA058091A7059091A80528170D
:102BE000390711F51092AB05809103028823D1F0CB
:102BF0008091A5059091A605892BA1F01092C9009E
:102C0000E091A505F091A605199580E98093C9008A
:102C10001092C8001092CD0083E08093CC008EE02B
:102C20008093CA00109203028091A9059091AA0591
:102C300001969093AA058093A905FF91EF91BF910A
:102C4000AF919F918F917F916F915F914F913F9144
:102C50002F910F900BBE0F900FBE0F901F901895E5
:102C60000F931F93CF93DF93EC010E94B92EFE01C7
:102C7000E35DFD4F9183808301978231924008F09C
:102C80004CC042E152E08E01055E1F4FB801CE01FB
:102C90000E94EC38F801ACE2B2E048E04A0F219122
:102CA0008D9130E0082E000C990B28173907A9F5F3
:102CB0004A13F5CF0CA110E0102F00278BA1082B91
:102CC000FE01E15DFD4F11830083011580E51807CA
:102CD00001F54FA1329640838AA590E0982F88276E
:102CE00029A5822B3196918380836BA570E0762F86
:102CF00066272CA5622B32967183608332960190F1
:102D0000F081E02D309759F09E01235D3F4F1995DA
:102D100006C0011520E2120711F000E010E0C80122
:102D2000DF91CF911F910F91089578941F920F9288
:102D30000FB60F9211240BB60F92CF92DF92EF9243
:102D4000FF920F931F932F933F934F935F936F9334
:102D50007F938F939F93AF93BF93CF93DF93EF9323
:102D6000FF93809170008E7F809370000FE310E0DE
:102D70008BE1E82EF12C9BE2C92ED12CC091B50538
:102D8000D091B6052097F9F40332110508F43AC042
:102D900003521109E091B305F091B405908180913F
:102DA000B205282F2095922390839BE0D70111979D
:102DB000F1F79150D9F79081892B8083C601019753
:102DC000F1F780E00DC00B301105E0F00B50110958
:102DD000E091B705F091B805EC0FFD1F31978081A8
:102DE0006BDA2196D093B605C093B50580910102A8
:102DF000909102028C179D0708F0C0CF1092B60583
:102E00001092B50580917000816080937000FF91F1
:102E1000EF91DF91CF91BF91AF919F918F917F9172
:102E20006F915F914F913F912F911F910F91FF9063
:102E3000EF90DF90CF900F900BBE0F900FBE0F90D2
:102E40001F90189581E08093A40580910002282F9F
:102E500030E0F901E358FB4FE491F0E0EE0FFF1F83
:102E6000E75BFB4F459154915093B4054093B305F4
:102E7000F901ED53FB4FE491E093B20561E008DD09
:102E800083E08093B100E0E7F0E08081816080839F
:102E90000895CF93DF931816190644F080917000BF
:102EA0008E7F809370001092A40519C0EC01809170
:102EB000B7059091B8050E94575ACE01C130D24053
:102EC00014F080E092E090930202809301020E944D
:102ED000C2599093B8058093B705892B29F41092B5
:102EE00002021092010207C08091A405811103C063
:102EF000DF91CF91A7CFDF91CF910895EF92FF920D
:102F00001F93CF93DF931F921F92CDB7DEB7162F7B
:102F10002091A405211105C089839A8393DF9A81AA
:102F200089817C0121E0E21AF108E114E2E0FE0669
:102F300090F420910102309102022817390708F419
:102F4000A8DF8091B7059091B805009721F08E0D0C
:102F50009F1DFC0110830F900F90DF91CF911F9167
:102F6000FF90EF9008954F925F926F927F928F92B1
:102F70009F92AF92BF92CF92DF92EF92FF920F9308
:102F80001F93CF93DF93CDB7DEB729970FB6F89491
:102F9000DEBF0FBECDBFE0912906F0912A063C9618
:102FA000E031F10508F0F5C18827EC54FF4F8F4F51
:102FB0000C9427666CE176E086EA98E0E8DA0FB6D2
:102FC000F894A895809160008861809360001092C9
:102FD00060000FBE80912106811107C086E096E057
:102FE0000E94AF2F81E08093210683EC95E09093BF
:102FF0005609809355096CE271E080E090E084DC32
:103000001FB7F8948091C205811123C0E2EBF4E070
:103010008491E8EFF4E09491E82FF0E0EE0FFF1FC9
:10302000E15DFB4FA591B491EC91E92319F461E0C6
:1030300085E3FFDB61E085E32BDC8CB580618CBD33
:103040008CB580648CBD61E084E322DC61E083E3C5
:103050001FDC8091C2058F5F8093C2051FBF249A39
:1030600080E590E00E94A23E67E080E090E00E9450
:10307000B62765E58BE190E00E94B62765E58AE119
:1030800090E00E94B6270E94A13E80E090E49093D9
:10309000E0078093DF0780E090E69093E807809355
:1030A000E70780E098E49093E2078093E10780E0EF
:1030B00098E69093EA078093E90780E090E5909383
:1030C000E4078093E30780E090E79093EC07809318
:1030D000EB0780E098E59093E6078093E50780E0B2
:1030E00098E79093EE078093ED0780E590E00E94CB
:1030F000A23E46E050E06CE275E089E090E00E947C
:103100008D2783EA93E09A8389831B821C821D8228
:103110001E82CE0103960E949A3E0E94A13E80919B
:10312000550990915609DC0192961D921D921D92AF
:103130001C929597FC0116A217A210A611A69A96AA
:103140001D921D921D921C929D9740EE5EE260E0E2
:1031500070E046AB57AB60AF71AF40EA5FE060E054
:1031600070E0DA964D935D936D937C93DD9718969E
:1031700026E0FD01322F11923A95E9F7AC01425F4A
:103180005F4F34E1FA0111923A95E9F7ECE2F5E08C
:1031900001900D922A95E1F7FC01EE5BFF4F108242
:1031A0000E946F368130910509F04DC080E590E0B6
:1031B0000E94A23E6091550970915609625F7F4F4F
:1031C000CE010196F5D9CE0103960E949A3E6091F8
:1031D0005509709156096A5E7F4FCE010196E8D974
:1031E00044E050E0BE016D5F7F4F81E090E00E94BF
:1031F0008D2760915509709156096E5E7F4FCE0103
:103200000196D6D944E050E0BE016D5F7F4F85E066
:1032100090E00E948D270E94A13E60915509709117
:103220005609625E7F4FCE010196C2D98B819C8187
:10323000AD81BE818093510990935209A0935309A7
:10324000B09354091DC0892BD9F464EF75E086EA68
:1032500098E09DD986EF9FEF90932A0680932906E8
:103260008BDBDC01CB01805A9541AF4FBF4F809380
:10327000020890930308A0930408B093050808C0BF
:103280000E94D44981E090E090932A068093290619
:1032900099E288E10FB6F894A895809360000FBE7C
:1032A00090936000A89575C060E070E080E090E0C9
:1032B0000E94DB4090932A06809329068091520554
:1032C00090915305009709F464C066E379E10E9488
:1032D0005F2F5FC0A89519860E947D2B811159C070
:1032E0000091FC071091FD070115110509F451C06B
:1032F000C8010E94DD2A682E712CF2E06F1671045D
:103300000CF09EC146C00E947D2B811142C082E01C
:1033100090E03BC031DB009102081091030820913E
:10332000040830910508061717072807390788F59C
:1033300010922A06109229062CC01EDB009102086A
:10334000109103082091040830910508061717070B
:1033500028073907E0F21DC060E070E080E090E0EF
:103360000E942443892B99F607DBDC01CB018857A7
:103370009C4EAF4FBF4F8093020890930308A093D9
:103380000408B093050886EF9FEF90932A06809378
:1033900029060FB6F894A895809160008861809303
:1033A0006000109260000FBE8091290690912A065D
:1033B000181619060CF01FC10091550910915609F5
:1033C0000115110509F417C1D7DA4B015C01780129
:1033D000BEE3EB0EF11CF70180819181A281B381E4
:1033E000A5019401281B390B4A0B5B0BCA01B901DB
:1033F000683E33E073078105910508F446C028EE66
:1034000033E040E050E00E943762861A970AA80A2B
:10341000B90AD7018D929D92AD92BC921397F80193
:1034200086A597A5A0A9B1A969017A01CC0CDD1CDC
:10343000EE1CFF1C8C159D05AE05BF0528F416A6D5
:1034400017A610AA11AA09C0821B930BA40BB50BD7
:10345000F80186A797A7A0ABB1ABF80182A993A901
:10346000A4A9B5A98C159D05AE05BF0528F412AA1F
:1034700013AA14AA15AA09C0821B930BA40BB50B9F
:10348000F80182AB93ABA4ABB5ABF80186A597A5C9
:10349000A0A9B1A9892B8A2B8B2B69F4EE5BFF4F76
:1034A0008081833041F484E08083C8010E946F36BC
:1034B00001967C0102C0E12CF12CF80182A993A9AC
:1034C000A4A9B5A9892B8A2B8B2BA1F4EE5BFF4F06
:1034D0008081833011F081110DC01082F8013E9679
:1034E00084E1DF011D928A95E9F7C8010E946F36D9
:1034F00003967C01B2E0EB16F10429F0E4E0EE164D
:10350000F10409F04CC080E590E00E94A23E609179
:10351000550970915609625F7F4FCE01019648D8D8
:10352000CE0103960E949A3E60915509709156090A
:103530006A5E7F4FCE0101963BD844E050E0BE0169
:103540006D5F7F4F81E090E00E948D27609155096B
:10355000709156096E5E7F4FCE01019629D844E0E6
:1035600050E0BE016D5F7F4F85E090E00E948D27A7
:103570000E94A13E6091550970915609625E7F4F8D
:10358000CE01019615D88B819C81AD81BE8180933F
:10359000510990935209A0935309B0935409F2E052
:1035A000EF16F10491F034F4EA94EF2821F561E884
:1035B00075E010C043E0E416F10451F054E0E51664
:1035C000F104C9F46FE475E010C061E775E00DC067
:1035D0006EE575E086EA98E00E94C71286EF9FEFDD
:1035E00090932A068093290606C086EA98E00E94F6
:1035F000C7120E94D44999E288E10FB6F894A895C1
:10360000809360000FBE9093600080912906909196
:103610002A0629960FB6F894DEBF0FBECDBFDF9104
:10362000CF911F910F91FF90EF90DF90CF90BF90BF
:10363000AF909F908F907F906F905F904F90089584
:1036400060E0C8010E948443DC011996AD90BC90F3
:103650001A9761E0C8010E948443FC01818492842E
:10366000F2E06F16710409F47BC162E0C8010E94A8
:103670008443DC011996CD90DC901A97B3E06B1669
:10368000710409F471C163E0C8010E948443FC0124
:10369000E184F284F4E06F16710451F064E0C80133
:1036A0000E948443DC0119960D911C911A9703C066
:1036B0008E01075F1F4F9092F3098092F209D0921A
:1036C000F509C092F40965ED75E086EA98E00E947C
:1036D0008E11B40186EA98E00E94D71263ED75E07E
:1036E00086EA98E00E948E114AE050E0B60186EA30
:1036F00098E00E9456126CEC75E086EA98E00E9411
:103700008E11B70186EA98E00E94D71267EC75E047
:1037100086EA98E00E948E110E947D2B8111E4C000
:103720006091F2097091F30980915D0990915E09B1
:103730004091F4095091F509DC01ED91FC9161157E
:10374000710521F00088F189E02D16C00684F78507
:10375000E02D23EA33E03A8329834090EE0950902C
:10376000EF096090F0097090F1094B825C826D82E4
:103770007E82BE016F5F7F4F19958130910509F000
:10378000ACC09093E0098093DF0987E0E5E3F2E0C5
:10379000DE01119601900D928A95E1F7FE013196B6
:1037A000A4E6B9E06E0128E0C20ED11C81918D9390
:1037B000EC15FD05D9F7E114F10429F00115110507
:1037C00021F082EC03C082E001C082E880936B09A3
:1037D00010926C098FE080936D094FE050E06FE527
:1037E00079E0C5010E94EB2AE114F10479F0AC0103
:1037F0006FE579E0C7010E94EB2A0115110531F050
:10380000AC016FE579E0C8010E94EB2AAC0145509C
:1038100051096FE579E080E10E940C2BADD86093EF
:10382000E1097093E2098093E3099093E4096093BE
:10383000E5097093E6098093E7099093E809809180
:103840005D0990915E09DC01ED91FC910084F185A8
:10385000E02D1995892BB9F48FD80091E5091091C5
:10386000E6092091E7093091E809DC01CB01801BD2
:10387000910BA20BB30B88399A43A105B105F8F25D
:103880008CEF9FEF1AC0C6010E94D5470497C9F478
:1038900080916209811110C06FD86093E50970931F
:1038A000E6098093E7099093E8091092E9091092DC
:1038B000F9091092F80918C090E09093F9098093E3
:1038C000F80980915D0990915E09DC01ED91FC9110
:1038D0000488F589E02D19951BC08EEF9FEF90931A
:1038E000F9098093F80914C069EB75E086EA98E05D
:1038F0000E948E11B50186EA98E00E94B71287E215
:1039000094E00E94222D0E94A94983E090E03DCDE1
:103910006DEA75E086EA98E00E948E116091F809E0
:103920007091F9094AE050E086EA98E00E94561248
:1039300065E975E086EA98E00E94C7121DD8DC01AF
:10394000CB0188579C4EAF4FBF4F80930208909396
:103950000308A0930408B093050884EF9FEF15CDEA
:103960008BE5C82E87E0D82E7E0129E0E20EF11CFF
:103970008701A1CE85ED8093BC008091BC0084FDC1
:10398000FCCF1092BA07089540916F06262F30E0C1
:10399000240F311D21323105DCF42091BA07243087
:1039A000C9F4FC0180E090E0861758F430916F066E
:1039B0002191DC01A35BB94FA30FB11D2C9301969C
:1039C000F3CF80916F06680F60936F0680E00895D3
:1039D00081E0089582E008950895E0912C06809199
:1039E0002B06E81730F4F0E0E35DF94F808190E0BA
:1039F00008958FEF9FEF089590912C0680912B06EC
:103A0000981750F4E92FF0E0E35DF94F208130E0A2
:103A10009F5F90932C0602C02FEF3FEFC9010895DE
:103A200080912B0690E020912C06821B910908952D
:103A3000CF92DF92EF92FF920F931F93CF93DF937A
:103A40007C01262F972F8A018091BB07882391F054
:103A5000C62FD72F6E01C40ED51ECC15DD0569F01B
:103A60006991D701ED91FC910190F081E02DC701A2
:103A70001995F3CF642F822F87DFC801DF91CF9193
:103A80001F910F91FF90EF90DF90CF900895CF930B
:103A9000DF931F92CDB7DEB769832091BB07222346
:103AA000D1F02091DE07203240F021E030E0FC012F
:103AB0003383228380E090E014C08091BC07E82F1C
:103AC000F0E0E354F84F998190838F5F8093BC07B7
:103AD0008093DE0704C061E0CE01019655DF81E0EE
:103AE00090E00F90DF91CF9108950895EF92FF92AB
:103AF0000F931F93CF93DF93009719F48FEF9FEFEE
:103B000086C0FC01E484F584D7010D911C91D80195
:103B1000ED91FC910688F789E02DC801199588235D
:103B200069F3D801ED91FC910084F185E02DC80185
:103B30001995D801ED91FC91892B61F30284F385ED
:103B4000E02DC8011995EC010196C1F2F8018589B3
:103B5000882349F04C2F50E060E070E02AE086EACC
:103B600098E00E94C711D70112968C91882309F41E
:103B70004DC0C532D10509F049C0D801ED91FC9185
:103B80000084F185E02DC801199502975CF0D801F9
:103B9000ED91FC910688F789E02DC80119958111F6
:103BA000ECCFACCFD1E0C0E0D801ED91FC91028424
:103BB000F385E02DC80119958F3FBFEF9B0709F4EE
:103BC0009DCF9C01215431092A31310530F09C01EF
:103BD000215631092A31310538F48D2F8295807FA5
:103BE000829FC00D11240AC0C0978A30910530F41D
:103BF0009D2F9295907F989FC00D1124DD2311F089
:103C0000D0E0D2CF8C2FCC0F990B01C0CE01DF9129
:103C1000CF911F910F91FF90EF900895FC0181814A
:103C20009091BA079111FCCF91E09093BA079093CD
:103C3000B9072FEF2093B8071092B7071092B60775
:103C40009093950790919507880F892B80939507FE
:103C500080919407813061F41092940780919507C8
:103C60008093BB008091BC0083FDF8CF85EC01C040
:103C700085EE8093BC008091BA078130E1F380919A
:103C8000B707811103C08091B70701C081E0A6E9A1
:103C9000B7E02DE236E0F9019E2F921B981718F439
:103CA0009D919193F9CF10922C0680932B0683E47B
:103CB00099E0A2CE08951F920F920FB60F92112491
:103CC0000BB60F922F933F934F935F936F937F9316
:103CD0008F939F93AF93BF93EF93FF938091B9001E
:103CE000887F803609F49CC068F5883209F45BC08F
:103CF00090F4803109F454C038F4882309F4F6C0F4
:103D0000883009F44DC0F5C0883109F44CC08032C8
:103D100009F45DC0EEC0803409F468C048F4803313
:103D200009F455C0883309F0E4C08093B807D8C0BF
:103D3000803509F44FC0883509F45DC0883409F036
:103D4000D8C0D6C0883909F4C7C0A8F4883709F4A8
:103D500067C038F4883609F463C0803709F460C05E
:103D6000C8C0883809F4B8C0803909F45FC0803809
:103D700009F0BFC05BC0803B09F486C038F4803ACC
:103D800009F466C0883A09F47FC0B3C0803C09F4E6
:103D9000A7C0883C09F4A4C0883B09F48AC0A9C024
:103DA0008091950710C09091B7078091B60798173A
:103DB00070F5E091B70781E08E0F8093B707F0E0D0
:103DC000EA56F84F80818093BB0085EC86C08093D3
:103DD000B8078EC0E091B70781E08E0F8093B707D8
:103DE0008091BB00F0E0EA56F84F80839091B707CE
:103DF0008091B6076EC0E091B70781E08E0F809387
:103E0000B7078091BB00F0E0EA56F84F80838091BD
:103E1000B90781116DC081E08093940784EA61C085
:103E200083E08093BA0710929306CFCF80919306D8
:103E3000803208F051C0E091930681E08E0F8093AC
:103E400093068091BB00F0E0ED58F94F8083BDCF21
:103E500085EC8093BC001092BA0780919306803263
:103E600030F4E0919306F0E0ED58F94F1082609144
:103E7000930670E0E0917106F091720683E796E098
:103E800019951092930635C084E08093BA0710927A
:103E9000700610926F06E0916D06F0916E0619950E
:103EA00080916F06811105C081E080936F061092AA
:103EB0004D06E091700681E08E0F80937006F0E071
:103EC000E35BF94F80818093BB00909170068091F5
:103ED0006F06981708F479CF85E88093BC0009C075
:103EE00085EC8093BC001092BA0703C01092B8070B
:103EF00041DDFF91EF91BF91AF919F918F917F91A4
:103F00006F915F914F913F912F910F900BBE0F904A
:103F10000FBE0F901F9018951092BA0781E0809302
:103F2000B9071092940761E084E10E94191461E0DE
:103F300085E10E941914E9EBF0E080818E7F808397
:103F400080818D7F808388E48093B80085E48093AE
:103F5000BC000895DC01E0E0615038F08D91E82765
:103F6000F0E0E75DF94FE491F7CF8E2F089581E0FF
:103F70000C945F2DFC01818191E09093BB078093AD
:103F8000DD071092BC071092DE0708951F93CF93B0
:103F9000DF93EC01162FEEDF61EE83E499E077DD2D
:103FA000612F83E499E073DDCE01DF91CF911F9102
:103FB000DECFAF92BF92CF92DF92EF92FF921F932C
:103FC000CF93DF93EC010E94BC146B017C0128EEBF
:103FD000C20E23E0D21EE11CF11C8BE4A82EB12CF2
:103FE0000E94BC146C157D058E059F0588F460EF5A
:103FF000CE01CCDFCE0112DE182F80FF11C0EF857D
:10400000F889309709F01995C5010197F1F7E8CFC4
:1040100081E08A8364E374E086EA98E00E94B71244
:10402000812FDF91CF911F91FF90EF90DF90CF9084
:10403000BF90AF9008951F93CF93DF93EC01162F9D
:10404000B8DFCE0197DF62ED83E499E020DD212F18
:1040500030E02095309584E0220F331F8A95E1F7F8
:10406000612F622B83E499E012DDCE0180DFCE0167
:10407000D5DD811711F084E08A83DF91CF911F9104
:104080000895CF93DF93EC0163EC80DFCE01DF91E5
:10409000CF91C4CD1F93CF93DF93EC018ADFCE0184
:1040A000F0DF60E0CE01C7DFCE0183DFCE0162DF4B
:1040B00064EB83E499E0EBDCCE0159DFCE0179DFDC
:1040C000182F82FF02C082E08A838881882331F022
:1040D000CE01D7DF682F6160CE01ADDF11FB8827ED
:1040E00080F9DF91CF911F910895CF93DF93EC0179
:1040F000C8DF682F6460CE01DF91CF919CCFEF9233
:10410000FF921F93CF93DF931F92CDB7DEB77C0151
:10411000162F49834EDF4981442311F0C701E5DFA3
:10412000C70128DF65EA83E499E0B1DC612F83E40D
:1041300099E0ADDCC7010F90DF91CF911F91FF9007
:10414000EF9015CF6F927F928F929F92AF92BF9216
:10415000CF92DF92EF92FF920F931F93CF93DF9353
:10416000FC012485211196C0872E762EEC0192DF6A
:10417000811108C06FE374E086EA98E00E94B712EC
:104180008FEF89C0CE0115DF40E060EFCE01B7DFD1
:10419000E12CF12C66246A94CC24C394D12C0E2DEE
:1041A00006950695069510E08E2D8770560101C084
:1041B000AA0C8A95EAF78B85082E000C990BE81655
:1041C000F90634F4FE01E00FF11F93809A2006C037
:1041D00099249394E816F90609F0912CCE01E9DEB2
:1041E000CE01C8DE68E783E499E051DC911002C09B
:1041F00060E001C060E883E499E049DCCE01B7DE0D
:10420000CE01D7DE282F2074982F907885FF13C019
:104210002223B9F0482F50E060E070E022E086EA07
:1042200098E00E94C7116BE474E086EA98E00E946F
:10423000B7128EEF30C0211104C0911104C06E2C52
:1042400008C0992331F0FE01E00FF11F8381A82AF5
:1042500006C0FE01E00FF11FA0948381A822A38273
:10426000FFEFEF1AFF0A80E4E816F10409F097CF98
:104270006B86EFEF6E1202C081E08C87DE01139631
:10428000E72DF82D2B968D918193AC17BD07D9F7AB
:1042900081E001C080E0DF91CF911F910F91FF90ED
:1042A000EF90DF90CF90BF90AF909F908F907F90D6
:1042B0006F900895CF92DF92EF92FF920F931F932A
:1042C000CF93DF931F92CDB7DEB78C01F62E40E07F
:1042D00065E5798314DFCF2C7981D72E760188E0CC
:1042E000E80EF11CF60161916F0140E0C80107DFA3
:1042F000CE14DF04B9F70F90DF91CF911F910F918A
:10430000FF90EF90DF90CF900895AF92BF92CF9241
:10431000DF92EF92FF920F931F93CF93DF931F9241
:104320001F92CDB7DEB77C018A01FC0185819681A1
:1043300069837A83AFDE69817A81882381F1F7010D
:1043400085819681B7DF40E06EEBF701858196812C
:10435000D6DE58016801F9E0CF0ED11CF7010581C6
:104360001681C80126DEC80105DE66E983E499E00E
:104370008EDBC801FCDDC8011CDE61EEC80106DE73
:10438000C8014CDCF50181935F01EC15FD0531F7A7
:10439000F701858196817EDE91E0813009F090E021
:1043A000892F0F900F90DF91CF911F910F91FF9068
:1043B000EF90DF90CF90BF90AF900895CF93DF93B1
:1043C000EA01A3DF882331F068E0CE01C3DD91E08C
:1043D0002885821390E0892FDF91CF910895CF93A4
:1043E000DF93CDB7DEB729970FB6F894DEBF0FBEC7
:1043F000CDBFAE014F5F5F4FE1DF882389F08D8134
:104400008F3361F020F48F3159F489E00CC08F357F
:1044100019F08F3739F004C08BE005C08AE003C083
:1044200080E001C08CE029960FB6F894DEBF0FBE85
:10443000CDBFDF91CF9108950F931F93CF93DF935B
:104440000097B9F0EC010C851D85D8018D919C91E8
:10445000DC01ED91FC910488F589E02D1995C801E6
:104460000E94575ACE01DF91CF911F910F910C946A
:10447000A25BDF91CF911F910F910895FB012481E1
:104480003581428153812417350758F44081518189
:10449000DA01A20FB31F8C938481958101969583D5
:1044A000848380E00895CF93DF93EC01E881F98164
:1044B0000284F385E02DCE0119950196B9F7DF91BD
:1044C000CF910895FC01A285B3851097A9F0868548
:1044D0009785029788F0CD010196938782876C9328
:1044E000868597850197978786870284F385E02DD7
:1044F000108281E090E0089580E090E00895FC0152
:10450000868197818F3F2FEF920729F02FEF3FEFA2
:10451000378326830895A085B185109789F0248577
:1045200035852115310561F0CD0101969187808790
:104530008C912150310935872487082E000C990B66
:104540000895FC0186819781019639F481E02485E4
:104550003585232B19F480E0089581E00895CF92EA
:10456000DF92EF92FF920F931F93CF93DF937C0123
:104570006A018B01C0E0D0E0CC15DD0589F0D701E0
:10458000ED91FC910284F385E02DC70119958F3FD1
:10459000BFEF9B0729F0F80181938F012196ECCFA3
:1045A000CE01DF91CF911F910F91FF90EF90DF909F
:1045B000CF900895CF93DF931F92CDB7DEB7DC0184
:1045C000ED91FC910088F189E02D69831995DC015A
:1045D000ED91FC910190F081E02D69810F90DF91C8
:1045E000CF911994CF93DF93FC01268137812F3F20
:1045F0003F4FF9F4EC01288539858A859B85820F28
:10460000931F8115904198F4E881F9810284F38524
:10461000E02DCE011995813291056CF3E881F98185
:104620000684F785E02D682FCE01199502C080E041
:1046300001C081E0DF91CF910895062E000C770B29
:10464000FC01778366830895CF93DF93DC01169690
:104650002D913C9117972F3F3F4F31F5EC01E881A9
:10466000F9810088F189E02DCE011995DC01ED91E9
:10467000FC910084F185E02D1995892B99F0E88152
:10468000F9810284F385E02DCE01199581329105DF
:1046900034F3E881F9810684F785E02D682FCE0197
:1046A000199502C080E001C081E0DF91CF910895AB
:1046B000FC018481958108950F931F93CF93DF931D
:1046C000EC018B0165E574E00E94D712011511051C
:1046D000B9F1F80161918F01662391F1603220F008
:1046E000623211F06C3541F56CE5CE010E94871104
:1046F000F801319780818C30D1F044F48930D9F0C1
:104700008A30B9F0883029F762E616C0823259F053
:1047100024F48D30F1F662E70FC08F3231F08C3522
:10472000C1F66CE509C062E207C06FE205C066E64B
:1047300003C06EE601C064E7CE010E948711C9CFB5
:1047400062E2CE010E94871180E090E0DF91CF917C
:104750001F910F910895AF92BF92CF92DF92EF9287
:10476000FF920F931F93CF93DF9300D01F92CDB78B
:10477000DEB76115710509F493C06B01182FDB01D9
:104780001C96AD90BC901D97F501E080F180D7019B
:10479000ED91FC910688F789E02DC70119958111EB
:1047A00003C0C60149DE7CC0F5019281911114C09D
:1047B000D701ED91FC910190F081E02D612FC701AF
:1047C0001995F7018589882309F467C0612F86EA66
:1047D00098E00E94871161C0812F8F7D81548A31BA
:1047E00038F380ED810F8A3018F383ED810F82302A
:1047F000F8F21F35E9F21E37D9F21132B1F086EC2A
:10480000810F823090F08AED810F873070F01D3378
:1048100061F0812F8F7E8F3241F08DED810F8230DC
:1048200020F01B3511F01D3511F491FFC1CF198215
:104830001A821B821C82812F012E000C990B9F93E0
:104840001F9387E594E09F938F938E010F5F1F4F17
:104850001F930F930E9428670F900F900F900F9057
:104860000F900F9083E0D82ED00ED701ED91FC91E0
:104870000190F081E02DD8016C91C7011995F701E5
:104880008589882331F0D8016C9186EA98E00E94EE
:1048900087110F5F1F4FD012E8CF80E090E002C079
:1048A0008FEF9FEF0F900F900F900F90DF91CF91B0
:1048B0001F910F91FF90EF90DF90CF90BF90AF903E
:1048C0000895FC012085318582859385AC014F5F79
:1048D0005F4F53874287820F931F0E94296281E0B6
:1048E00090E00895FC01868197818F3F2FEF92071A
:1048F00029F02FEF3FEF37832683089520853185F8
:1049000082859385AC014F5F5F4F53874287820F4B
:10491000931F0E942162082E000C990B0895FC0140
:10492000868197818F3F2FEF920729F02FEF3FEF7E
:10493000378326830895808591850C94025CCF92FD
:10494000DF92EF92FF92CF93DF93EC018E819F81F4
:104950008F3F2FEF920759F02FEF3FEF3F832E83CA
:10496000DF91CF91FF90EF90DF90CF9008950E945C
:10497000BC146B017C01A4EFCA0EA1E0DA1EE11C9D
:10498000F11CE881F9810088F189E02DCE011995AB
:10499000DC01ED91FC910084F185E02D1995892BC6
:1049A00039F40E94BC146C157D058E059F0548F3F3
:1049B000E881F9810088F189E02DCE011995DC01AB
:1049C000ED91FC910284F385E02DDF91CF91FF9072
:1049D000EF90DF90CF901994CF92DF92EF92FF92F9
:1049E0000F931F93CF93DF938C017B0186E090E0C0
:1049F0000E94C259EC019093330580933205F8016F
:104A000001900020E9F7CF01801B910B0E94C25951
:104A10006C01B8010E94AC66F80101900020E9F732
:104A20003197E01BF10BEC0DFD1D1082D982C8827D
:104A3000FB82EA8280912A0590912B059D838C83CD
:104A4000D0932B05C0932A05DF91CF911F910F9131
:104A5000FF90EF90DF90CF9008958F929F92AF924A
:104A6000BF92CF92DF92EF92FF920F931F93CF935B
:104A7000DF936115710509F4FBC0FB010085002E71
:104A8000000C110B220B330B0730110508F0F0C09E
:104A9000DB01EC01F8018827EC53FF4F8F4F0C949A
:104AA00027666DE574E006C019968C91882389F01D
:104AB00062E674E0CE01DF91CF911F910F91FF90DC
:104AC000EF90DF90CF90BF90AF909F908F900C941D
:104AD000B21167E674E0EECF19964D915D916D913C
:104AE0007C911C972AE030E0CE01DF91CF911F919D
:104AF0000F91FF90EF90DF90CF90BF90AF909F907D
:104B00008F900C940F121996CD90DD90ED90FC9043
:104B10001C9720E030E0A901C701B6010E94F962AC
:104B200087FF09C06DE674E0CE010E94D712F7FA44
:104B3000F094F7F8F094C701B6010E946A634B0144
:104B40005C012AE0AB01BC01CE010E94C7116FE6F7
:104B500074E0CE010E94D712C501B4010E94966391
:104B60009B01AC01C701B6010E9494622DEC3CECA4
:104B70004CE45DE30E94956220E030E040E251E4C5
:104B80000E944C640E946A63AB0160E070E02AE01E
:104B9000CE010E94C7116CC019966D917C911A9735
:104BA000CE01DF91CF911F910F91FF90EF90DF9099
:104BB000CF90BF90AF909F908F907ECD16960D9125
:104BC0001C9117976BE5CE010E948711019619F48D
:104BD0008FEF9FEF4FC00115110569F0B801CE01AD
:104BE0003CDF0196A9F3F80102811381011511053B
:104BF00091F36CE2E8CF6DE52DC016960D911C91F6
:104C000017976BE7CE010E948711019609F30115F2
:104C10001105F9F0F80160817181CE014DDD019639
:104C2000B9F26AE3CE010E948711019689F2B801B8
:104C3000CE0113DF019661F2F801028113810115A3
:104C4000110529F36CE2CE010E9487110196F9F655
:104C5000BFCF6DE7CE010E94871121E030E00196C1
:104C600011F020E030E088279927821B930B02C0C7
:104C700080E090E0DF91CF911F910F91FF90EF9036
:104C8000DF90CF90BF90AF909F908F900895CF937B
:104C9000DF93EC01E881F9810284F385E02DCE01F8
:104CA00019958F3F2FEF920771F0E881F9818132DA
:104CB000910594F30684F785E02D682FCE011995B0
:104CC00080E090E002C08FEF9FEFDF91CF910895D9
:104CD000EF92FF920F931F93CF93DF938C017B0191
:104CE000DC01ED91FC910284F385E02D199582970A
:104CF00049F584E0F701808786E090E00E94C25980
:104D0000EC01892BF9F0E4E9F6E0F983E88380E02F
:104D100091E0DF019C011D9221503040E1F79B831F
:104D20008A831D821C82D801ED91FC910284F38557
:104D3000E02DC80119958F3FBFEF9B0731F4CE01DD
:104D40000E94575A8FEF9FEF70C08232910509F48D
:104D500049C0803291050CF445C08C35910511F0A5
:104D6000BE013EC0D801ED91FC910284F385E02D97
:104D7000C80119958F3FBFEF9B0709F38236910554
:104D800039F15CF48F32910501F18C359105D1F048
:104D9000829749F6BE0182E223C08E369105D9F092
:104DA0003CF48636910509F0BECFBE018CE018C0F8
:104DB0008237910599F08437910509F0B4CFBE018F
:104DC00089E00EC0BE018CE50BC0BE018FE208C0B9
:104DD000BE0188E005C0BE018AE002C0BE018DE0D0
:104DE0004DDBA1CF8C819D81009749F0E881F9814D
:104DF0008E0F9F1FFC0131978081882319F0BE011F
:104E000080E03CDB8C819D810E94C2598C0100971F
:104E100039F064E976E00E94AC66CE010E94575AF0
:104E2000F7011287018780E090E0DF91CF911F9119
:104E30000F91FF90EF9008958DE090E00E94C2598D
:104E4000009729F02DE0FC0111922A95E9F70895C9
:104E50002C9A08952C9808951F93CF93DF93182FC1
:104E600066E270E00E943A30C82FD0E067E270E05E
:104E7000812F0E943A30DC2FCC279E01282BC901BC
:104E8000DF91CF911F9108951F93CF93DF93182F38
:104E900060E270E00E943A30C82FD0E061E270E03A
:104EA000812F0E943A30DC2FCC279E01282BC9018C
:104EB000DF91CF911F9108958EBD00000DB407FEC4
:104EC000FDCF8EB50895CF92DF92EF92FF920F93B0
:104ED0001F93CF93DF93EC017A018B016C01C40E19
:104EE000D51ECC15DD0579F0B5DF8FE0E5DF8D2F20
:104EF000E3DF8C2FE1DF219680E0DEDFF801819394
:104F00008F01A6DFEECFC701DF91CF911F910F91E7
:104F1000FF90EF90DF90CF900895CF92DF92EF92C5
:104F2000FF920F931F93CF93DF93EC017A018B01D4
:104F30006C01C40ED51ECC15DD0571F08BDF80EF42
:104F4000BBDF8D2FB9DF8C2FB7DF2196F801819160
:104F50008F01B2DF7DDFEFCFC701DF91CF911F91CE
:104F60000F91FF90EF90DF90CF9008951F93CF9314
:104F7000DF931F921F92CDB7DEB7182F6A839983F4
:104F800069DF80EF99DF9981892F96DF812F94DF88
:104F90006A81862F91DF5CDF81E00F900F90DF91B7
:104FA000CF911F910895CF92DF92EF92FF920F93CE
:104FB0001F93CF93DF938C017B016A013DDFEC01EE
:104FC000892B09F182E08887A601DD0C660B770B3F
:104FD00049875A876B877C8788819981009711F070
:104FE0000E94575AC7010E94546699838883BE0164
:104FF000C801DF91CF911F910F91FF90EF90DF904B
:10500000CF900C94CF43DF91CF911F910F91FF90E0
:10501000EF90DF90CF9008958F929F92AF92BF92C2
:10502000CF92DF92EF92FF920F931F93CF93DF9374
:10503000CDB7DEB7C150D1400FB6F894DEBF0FBE7A
:10504000CDBF282F8091FC0989832A83213090F0DD
:10505000253010F0273171F48091FD099091FE09FF
:105060009B838C838091FF099091000A9D838E839E
:1050700096E001C092E08E010F5F1F4F213120F4B6
:105080002F3030F48BEF01C08AEE820F823078F43B
:105090003091810A8091820AF801E90FF11D808325
:1050A00081E0890FF801E80FF11D9E5F30832F30FA
:1050B00021F150F4253091F0263009F0B1C0309143
:1050C000850A8091860A0EC0263109F48AC02731EC
:1050D00009F458C0203109F0A3C054C03091830AAC
:1050E0008091840AF801E90FF11D808381E0890F26
:1050F000F801E80FF11D9E5F92C04091830A509124
:10510000840AF801E90FF11D508382E0890F31E034
:10511000390FF801E30FF11D4083BA01677077275B
:10512000A3E056954795AA95E1F7672B19F031E072
:10513000340F01C0342FB3E0B90FF801E80FF11DAF
:105140003083A4E0A90F60E070E04FEF4A0F6317CF
:10515000B0F450E0CB0195958795400F511F880F13
:10516000991FFC01EB57F54F60FD02C0808101C023
:105170008181FA0180836F5F7F4FAF5FE6CF9B2F06
:10518000930F4EC03091830A8091840AF801E90F91
:10519000F11D808381E0890FF801E80FF11D308354
:1051A00063E0690F9E5FF801E90FF11D932F990FDE
:1051B0009083E5E8FAE0862F40E0431780F47081A1
:1051C00051813296D801A80FB11D5C9351E0580F60
:1051D000D801A50FB11D8E5F7C934F5FEECF960F68
:1051E0001FC08091850A3091860AF801E90FF11DF0
:1051F000308331E0390FF801E30FF11D80833091E6
:10520000870A8091880A42E0490FF801E40FF11DF6
:10521000808383E0890FF801E80FF11D9C5F3083E4
:105220007801F8014FEF5FEFD02E8E2F801B89178A
:10523000A0F48191482768E070E0DA01B695A7955F
:1052400040FF06C0AD0131E0432730EA532701C0DB
:10525000AD016150710989F7E8CFF801E90FF11D3F
:10526000408332E0C32EC90E9F5FF801E90FF11DA4
:105270005083F801EC0DF11D10828091FA09909194
:10528000FB09DC01ED91FC910284F385E02DCF5FF9
:10529000DE4F2883C150D1401995CF5FDE4F288162
:1052A000C150D140019649F7E091100BF091110BDC
:1052B000309731F01995CF5FDE4F2881C150D14032
:1052C000A091FA09B091FB099E2D9D199C1588F4B7
:1052D000F70161917F01ED91FC9111970190F081AF
:1052E000E02DCD01CF5FDE4F2883C150D14019950D
:1052F000E2CFED91FC9111970680F781E02DCD0171
:10530000CF5FDE4F2883C150D1401995E091120B39
:10531000F091130BCF5FDE4F2881C150D140309701
:1053200031F01995CF5FDE4F2881C150D140CF5F5A
:10533000DE4F2883C150D1400E94BC144B015C0158
:1053400028E0D22EC12CCF5FDE4F2881C150D14042
:10535000E22EF12C8091FA099091FB09DC01ED918C
:10536000FC910084F185E02D1995892BC1F0809185
:10537000FA099091FB09DC01ED91FC910284F3851F
:10538000E02D19959091FC09891711F0CC2099F125
:10539000F801EC0DF11D8083DA94C39407C0E0910D
:1053A0000E0BF0910F0B309709F01995B5E0CB1269
:1053B00022C0EA818E2F8F7790E08E159F0509F02D
:1053C000A3C0E7FF04C08B81882349F181C08E2FE1
:1053D00090E0FC013197E731F10568F48827E55347
:1053E000FF4F8F4F0C94276693E0D92E04C0DB80CB
:1053F00002C085E0D82E0E94BC14DC01CB018819C4
:105400009909AA09BB09813D9740A105B10508F09A
:10541000D2C0D1109FCFF4E0FC1508F079C0AFEFF7
:10542000BFEF40E0D12CC6010297242F30E02817AF
:105430003907C4F4200F311FF9012081A22728E089
:1054400030E0BD0176956795A0FF06C0DB01F1E075
:10545000AF27F0EABF2701C0DB012150310989F7EE
:105460004F5FE3CF800F911FFC0180818A134EC0F4
:10547000F601EC0FFD1F80818B1348C049C04034FA
:10548000D8F4880F991FFC01E650F64FA5E0B0E074
:10549000AC0FBD1FA80FB91F2C9130E0322F22276F
:1054A000A4E0B0E0AC0FBD1FA80FB91F8C91D901CB
:1054B000A82BCD0190878783242F4F5F842F90E006
:1054C00086179707E4F220930D0B50FD61C080E032
:1054D0001092070B1092090B1092080B10920C0BF4
:1054E000CF5FDE4F0FB6F894DEBF0FBECDBFDF91AA
:1054F000CF911F910F91FF90EF90DF90CF90BF90D1
:10550000AF909F908F90089581EEE2CF83EEE0CF31
:105510008A81853028F4833028F4813080F5D7CF14
:105520008731A9F68B8190E0AC0155954795309174
:105530000D0B20E0822F90E084179507ECF42034C7
:10554000C0F4FC013296EE0FFF1F880F991FBC01BB
:105550006650764FCE018E0F9F1FDC018C9190E03C
:10556000982F8827E00FF11F3081832BFB01908754
:105570008783322F2F5FDECF30930D0BA8CF5B8157
:10558000652F70E07595679520910D0B40E096CFE3
:10559000403468F4880F991FFC01E650F64FD8019B
:1055A000A80FB91F13968C9190E0908787834F5F67
:1055B00040930D0B8CCF82EE8BCFDC011696ED91D4
:1055C000FC91179780E0309729F08F5F0280F3817C
:1055D000E02DF9CF0895CF93DF93DC014E5F5F4F4D
:1055E000FC019F012A1B3B0B9191992339F0EB01A0
:1055F000C40FD51F98834F5F5F4FF3CFCA01821B43
:10560000930B680F791FFB0132973083319620830B
:10561000CA01DF91CF910895CF92DF92EF92FF926E
:105620000F931F93CF93DF9300D01F92CDB7DEB7B8
:105630009A01E0E0922F9F77220F232F221F330B36
:1056400031952115310509F0906801E00E0FA1E0B8
:10565000B0E0AC0FBD1FAE0FB11DFD019083211551
:10566000310511F0E02FE6CF10E0DB01A01BB10BFC
:1056700014968C93FE0131966F0180E090E08017C4
:10568000910764F4F601F1906F019C01201B310B2E
:10569000260F371FF901F5820196F1CF80915D0940
:1056A00090915E094F5F5F4F040F151FFC01208131
:1056B0003181F90122813381A801BD01F9011995D8
:1056C0007C010E94BC146093E1097093E20980930D
:1056D000E3099093E40981E0E016F10609F080E027
:1056E0000F900F900F900F90DF91CF911F910F911E
:1056F000FF90EF90DF90CF90089580915D09909199
:105700005E09009759F1DC01ED91FC910688F7895B
:10571000E02D1995811124C08091F8099091F90923
:10572000892BE1F48DEF9FEF9093F9098093F809AD
:1057300080915D0990915E09DC01ED91FC910680FC
:10574000F781E02D199580915D0990915E09DC014A
:10575000ED91FC910488F589E02D199580E008957C
:1057600081E00895EF92FF920F931F93CF93DF9301
:105770007C018B01EB0109900020E9F72197C61B02
:10578000D70BBBDF8823A1F1F70101900020E9F7D7
:105790003197EE19FF09CE010796E80FF91FE1389E
:1057A000F10530F545E050E06FE579E0C70113DF22
:1057B000F80120E030E02C173D0759F04191D90164
:1057C000A80FB91FA35AB64F12964C932F5F3F4FA5
:1057D000F2CF25503109A901480F591F6FE579E033
:1057E00080E3DF91CF911F910F91FF90EF9014CF45
:1057F00080E0DF91CF911F910F91FF90EF9008957E
:10580000CF92DF92EF92FF920F931F93CF93DF938C
:1058100000D01F92CDB7DEB78C017B0129833A837C
:105820004B835C8309DB6C0129813A814B815C816C
:10583000892B19F183E0F60180872187328743871E
:10584000548780819181009711F00E94575AC701B7
:105850000E945466F60191838083B601C8010F90BF
:105860000F900F900F90DF91CF911F910F91FF90AC
:10587000EF90DF90CF900C94CF430F900F900F904C
:105880000F90DF91CF911F910F91FF90EF90DF90DC
:10589000CF900895EF92FF920F931F93CF93DF93D2
:1058A000CDB7DEB760970FB6F894DEBF0FBECDBFA1
:1058B0007C0180E091E00E94C2598C01892BD1F0DB
:1058C0001C821B821E821D828FEF9FEF98878F8321
:1058D00080E492E09A8389831A8619861C870B8755
:1058E00080E091E0988B8F871E861D86B701CE01E0
:1058F0000196B3D8C80160960FB6F894DEBF0FBE0C
:10590000CDBFDF91CF911F910F91FF90EF90089540
:105910000F931F93CF93DF93EC012097F1F00A814F
:105920001B81888587FD05C08E819F81009709F0C6
:10593000EFDF8885843031F489859A85009711F0EE
:105940000E94575A88819981009711F00E94575AF6
:10595000CE010E94575AE801E0CFDF91CF911F910D
:105960000F910895CF93C82F462F61E070E078D350
:1059700061E070E08C2F7ED38111FACFCF91089532
:105980008F929F92AF92BF92CF92DF92EF92FF924F
:105990000F931F93CF93DF93B82E4B018A01A22E52
:1059A00068E270E067D3C82FD0E069E270E08B2D29
:1059B00061D3DC2FCC27C82B9E013770CB2CD12C88
:1059C000C601880F991FAC014951584F6A01FA016D
:1059D00080819181820F931FA801420F531F413094
:1059E000584090F060E078E07B01E21AF30AA701EA
:1059F000B40169DAA8014E195F09B4016E0D7F1D6B
:105A0000F6018081918102C0A801B4015CDAA11085
:105A10000CC0C00FD11F4D2F68E270E08B2D20D33A
:105A20004C2F69E270E08B2D1BD3DF91CF911F913A
:105A30000F91FF90EF90DF90CF90BF90AF909F902D
:105A40008F900895CF93DF93FC0101900020E9F738
:105A50009F01281B390B285F3F4F2138310558F52E
:105A6000EC014BDE882339F18091DF099091E00948
:105A7000019611F481E090E09093E0098093DF09B2
:105A80008091DF099091E009909364098093650902
:105A900047E050E06FE579E0CE019DDDFC01E35A7F
:105AA000F64F1282AC01445051096FE579E082E86B
:105AB000DF91CF91B1CD80E0DF91CF910895382F64
:105AC0002091DE079091DD07213208F049C08091D6
:105AD000BA078111FCCF42E04093BA073093B9076F
:105AE0003FEF3093B8071092B7072093B607ADEB9E
:105AF000B7E046E957E0FA013E2F341B321718F49D
:105B00003D913193F9CF1092950720919507990F08
:105B1000922B9093950790919407913061F4109295
:105B20009407909195079093BB009091BC0093FDD2
:105B3000F8CF95EC01C095EE9093BC009091BA0718
:105B40009230E1F39091B8079F3F79F08091B807C8
:105B5000803241F08091B807803331F084E005C095
:105B600081E003C082E001C083E01092BC07109284
:105B7000DE071092BB070895DF92EF92FF920F931A
:105B80001F93CF93DF93CDB7DEB729970FB6F89465
:105B9000DEBF0FBECDBF8C017B01AE014F5F5F4FFB
:105BA0000E94DE21D82E882309F459C0F701808194
:105BB000803109F454C08FE18D83F801858196818D
:105BC0000E944A20B701F801858196810E945A21DE
:105BD00040E06EE4F801858196810E947F2040E0DC
:105BE0006B81F801858196810E947F2040E06C8165
:105BF000F801858196810E947F20F70180818031A4
:105C000039F040E06D81F801858196810E947F2006
:105C1000F801858196810E944A20B701F8018581AB
:105C200096810E945A21F801408168E4858196811D
:105C30000E947F2064E170E080E090E00E94841484
:105C4000F8018081882331F06AE070E080E090E024
:105C50000E948414F801858196810E944A208D2D2E
:105C600029960FB6F894DEBF0FBECDBFDF91CF915E
:105C70001F910F91FF90EF90DF900895EF92FF92A8
:105C80000F931F93CF93DF93EC018C01085F1F4F9D
:105C90007E01699170E084E0759567958A95E1F7DA
:105CA00040E150E086EA98E00E945612F7016081D8
:105CB0006F7070E040E150E086EA98E00E94561272
:105CC000C017D10729F7DF91CF911F910F91FF9056
:105CD000EF900895CF93DF931F92CDB7DEB769831E
:105CE000DC01ED91FC910280F381E02D41E050E078
:105CF000BE016F5F7F4F19950F90DF91CF9108958F
:105D0000FC01818D928D0895FC0184899589089507
:105D100023EA33E0FC0131832083FB014089518970
:105D200062897389FC014283538364837583089578
:105D3000DC01ED91FC91048CF58DE02D199480E04F
:105D40000895FC019485FB018485981303C081E0CC
:105D5000943009F480E0089521E0FC0184858430CA
:105D600009F420E0822F08950895FC0184850C94A5
:105D70009B380F931F93CF93DF93CDB7DEB7289750
:105D80000FB6F894DEBF0FBECDBF8C01F801818D38
:105D9000928D892B49F0D801ED91FC910284F38515
:105DA000E02DC8011995F2CF808D0E947B3818161E
:105DB00019065CF548E050E0BE016F5F7F4FD801E7
:105DC00058968C910E949B389C0118161906DCF499
:105DD00089819A81AB81BC81F801808B918BA28BE8
:105DE000B38B8D8190E0982F88272E81820F911D93
:105DF000958B848B2F8130E0322F22278885280FC6
:105E0000311D328F218FC90102C080E090E02896B9
:105E10000FB6F894DEBF0FBECDBFDF91CF911F91BB
:105E20000F910895AF92BF92CF92DF92FF920F939E
:105E30001F93CF93DF938C015B01EA01FC01C688BD
:105E4000D788F08C80E590E00E94A23E8F2D0E94C2
:105E5000B9478C179D0720F48F2D0E94B947EC019C
:105E60009E01A501B6018F2D0E9454470E94A13EBC
:105E7000F801868997898C0F9D1F978B868BCE01A1
:105E8000DF91CF911F910F91FF90DF90CF90BF9046
:105E9000AF900895CF93DF93EC01888D843061F04B
:105EA0000E943239E88DF0E0EE0FFF1FE151F84F0C
:105EB0001182108284E0888FDF91CF910895EF9254
:105EC000FF921F93CF93DF93FC01208D243011F0BC
:105ED00080E01CC07B01EC0110E0812F0E94FB39A7
:105EE000811102C0188F05C08831E1F31F5F1430A3
:105EF000A1F7888D843061F3FD86EC861A8E198EA9
:105F000020E0A70162E00E94443981E0DF91CF9157
:105F10001F91FF90EF9008950F931F93CF93DF93FE
:105F20001F92CDB7DEB78C01DC01ED91FC910084AE
:105F3000F185E02D1995892B51F0BE016F5F7F4FE0
:105F4000F80184850E944538898190E002C08FEF76
:105F50009FEF0F90DF91CF911F910F910895FC015A
:105F60001382128288EE93E0A0E0B0E084839583F0
:105F7000A683B7838CE692E09183808383EA93E0E3
:105F800097878687108A118A128A138A84E0808F05
:105F90000895CF92DF92EF92FF920F931F93CF93CA
:105FA000DF93CDB7DEB7E1970FB6F894DEBF0FBE33
:105FB000CDBF7C016A0103EA13E01A8309831B82C7
:105FC0001C821D821E82CE01099668AB79ABC7DFA9
:105FD0001DA30CA31EA21FA218A619A680915109E9
:105FE00090915209A0915309B09154098CA79DA793
:105FF000AEA7BFA78B839C83AD83BE8318861F8209
:10600000AE014C5D5F4F68A979A9CE0101960FD40E
:1060100081309105B1F4D701ED91FC910488F589A7
:10602000E02D1BA70AA78EA19FA1A8A5B9A58CA7A3
:106030009DA7AEA7BFA7A601BE01665D7F4FC701A2
:106040001995E1960FB6F894DEBF0FBECDBFDF9174
:10605000CF911F910F91FF90EF90DF90CF90089517
:106060009B0190E00496982F8827642F820F931F3E
:106070000C94B6270F931F93CF93DF931F92CDB746
:10608000DEB790E00496982F88278C01060F171F23
:106090000E942A278FE00E945C27812F0E945C27A4
:1060A000802F0E945C2780E00E945C2789830E94E9
:1060B000282789810F90DF91CF911F910F9108952B
:1060C000CF93FC01C08D80E590E00E94A23E60E28B
:1060D00070E08C2F47DC62E070E08C2FCBDF84FD1A
:1060E00017C062E070E08C2FC5DF83FF0AC048E173
:1060F00062E070E08C2FB4DF0E94A13E80E090E06F
:1061000010C00E94A13E80E590E00E94A23EE3CF35
:1061100040E162E070E08C2FA3DF0E94A13E81E0AD
:1061200090E0CF910895CF93DF93C82FD62F472FBC
:1061300060E170E095DF4D2F61E170E08C2FDF9121
:10614000CF918ECFFF920F931F93CF93DF93FB01DD
:10615000DC0157961C921E9256975896FC908281AD
:10616000811109C08381811106C08481811103C01E
:1061700085818823F1F041155105D9F08A01EF019D
:1061800080E590E00E94A23EBE016E5F7F4F2F2D02
:1061900030E0922F882744E050E0845F9B4F0E94BC
:1061A0008D27B8018F2DBFDF0E94A13E81E090E0D6
:1061B00002C080E090E0DF91CF911F910F91FF909E
:1061C0000895FC018485843011F00C94FB3980E043
:1061D0000895CF93DF93FC0124852430C9F0EC01AE
:1061E000F0DF843181F0882371F0883161F08C31E7
:1061F00061F4E881F9810084F185E02DCE011995E3
:1062000021E0892B19F420E001C021E0822F01C098
:1062100080E0DF91CF910895CF92DF92EF92FF92CD
:106220001F93CF93DF93FC011485143091F1EC019F
:1062300080E590E00E94A23E68E070E0812F92DB52
:106240000E94A13E0E94BC146B017C01CE01B9DF0B
:106250008823A9F061E070E080E090E00E9484145F
:106260000E94BC14DC01CB018C199D09AE09BF0949
:10627000883E9340A105B10548F38C85F3D7EC85A2
:10628000F0E0EE0FFF1FE151F84F1182108284E021
:106290008C87DF91CF911F91FF90EF90DF90CF908F
:1062A000089580E3FB0180833296842F82958F705E
:1062B00090E1899F401911244A3014F4405D01C0D7
:1062C000495C4293482F8111F0CF08952F923F925D
:1062D0004F925F926F927F928F929F92AF92BF92F6
:1062E000CF92DF92EF92FF920F931F93CF93DF93A2
:1062F000CDB7DEB7E3970FB6F894DEBF0FBECDBFC4
:106300007C011A012B0139010E94BC144B015C0174
:1063100087010D5B1F4FC8012CDD18161906A4F06C
:106320000E94BC14DC01CB0188199909AA09BB0998
:10633000281639064A065B06D0F062E370E080E07A
:1063400090E00E948414E7CF42E250E0BE016F5F0C
:106350007F4FC80141D78981823011F080E04BC165
:10636000F8018489958983349105C1F702C08FEFC4
:1063700042C16D817E818F8198850E942F664B017D
:106380005C01F301608371838283938346E050E074
:10639000B701685F7F4FCE014D960E946D66892BD5
:1063A000E9F6F70180819181A281B381881699066F
:1063B000AA06BB0698F284819581A681B7818815CB
:1063C0009905AA05BB0550F289899A89AB89BC89D0
:1063D00086879787A08BB18B8EECA82EB12CC80135
:1063E00019D7F1E0AF1AB108D1F719A6670182E217
:1063F000C80ED11CF701B696FBA7EAA7C7018A967B
:106400009DA78CA73C974F0189969FA78EA7389789
:10641000F9ABE8AB1701F6E12F0E311CC5979BAB2A
:106420008AABF801818D928D181619060CF0E2C026
:10643000C801F0D68333910509F4BBC0ECF4813078
:106440009105A9F11CF4892B61F3CAC08330910531
:10645000A9F1069709F0C4C0C801DCD65C0144E08C
:1064600050E06AA97BA9C801B7D6412C512CBB24A6
:10647000F4E0AF1AB1083AC08A33910509F471C04B
:106480003CF48533910569F0C69709F439C0A8C07A
:106490008B33910509F479C08F3F910509F4C1CF81
:1064A0009FC0C801B7D6C801B5D689A7BACFC80161
:1064B000B1D644E050E068A979A935C0C801AAD690
:1064C0005C0144E050E0B101C80186D6412C512C5A
:1064D000BB2494E0A91AB1084A145B040CF0A1CFC4
:1064E000C80198D6EFEF4E1A5E0AF6CF4A145B0445
:1064F0000CF097CFC8018ED68FEF481A580AF6CF06
:10650000C80188D6B82EF701828D81110FC0838D06
:1065100081110CC0848D811109C0858D811106C047
:1065200044E050E0B401C80157D67BCFEEA5FFA5EB
:106530004080518062807380B401CE0183960E94B6
:10654000D8128DA19EA1AFA1B8A584159505A60569
:10655000B70531F3BB2009F464CFC8015BD6BA9408
:10656000F9CFC80157D644E050E06AA57BA5C80121
:1065700033D6F70166A177A180A591A50E942F6669
:1065800066A377A380A791A74CCFC80143D644E068
:1065900050E06CA57DA5C8011FD6F70162A573A5C3
:1065A00084A595A50E942F6662A773A784A795A7C7
:1065B00038CFC8012FD644E050E0B601C8010CD650
:1065C000F70162A173A184A195A10E942F6662A325
:1065D00073A384A395A366A777A780AB91AB21CFC4
:1065E000C80118D6B82EBB2009F41BCFC80112D69B
:1065F000BA94F9CF89A5E3960FB6F894DEBF0FBE23
:10660000CDBFDF91CF911F910F91FF90EF90DF9061
:10661000CF90BF90AF909F908F907F906F905F9042
:106620004F903F902F9008957F928F929F92AF92BC
:10663000BF92CF92DF92EF92FF920F931F93CF936F
:10664000DF93CDB7DEB7A6970FB6F894DEBF0FBEC7
:10665000CDBF8C01762E942E852E20E2B22ECE0157
:1066600001967C01FC012B2D11922A95E9F783EA12
:1066700093E09AA389A38FEF8BA38CA38DA38EA302
:10668000680183E4C80ED11C43E450E0BE016F5D95
:106690007F4FC60157DD019609F4B5C081E08983BB
:1066A0008A8386E0A82EAB821C82F8016481758102
:1066B000868197810E942F666D837E838F83988762
:1066C00089869A8680E890E09C878B874CE150E031
:1066D000B701C601A7DBF7012B2D11922A95E9F727
:1066E000480188E0880E911CF401D70101900D92B9
:1066F000AA94E1F740E150E0B701C60193DBF7014E
:106700001192BA94E9F796E0A92EB12C40E250E03C
:10671000B701C60187DBF1E0AF1AB108B9F783E62C
:10672000898392E89A8393E59B838C8385E38D83A9
:1067300081E08E837F829DE3988797E099878A879F
:1067400086E0F401DE011B9601900D928A95E1F737
:106750008CE0898B8A8B61E774E0CE0143960E94BE
:10676000AC66F8014385BE01675E7F4FC80199DDC5
:10677000F8014485BE01655E7F4FC80192DDF801D6
:106780004585BE01635E7F4FC8018BDD4EE150E061
:10679000B701C60147DBF3E07F121DC082E38983A6
:1067A00084E08A83F80196859B8397859C839089F2
:1067B0009D8391899E8396E39F838887828D8987B5
:1067C000838D8A87848D8B87858D8C874CE050E004
:1067D000B701C60127DB87E3898386E08A8391E0DE
:1067E0009B8393E09C838D838FE08E838AE38F83EA
:1067F0008BE388878FEF898749E050E0B701C601B6
:1068000011DBC6015DDCA6960FB6F894DEBF0FBEA5
:10681000CDBFDF91CF911F910F91FF90EF90DF904F
:10682000CF90BF90AF909F908F907F9008952F92C0
:106830003F924F925F926F927F928F929F92AF9210
:10684000BF92CF92DF92EF92FF920F931F93CF935D
:10685000DF93CDB7DEB765970FB6F894DEBF0FBEF6
:10686000CDBF7C016B013A01FB0120E080E090E0AC
:106870006AE03191332309F140ED430F4A3080F44F
:10688000689FA001699F500D1124CA01C097830F12
:10689000911D37FD9A958F3F910559F350F313C021
:1068A0003E3289F4233079F0D301A20FB11D129644
:1068B0008C932F5F80E090E0DCCF233021F4F30154
:1068C000858381E020C0F701428153816481758115
:1068D0008091590990915A09A0915B09B0915C0986
:1068E000481759076A077B0709F484C10E94BC1442
:1068F0008701085F1F4F6F7077277C5FC801DFDA61
:10690000813019F080E090E0D1C183EA93E09A836E
:106910008983F70182819381A481B5818B839C83D4
:10692000AD83BE8345E350E0BE016F5F7F4FC8017A
:1069300009DC892B19F4C12CD12C58C10E94BC143C
:10694000F701778366837627672776277A836983BB
:1069500042E050E0BE016F5F7F4FC80163DA81E023
:1069600090E09E878D8742E050E0BE01635F7F4FDD
:10697000C80158DA80E091E09E878D8742E050E0C0
:10698000BE01635F7F4FC8014DDA1E861D8642E05F
:1069900050E0BE01635F7F4FC80144DA42E050E03F
:1069A000BE01635F7F4FC8013DDA42E050E0BE01A7
:1069B000635F7F4FC80136DA5601F5018081882375
:1069C00001F1F6015F018191811113C045018C181D
:1069D0009D081814190484F48F8641E050E0BE012C
:1069E000615F7F4FC8011EDAA401B601C8011ADA3F
:1069F00003C08E3239F7EACF6501FFEFCF1ADF0A05
:106A0000DCCF1F8641E050E0BE01615F7F4FC801CF
:106A100009DAC12CDD24D394DE86CD8642E050E035
:106A2000BE01635F7F4FC801FDD9DE86CD8642E09F
:106A300050E0BE01635F7F4FC801F4D9C80140DB5D
:106A4000892B09F478CF63E0A62EB12CF2E06F0E0B
:106A5000711C0E94BC141B012C01C8018AD9181694
:106A60001906A4F00E94BC14DC01CB018219930921
:106A7000A409B509813A9F40A105B105D0F462E3AC
:106A800070E080E090E00E948414E7CFF70142813B
:106A9000538164817581808D918DA28DB38D48174E
:106AA00059076A077B0741F4848D958DC59721F4BA
:106AB00006C02FEF3FEF90C02EEF3FEF8DC0F701E4
:106AC00081A192A10C970CF49BC04CE050E0BE0158
:106AD0006F5F7F4FC80180D38B8190E0982F88270C
:106AE0002C81822B9A8B898B298130E0322F2227AF
:106AF0004A81242BF701468157814217530709F039
:106B00007CC097FF7AC08F709270892B09F0CBC040
:106B1000CF80D12CDC2CCC248885C82AC114D10488
:106B200009F4BEC0812C912C8D8190E0982F88278C
:106B30002E81822B8816990608F465C0812C912C31
:106B400041E050E0BE016D5E7F4FC80145D38B89A7
:106B5000982F907C09F083C0811177C08B898111B7
:106B6000EFCF42E050E0BE01615F7F4FC80134D3F8
:106B700042E050E0BE01635F7F4FC8012DD3C801E2
:106B800049D3C80147D3C80145D3C80143D342E024
:106B900050E0BE016F5E7F4FC8011ED38F8598897C
:106BA0008115914009F05FC02D853E85322723274E
:106BB00032272130310509F056C089899A8981151B
:106BC000944009F06AC044E050E0B301C8012C8B46
:106BD0003D8B02D32C893D896901F1E0AF1AB108E0
:106BE00029F02FEFC216D20609F433CFC80152D9CB
:106BF000C6015CC08EEF9FEF59C02CEF3FEFECCF8A
:106C00002DEF3FEFE9CF41E050E0BE01635F7F4FE2
:106C1000C801E2D28D8581110FC08D858111F3CF1E
:106C2000C801F8D2C801F6D2C801F4D2C801F2D224
:106C3000FFEF8F1A9F0A78CF8D859FEF980F9D8762
:106C4000882359F3C801E6D2F7CF8B899FEF980FBD
:106C50009B8B882309F482CFC801DCD2F6CFC80110
:106C6000D9D21B8A7BCF412C512C89899A899827AC
:106C7000892798274816590630F4C801CBD28FEFE0
:106C8000481A580AF2CFEFEF8E1A9E0A8C149D0410
:106C900009F056CF26EF3FEF9FCF27EF3FEF9CCF76
:106CA0002AEF3FEF99CF2BEF3FEF96CF65960FB6C8
:106CB000F894DEBF0FBECDBFDF91CF911F910F9132
:106CC000FF90EF90DF90CF90BF90AF909F908F900C
:106CD0007F906F905F904F903F902F9008952F92EC
:106CE0003F924F925F926F927F928F929F92AF925C
:106CF000BF92CF92DF92EF92FF920F931F93CF93A9
:106D0000DF93CDB7DEB727970FB6F894DEBF0FBE7F
:106D1000CDBF8C010E94385B2FEC37E040E050E0A3
:106D20000E945962DC01CB010196A11DB11DF80141
:106D300084839583A683B78380839183A283B3835F
:106D40005801F3E4AF0EB11CC501A4D864E470E0AF
:106D5000C501B5D8882309F437C10E94BC142B01A2
:106D60003C01812C912C1D82C8018E5B9F4F9F831B
:106D70008E8343E0342E58EEC52E53E0D52EE12C01
:106D8000F12C62E0262EAE81BF818C91833009F414
:106D900002C181111FC0F80184819581A681B7814C
:106DA0000196A11DB11D84839583A683B7830E949C
:106DB000BC146419750986099709A70196010E94F8
:106DC0003762A90161E0C8012FDC81E0AE81BF819B
:106DD0008C93C2C08430F1F4F80184819581A6813E
:106DE000B7810196A11DB11D84839583A683B783C6
:106DF0000E94BC146419750986099709A7019601B8
:106E00000E943762A90163E0C8010EDCAE81BF8138
:106E10002C92A2C0813051F5F80142AD53AD64AD62
:106E200075AD9E012F5F3F4FC80150DA8D838230D0
:106E300009F092C089819A81AB81BC81F801848379
:106E40009583A683B7830E94BC14641975098609CB
:106E50009709A70196010E943762A90163E0C80162
:106E6000E3DBED81AE81BF81EC937DC0823009F020
:106E700073C0D801DA964D915D916D917C91DD974B
:106E80009E012F5F3F4FC80121DA8D83853009F0C5
:106E90005CC0EE81FF813082F80182A193A1A4A1A0
:106EA000B5A1892B8A2B8B2B41F484E893E0A0E0D9
:106EB000B0E082A393A3A4A3B5A3F80186A197A1F0
:106EC000A0A5B1A5892B8A2B8B2B61F482A193A15C
:106ED000A4A1B5A1B695A7959795879586A397A3E5
:106EE000A0A7B1A7F80182A593A5A4A5B5A5892B54
:106EF0008A2B8B2BA9F482A193A1A4A1B5A1AC01EB
:106F0000BD0123E076956795579547952A95D1F76A
:106F1000841B950BA60BB70B82A793A7A4A7B5A7B5
:106F2000F80186A197A1A0A5B1A586A797A7A0ABB8
:106F3000B1AB82A593A5A4A5B5A582AB93ABA4AB39
:106F4000B5AB88248394912C0EC0FD81F63021F4DA
:106F5000AE81BF811C9207C0BD81BF3F21F4EE818D
:106F6000FF8110821D82F1E08F16910409F40BCF8E
:106F70000E94BC14DC01CB0184199509A609B7094C
:106F8000F80126A937A940AD51AD281739074A079E
:106F90005B0708F0F8CEC5010E944A2FF8018481F2
:106FA0009581A681B7810196A11DB11D848395832A
:106FB000A683B7830E94BC14F801FE966083718398
:106FC00082839383C40102C080E090E027960FB6CD
:106FD000F894DEBF0FBECDBFDF91CF911F910F910F
:106FE000FF90EF90DF90CF90BF90AF909F908F90E9
:106FF0007F906F905F904F903F902F9008959FE902
:10700000980F963010F429EA05C09FEB980F963040
:1070100018F429EC280F05C090ED980F9A3008F469
:10702000292F822F08950F931F93CF93DF93282F3B
:10703000DC01C42FD52F8A2F821B8617D0F48D0137
:10704000ED91F0E084E0F595E7958A95E1F7E0575A
:10705000FD4F808188832296CE010197F80130810F
:10706000E32FEF70F0E0E057FD4F3081FC013083FB
:10707000E2CFFA01E60FF11DE60FF11D1082DF915C
:10708000CF911F910F91089508951F93CF93DF9390
:107090001F921F92CDB7DEB7182F80E590E069836D
:1070A0007A8350D621E041E050E069817A81812FD6
:1070B0000E94C02C46D681E090E00F900F90DF91A7
:1070C000CF911F910895CF93DF931F92CDB7DEB775
:1070D000FC01218D328D232B41F0BE016F5F7F4F6C
:1070E000808DD3DF898190E002C08FEF9FEF0F90FA
:1070F000DF91CF910895FF920F931F93CF93DF936A
:10710000F82E80E590E01ED6C0E0D0E08F2D0E94E2
:107110002C278C01892B21F08F2D0E942C27EC012C
:10712000C017D10799F70DD6CE01DF91CF911F91EE
:107130000F91FF900895AF92BF92CF92DF92EF929E
:10714000FF921F93CF93DF93182F5B017A0180E5A5
:1071500090E0F8D5C0E0D0E0812F0E942C276C0190
:10716000892B21F0812F0E942C27EC01CC15DD0505
:1071700099F7209799F463E070E0812F0E943A30EC
:107180008431F1F08823E1F0C1E0D0E08C3111F4DA
:10719000C0E0D0E0D195C195D10912C0EC16FD0632
:1071A0000CF4E7011C161D065CF420E0AE01B501ED
:1071B000812F0E94C02C60E470E0812F0E94B22CCD
:1071C000C0D5CE01DF91CF911F91FF90EF90DF905E
:1071D000CF90BF90AF900895CF93DF93FC01218DA6
:1071E000328D2115310519F48FEF9FEF10C0EC019E
:1071F0004217530708F0A901888D9DDF181619065C
:107200009CF7298D3A8D281B390B3A8F298FDF91F6
:10721000CF9108950F931F93CF93DF931F92CDB714
:10722000DEB7FC01218D328D232B59F08C0141E01A
:1072300050E0BE016F5F7F4F808D7DDF181619060D
:107240001CF08FEF9FEF08C0F801818D928D0197A0
:10725000928F818F898190E00F90DF91CF911F9164
:107260000F910895CF93C82F80E590E06BD560E132
:1072700070E08C2F0E94B22C4FEF62E070E08C2FF8
:107280000E943030CF915DC5FF920F931F93CF9333
:10729000DF931F921F92CDB7DEB7F82E8A012A83A3
:1072A0006983E0DF80E590E04DD52A816981462F32
:1072B000422B60E070E08F2D0E94303001151105E7
:1072C00051F40091F7071091F8070F5F1F4F1093CB
:1072D000F8070093F707412F64E070E08F2D0E94BC
:1072E0003030402F65E070E08F2D0E94303061E03B
:1072F00070E08F2D0E94B22C24D581E00F900F906A
:10730000DF91CF911F910F91FF900895BF92CF927F
:10731000DF92EF92FF920F931F93CF93DF9300D0F2
:1073200000D0CDB7DEB7FC01208D243009F052C06B
:107330006A017B018C01B12C63E070E08B2D0E940F
:107340003A30811103C0F801B08E06C08831D9F3FC
:10735000B394F4E0BF12F0CFF801808D8430D1F106
:1073600096E0E1EAF2E0DE01119601900D929A9525
:10737000E1F7F70193819F779C8394819D839581A9
:107380009E83B7016E5F7F4F90E0982F882744E07F
:1073900050E0845F9B4F0E948D27B601F801808DDD
:1073A0000E949330F801808D90E0982F882746E066
:1073B00050E0BE016F5F7F4F8A5F9B4F0E948D2719
:1073C000F801128E118E20E8A60162E0808D5CDF4C
:1073D00081E001C080E026960FB6F894DEBF0FBEB4
:1073E000CDBFDF91CF911F910F91FF90EF90DF9074
:1073F000CF90BF9008951F93CF93DF931F92CDB787
:10740000DEB7182F80E590E09DD463E070E0812F17
:107410000E943A30898395D489810F90DF91CF9172
:107420001F91089569E277E086EA98E00C94C7120C
:10743000CF93DF93C1E1D0E068EE73E080E090E0AD
:107440000E9484144AE050E0BE0186EA98E00E945F
:10745000A212219789F7DF91CF9108956F927F92C1
:107460008F929F92AF92BF92CF92DF92EF92FF9254
:107470000F931F93CF93DF93CDB7DEB761970FB60E
:10748000F894DEBF0FBECDBF68E774E080910608B8
:10749000909107080E9491438C010097D1F10E94BE
:1074A000DD2A8230B1F560E0C8010E9484437C018E
:1074B00061E0C8010E948443DC0119960D911C9182
:1074C0001A97F701818521E09091A405992309F489
:1074D000D5C2909170009E7F909370001092A40589
:1074E00010920202109201028093000221110E9468
:1074F0002217C8010E94491767E878E086EA98E0F9
:107500000E948E114AE050E0B80186EA98E00E949D
:10751000A2126CE774E080910608909107080E941F
:1075200091439093FF078093FE07009709F4A7C04B
:107530000E94DD2A082F10E00115110509F49FC0F3
:10754000000F111F000F111FC8010E94C259909314
:10755000FB078093FA071092AD051092AC051092CC
:107560000108109200081092AB051092AF0510921E
:10757000AE050130F2E01F070CF489C2E12C72E085
:10758000F72EC70101960E94C2599093B1058093CE
:10759000B0059093AA058093A9058E0D9F1D909329
:1075A000A8058093A7050E94BC14609340057093C2
:1075B0004105809342059093430580E090E0E0917F
:1075C000B005F091B105E80FF91F10820196E81699
:1075D000F906ACF782E090E09093AD058093AC059E
:1075E00080E98093C9001092C8001092CD0083E01A
:1075F0008093CC008EE08093CA00F0920502E09266
:1076000004022091B0053091B1058091040290915F
:107610000502820F931F9093A8058093A705232B43
:1076200009F42EC265EE77E086EA98E00E948E119A
:107630004AE050E0B80186EA98E00E94A21287E191
:1076400096E09093A6058093A505809152059091B0
:107650005305009739F0FC01EA5CFD4F81E595E0A8
:10766000918380836DE678E086EA98E00E948E112F
:107670004AE050E0B80186EA98E00E94A212009128
:1076800006081091070862E874E0C8010E9491435F
:1076900090934B0580934A05DC0116968D919C9141
:1076A000179790934705809346056FE774E0C801EC
:1076B0000E949143909349058093480568E874E0DF
:1076C000C8010E94914390934D0580934C056FE84B
:1076D00074E0C8010E9491439093FD078093FC07DA
:1076E00064E974E0C8010E9491439093500580932F
:1076F0004F0561E678E086EA98E00E94C7126AE5E5
:1077000078E086EA98E00E948E1181E020914A0597
:1077100030914B05232B09F480E08BD762E578E0AC
:1077200086EA98E00E948E1181E020914805309110
:107730004905232B09F480E07CD76AE478E086EAE7
:1077400098E00E948E1181E020914C0530914D050A
:10775000232B09F480E06DD764E478E086EA98E0B2
:107760000E948E1181E02091FC073091FD07232BB0
:1077700009F480E05ED76CE378E086EA98E00E9446
:107780008E1181E020914F0530915005232B09F493
:1077900080E04FD7E0914F05F0915005309709F404
:1077A00005C280915105811101C2E680F78081E117
:1077B00090E00E94C2598C0188E1F8018183128215
:1077C0001082108A178610922C0610922B061092A7
:1077D000BC071092DE070E948C1F109337050093A0
:1077E000360583E190E00E94C259FC0185E79DE1E6
:1077F000928B818B168305831482108289E08183AA
:1078000011E012831383F0933F05E0933E0580EA75
:1078100090E00E94C25990933B0580933A0588E21C
:1078200090E00E94C25990933505809334051092E0
:107830002C0610922B061092BC071092DE070E94B5
:107840008C1F80913605909137050E94BA1F81E008
:107850000E945F2D811169C06DE178E086EA98E0B1
:107860000E94C712C0903605D0903705C6010E940D
:10787000BA1F40E060EFC6010E947F20C6010E944F
:10788000B71FE0913605F091370510836DEF77E073
:1078900086EA98E00E94C7128091360590913705DC
:1078A0000E944A20882331F061EF77E086EA98E071
:1078B0000E94C71200913E0510913F050E94BC1422
:1078C0004B015C01F0E18F0EF7E29F1EA11CB11C81
:1078D000D8011596ED91FC9116978FEF838714864A
:1078E000DF0113963B961D92AE17BF07E1F7F80133
:1078F000148277247394BE01665F7F4FD80115967A
:107900008D919C9116970E94A22018160CF4C1C06C
:107910008FE99BE49093390580933805E0913E050B
:10792000F0913F05128281E001C080E08093510513
:1079300001E010E068E0B62EE114F10409F436C16C
:10794000F7018085863009F095C0C080D180CE01D6
:1079500001964C01360190E1690E711CD6018C91A3
:107960004EDBA82EB2E0CB0ED11CF6013197808100
:1079700046DBA29450EFA5228A29F40181934F019E
:10798000C614D70459F7E0913C05F0913D05EE0F80
:10799000FF1F8091340590913505E80FF91F118381
:1079A0000083A0913C05B0913D0523E0AA0FBB1FC9
:1079B0002A95E1F780913A0590913B05A80FB91FF0
:1079C000FE0131968B2D01900D928A95E1F767E3C8
:1079D00078E086EA98E00E948E1160913C057091F3
:1079E0003D054AE050E086EA98E00E94561260E3C6
:1079F00078E086EA98E00E948E1180913C05909193
:107A00003D0533E0880F991F3A95E1F720913A053B
:107A100030913B05820F931F0E943E2E86EA98E02C
:107A20000E949F1260913C0570913D0543E0660FF6
:107A3000771F4A95E1F780913A0590913B05680FD1
:107A4000791FDB018C91883261F480913E05909121
:107A50003F050E94BC2D80913605909137050E940C
:107A6000752080913C0590913D05019690933D05D0
:107A700080933C05F701E280F3805ECF20E034CDB7
:107A80006EEC77E086EA98E00E94C712D8CD7801C4
:107A900078CD0E94BC14681579058A059B0508F00D
:107AA00037CF67E0CE010A960E94AA1F99898913F1
:107AB0006FC06EEE73E086EA98E00E94D712D8019C
:107AC0008C9181113AC015968D919C9116970E94C8
:107AD0004A20BE01665F7F4FF801858196810E9432
:107AE0005A2140E064EBD80115968D919C91169730
:107AF0000E947F20F801C580D680C6010E94D91F50
:107B0000C6010E94BA1F67E883E499E00E94471DFE
:107B100060E883E499E00E94471DC6010E94B71FF8
:107B2000C6010E94D91FD82ED80115968D919C911F
:107B300016970E944A20D5FE32C0AE014F5F5F4FBC
:107B4000BE01665F7F4FC8010E948521F801D18088
:107B50008A85803139F1BE01665F7F4FC8010E947E
:107B6000EF218D1520F4D80111968C910BC08A85D8
:107B7000803111F48CE006C0BE01665F7F4FC80102
:107B80000E94EF21F801818384818F5F8483B3CECB
:107B900064EF73E086EA98E00E94D712ACCED80179
:107BA0007C92CBCFBCE0BD15F0F2E4CF61960FB66E
:107BB000F894DEBF0FBECDBFDF91CF911F910F9123
:107BC000FF90EF90DF90CF90BF90AF909F908F90FD
:107BD0007F906F900895CF93DF931F92CDB7DEB75C
:107BE0006983DC01ED91FC910280F381E02D41E09D
:107BF00050E0BE016F5F7F4F19950F90DF91CF91DD
:107C00000895DC01ED91FC91068CF78DE02D19951E
:107C100091E089270895862F089581E086270895A9
:107C2000CF93DF931F92CDB7DEB741E050E0BE01A6
:107C30006F5F7F4FFC0184857EDA181619061CF4ED
:107C4000898190E002C08FEF9FEF0F90DF91CF917D
:107C50000895FC018485843009F04DCA80E090E0ED
:107C60000895CF92DF92EF92FF920F931F93CF93DD
:107C7000DF93CDB7DEB7E1970FB6F894DEBF0FBE46
:107C8000CDBF7C016A0103EA13E01A8309831B82DA
:107C90001C821D821E82CE01099668AB79AB0E94C0
:107CA000AF2F1DA30CA31EA21FA218A619A6809178
:107CB000510990915209A0915309B09154098CA790
:107CC0009DA7AEA7BFA78B839C83AD83BE83188679
:107CD0001F82AE014C5D5F4F68A979A9CE01019664
:107CE0000E94173481309105B1F4D701ED91FC91D8
:107CF0000684F785E02D1BA70AA78EA19FA1A8A542
:107D0000B9A58CA79DA7AEA7BFA7A601BE01665DBA
:107D10007F4FC7011995E1960FB6F894DEBF0FBEED
:107D2000CDBFDF91CF911F910F91FF90EF90DF902A
:107D3000CF90089544E050E0BC018FE090E00C94B7
:107D40008D2708958CBD9DBD08958F929F92AF920F
:107D5000BF92CF92DF92EF92FF920F931F93CF9338
:107D60006C015B017A01FC01C485C43041F481E0FF
:107D700090E0F6019383828380E090E04AC08A011C
:107D80004130584010F000E018E080E590E0DADF84
:107D90008C2F0E94B9474C0163E070E08C2F0E9449
:107DA0003A30873111F08C3121F48016910668F356
:107DB00002C000E010E080E590E0C4DF9801A5017A
:107DC00060E070E08C2F0E94544760E270E08C2FDE
:107DD0000E94B22C62E070E08C2F0E943A3084FD49
:107DE0000EC063E070E08C2F0E943A30811103C016
:107DF0008C2F38DABCCF80E590E0A4DFEBCF40E1F8
:107E000062E070E08C2F0E943030012B09F4AFCF7C
:107E1000C701CF911F910F91FF90EF90DF90CF900E
:107E2000BF90AF909F908F900895CF92DF92EF9286
:107E3000FF920F931F93CF93DF93FC01248524308F
:107E400009F07CC06A018B01EC01F12C8F2DD3DA93
:107E5000811102C0FC8607C08B7F8831D9F3F3946F
:107E6000F4E0FF12F3CF8C85843009F467C02091D1
:107E70000602309107022F5F3F4F11F420E030ECF3
:107E800030930702209306024091060250910702A8
:107E900020E061E0F9D9FC84F80182818F3F51F440
:107EA00083818F3F99F484818F3F81F485818F3F57
:107EB00069F442C081110AC0F8018381811106C0B2
:107EC0008481811103C085818823B1F1C114D1045B
:107ED00099F180E590E036DFB8016E5F7F4F8F2D1E
:107EE00090E0982F882744E050E0845F9B4F0E94E9
:107EF0008D27B6018F2D0E94933064E070E08F2DA6
:107F00000E94B22C0E94BC146B017C01F4E9CF0EDC
:107F1000F1E1DF1EE11CF11CCE010E94E13087314E
:107F200051F161E070E080E090E00E948414CE01A5
:107F30000E94E130811105C084E08C8780E090E0F0
:107F40001CC00E94BC14C616D706E806F90620F726
:107F50008C8588D9EC85F0E0EE0FFF1FE151F84FDA
:107F60001182108284E08C8763EA78E086EA98E0E8
:107F70000E94C712E3CF81E090E0DF91CF911F9183
:107F80000F91FF90EF90DF90CF9008958091520570
:107F900090915305009711F00E943016A89508950E
:107FA000A8950E94B317029754F00E94F04C80915C
:107FB000520590915305009711F00E9430160C94D1
:107FC000050F60E08DE00C94191461E08DE00C94D5
:107FD00019140F931F93CF93DF93EB0181E395E087
:107FE0009F938F9380E395E09F938F938FE295E02B
:107FF0009F938F938EE295E09F938F938DE295E010
:108000009F938F938CE295E09F938F9387E994E001
:108010009F938F938B818F938A818F930E94586750
:108020002DB73EB7205F3F4F0FB6F8943EBF0FBE4F
:108030002DBF069784F46EE079E086EA98E00E940E
:108040008E116A817B8186EA98E0DF91CF911F9142
:108050000F910C94B7120E94AF490CE215E0C0E0FA
:10806000D0E0F80161918F01CE010E942962219632
:10807000C630D105B1F760E279E086EA98E0DF9199
:10808000CF911F910F910C94C712CF93DF93CDB76F
:10809000DEB72C970FB6F894DEBF0FBECDBF1C82A3
:1080A0001B821E821D828FEF9FEF98878F838BEC40
:1080B00092E09A83898386E290E09A8789871C867A
:1080C0001B866EEF78E086EA98E00E94C712609106
:1080D000060870910708CE0101960E942D256FEFCA
:1080E000CE0101960E94612468EF78E086EA98E06C
:1080F0000E94C7122C960FB6F894DEBF0FBECDBFFC
:10810000DF91CF910895CF93DF93CDB7DEB7699715
:108110000FB6F894DEBF0FBECDBF8FE290E0A0E0B7
:10812000B0E089839A83AB83BC83FE01359685E1F9
:10813000DF011D928A95E9F764EE78E086EA98E01F
:108140000E94C712AE014E5F5F4F66E08CE295E081
:108150000E9413381E866CEA74E0CE0101960E94DC
:108160008D66BE016F5F7F4F86EA98E00E94B7126E
:10817000CE0101960E94222D1E8664EB74E0CE0192
:1081800001960E948D66BE016F5F7F4F86EA98E080
:108190000E94B7126EEB74E0CE0101960E94B22BE2
:1081A0000E94A94969960FB6F894DEBF0FBECDBFF5
:1081B000DF91CF910895AF92BF92CF92DF92EF926D
:1081C000FF920F931F93CF93DF93CDB7DEB7C256C5
:1081D000D1090FB6F894DEBF0FBECDBF2CE0E7EAA1
:1081E000F2E08E010F5F1F4FD80101900D922A958A
:1081F000E1F7FE013D9624E1DF011D922A95E9F7A2
:108200001816190644F4FB01628173814FE150E0B6
:10821000C8010E94D166809131051F928F93809191
:1082200030051F928F9380912F051F928F9380911D
:108230002E051F928F9380912D051F928F93809111
:108240002C051F928F9380EC94E09F938F931F9245
:1082500080E28F937E01F1E2EF0EF11CFF92EF922C
:108260000E94EB6668EE79E086EA98E00E94C71209
:1082700060EE79E086EA98E00E948E11B80186EA05
:1082800098E00E94D712B70186EA98E00E94B712E0
:108290000FB6F894A8958091600088618093600083
:1082A000109260000FBE6E0181E4C80ED11CD60191
:1082B00013961C921E92129788EE93E0A0E0B0E015
:1082C000F60184839583A683B78384E0848781EE57
:1082D00092E09183808316870587108A178680E550
:1082E00090E0928B818B158A66E77DE18BEA93E2C1
:1082F0000E94B85B8C010FB6F894DEBF0FBECDBFF5
:10830000892B09F4AFC083E090E00E94C259D801E4
:108310001D969C938E931C97FC01D182C082128281
:10832000C6010E94E930882319F0C6010E940C3171
:10833000D6011F966D917C91509751964D915C910D
:10834000529761157105B9F0CE01895A9F4FA296D7
:108350004FAFA297A3965FAFA3970E94D812A296A1
:108360004FADA297A3965FADA397BE01695A7F4F09
:10837000C6015BDD05C0F60165857685C60171DC49
:10838000892B21F4C8010E941C226CC0D6011D96C5
:10839000BC901D971E96AC90FF92EF9289E799E0F2
:1083A0009F938F931F930F930E94405CFF92EF92D5
:1083B00084E799E09F938F931F930F930E94405CF3
:1083C000D8011C96ED91FC911D9781E08283FF926C
:1083D000EF9281E799E09F938F931F930F930E94F1
:1083E000405CD8011C96ED91FC911D971282AF92D2
:1083F000BF928BE399E09F938F931F930F930E94FB
:10840000405C86E799E09F938F931F930F930E94A0
:10841000405CF601148A138AD8011C96ED91FC91F8
:108420001D97A080B1800FB6F894DEBF0FBECDBF00
:1084300083E3E82EF12CD501ED91FC910084F185C8
:10844000E02DC501199541970CF0A5C0B1E0EB1ADC
:10845000F10809F4A0C064E170E080E090E00E94BF
:108460008414E9CF00E010E0F601E388F48899E293
:1084700088E10FB6F894A895809360000FBE9093A2
:1084800060000115110509F467C0F8ECEF16F1045E
:1084900009F054C065ED79E086EA98E00E94C712C1
:1084A0006B961FAE1EAE6B976D961FAE1EAE6D9790
:1084B0008FEF9FEF6F969FAF8EAF6F9787E093E040
:1084C00069969FAF8EAF6997A1961FAF0EAFA19728
:1084D00080910608909107080E94882CCE01895A45
:1084E0009F4FC2D49093070880930608C8010E944A
:1084F0001C228091060890910708009779F46FEB91
:1085000079E086EA98E00E94C7120E94BC14DC0160
:10851000CB018856954CAF4FBF4F32C00E944A2CBA
:108520008C01BC0186EA98E00E94B712C8010E9443
:10853000575A0E942E3A82E090E067C067EA79E0DD
:1085400086EA98E00E948E114AE050E0B70186EA80
:1085500098E00E94A2120CC065E979E086EA98E0F2
:108560000E94C7126DE779E086EA98E00E94C71280
:108570000E94BC14DC01CB0188579C4EAF4FBF4F0B
:108580008093020890930308A0930408B093050811
:1085900085EF9FEF3AC07E01F7E5EF0EF11CFF92E9
:1085A000EF928FE299E09F938F931F930F930E9416
:1085B0005C5C0F900F900F900F900F900F900197B1
:1085C00009F052CFF70180819181D60154969C9396
:1085D0008E93539720E080E08A3021F08D3031F087
:1085E000282F04C02A3009F43FCF2AE0C801A29600
:1085F0002FAFA2970E94025CA2962FADA2978F3F49
:1086000059F7C8010E941C222FCFCE59DF4F0FB659
:10861000F894DEBF0FBECDBFDF91CF911F910F91B8
:10862000FF90EF90DF90CF90BF90AF900895C3DDA3
:1086300090C6882319F068E279E002C06BE279E025
:1086400086EA98E00C94C712CF93DF93CDB7DEB7DC
:108650002C970FB6F894DEBF0FBECDBF65ED78E066
:1086600086EA98E00E94C71286E290E00E942162AA
:108670008B37B9F51C821B821E821D828FEF9FEF04
:1086800098878F838BEC92E09A83898386E290E0CF
:108690009A8789871C861B86809106089091070817
:1086A0000E94882CCE010196DFD390930708809317
:1086B000060886EA98E00E949F1280910608909131
:1086C0000708892B19F468EB78E00DC061EB78E0BE
:1086D00086EA98E00E94C7120E942E3A81E090E05C
:1086E00008C064EC78E086EA98E00E94C71280E057
:1086F00090E02C960FB6F894DEBF0FBECDBFDF9191
:10870000CF910895A1DF25C6FC018681978100974E
:1087100039F0662329F06150FC0182819381F7CF03
:1087200008950F931F93CF93DF938B01FC01C681B4
:10873000D781209759F0B801888199810E947A6683
:10874000892B21F00A80DB81C02DF3CFCE01DF9190
:10875000CF911F910F910895CF93DF939B01672BCA
:1087600061F4E091A608F091A7080190F081E02D56
:10877000682F86EA98E0199508C0482F50E060E01D
:1087800070E086EA98E00E94C711EC0186EA98E062
:108790000E949F128C0F9D1FDF91CF910895DC01E5
:1087A0001696ED91FC91179761157105A1F0309720
:1087B00029F417967C936E9316970895828193817E
:1087C000009711F0FC01FACF73836283DB011596E9
:1087D000FC93EE93149708952F923F924F925F92DD
:1087E0006F927F928F929F92AF92BF92CF92DF92C1
:1087F000EF92FF920F931F93CF93DF93CDB7DEB726
:108800002B970FB6F894DEBF0FBECDBF8C012B01A6
:108810000E944726019609F4D1C2D801ED91FC913E
:108820000284F385E02DC80119957C018F3FBFEFCD
:108830009B0709F4C3C2D801ED91FC910684F7852A
:10884000E02D682FC8011995B2E2EB16F10429F466
:10885000B201C8010E946826B3C2EDE2EE16F1042F
:1088600029F0C701C0970A9708F045C1D801ED91DA
:10887000FC910284F385E02DC80119951C018F3FFE
:10888000BFEF9B0709F49AC28D9781F4D801ED914F
:10889000FC910284F385E02DC80119951C01019615
:1088A00009F48CC288248A94982C03C08824839469
:1088B000912CC101C097C12CD12C0A97C8F48AE031
:1088C000F82EFC9CC001FD9C900D1124B101605359
:1088D00071096C01C60ED71ED801ED91FC9102847E
:1088E000F385E02DC80119951C01C0970A9748F33C
:1088F000BEE22B163104C1F0C1018F7D8534910594
:1089000099F0C89CC001C99C900DD89C900D112471
:10891000092E000CAA0BBB0BF20181879287A3875B
:10892000B48782E08087DDC0B601DD0C880B990B2F
:108930000E9498636B017C01FEE22F163104B1F5B1
:10894000D801ED91FC910284F385E02DC8011995C1
:108950001C01A12CB12C20E030E040E251E4C70121
:10896000B6010E944C646B017C01B1016053710936
:10897000072E000C880B990B0E9498639B01AC0199
:10898000C701B6010E9495626B017C01B1E0AB1A90
:10899000B108D801ED91FC910284F385E02DC80166
:1089A00019951C01C0970A97B0F202C0A12CB12CF6
:1089B000C1018F7D8534910509F043C0D801ED9147
:1089C000FC910284F385E02DC80119951C018B32BE
:1089D000910559F4D801ED91FC910284F385E02DC5
:1089E000C80119951C01B1E00CC08D9761F4D80144
:1089F000ED91FC910284F385E02DC80119951C01CD
:108A0000BFEFBE8302C0E1E0EE83612C712C4AE02F
:108A1000C101C0978A309105C0F4469D9001479DE1
:108A2000300D11243901680E791ED801ED91FC91A9
:108A30000284F385E02DC8014B8719951C014B85F5
:108A4000E7CFB1E0BE83612C712CB401990C880B87
:108A5000990B0E949863A70196010E944C646B01D8
:108A60007C01B501BB0C880B990B0E9498634B01EC
:108A70005C01B301770C880B990B0E9498636F839C
:108A8000788789879A87EE816E2FEE0F770B880B98
:108A9000990B0E9498639B01AC016F817885898551
:108AA0009A850E944C649B01AC01C501B4010E94EF
:108AB00095629B01AC0160E070E080E291E40E946D
:108AC000AF649B01AC01C701B6010E944C64D201A6
:108AD00019966D937D938D939C931C9783E01896C4
:108AE0008C93D801ED91FC910684F785E02D622DE1
:108AF000C801199522C0BBE5EB16F10409F05FC06F
:108B0000D801ED91FC910284F385E02DC8011995FF
:108B10008B35910509F052C185E0F2018087C801CB
:108B20000E944726D801ED91FC910284F385E02D47
:108B3000C80119958D35910519F480E090E040C188
:108B4000D801ED91FC910684F785E02D682FC801CE
:108B50001995DD24DA940E941C277C01009709F402
:108B60002DC1DD2021F0F2019783868308C0D50155
:108B700013969C938E931297FC01B582A482C80130
:108B80000E944726B701C80127DE892B09F016C1CC
:108B9000C8010E944726D801ED91FC910284F3851B
:108BA000E02DC8011995D12C57018C32910599F20D
:108BB00021E030E08D35910509F088C085C0BBE724
:108BC000EB16F10409F087C0D801ED91FC91028405
:108BD000F385E02DC80119958B37910509F0EEC09A
:108BE00086E0F2018087C8010E944726D801ED91F6
:108BF000FC910284F385E02DC80119958D3791050C
:108C000009F49BCFD801ED91FC910684F785E02D06
:108C1000682FC8011995BB24BA940E941C277C01B7
:108C2000009709F4CBC0BB2021F0F2019783868323
:108C300008C0D60113969C938E931297FC01D5829F
:108C4000C482C8010E944726B701C8010E94682655
:108C5000019609F4B3C0C8010E944726D7011996AE
:108C60008D919C911A9711969C938E931A961C92B3
:108C70001E921997D801ED91FC910284F385E02DA5
:108C8000C8011995CA9709F099C0C8010E944726E2
:108C9000B701C801A1DD019609F490C0C8010E9486
:108CA0004726D801ED91FC910284F385E02DC8019F
:108CB0001995B12C67018C32910509F4AECF21E0F2
:108CC00030E08D37910511F420E030E088279927B6
:108CD000821B930B75C0BEE6EB16F10411F51982E9
:108CE0001A821B821C82D801ED91FC910484F585C7
:108CF000E02D44E050E0BE016F5F7F4FC801199541
:108D0000049709F05BC044E050E06DE574E0CE01EB
:108D100001960E94C366009709F050C0F2011086C8
:108D20004FC0F6E6EF16F10419F5CE0101967C016D
:108D300085E0D7011D928A95E9F7D801ED91FC9164
:108D40000484F585E02D45E050E0B701C801199590
:108D50000597A1F545E050E067E674E0C7010E9481
:108D6000C366009759F521E0F2012087118628C0DB
:108D7000F4E7EF16F10411F519821A821B821C82A6
:108D8000D801ED91FC910484F585E02D44E050E09C
:108D9000BE016F5F7F4FC8011995049779F444E0D5
:108DA00050E062E674E0CE0101960E94C36600972F
:108DB00029F421E0F2012087218702C08FEF9FEF85
:108DC0002B960FB6F894DEBF0FBECDBFDF91CF91CB
:108DD0001F910F91FF90EF90DF90CF90BF90AF90D9
:108DE0009F908F907F906F905F904F903F902F90CB
:108DF0000895CF92DF92EF92FF92CF93DF93EC0131
:108E00000E94BC146B017C0180915D0990915E0908
:108E1000DC01ED91FC910084F185E02D1995892B01
:108E200079F40E94BC14AB01BC014C195D096E09B8
:108E30007F0948395A436105710530F380E00DC060
:108E400080915D0990915E09DC01ED91FC910284B5
:108E5000F385E02D1995888381E0DF91CF91FF9014
:108E6000EF90DF90CF9008950F931F93CF93DF93F0
:108E7000009789F08C010E941C27EC01892B59F086
:108E8000C8010E944726BE01C801A6DC019631F444
:108E9000CE010E94882C80E090E001C0CE01DF91DD
:108EA000CF911F910F9108959F92AF92BF92CF9251
:108EB000DF92EF92FF920F931F93CF93DF93982E41
:108EC0008B015A01690164E270E00E943A30E82E99
:108ED000F12C65E270E0892D0E943A30FE2CEE24E0
:108EE000E82AE701C00FD11F9E013770E92CF12C51
:108EF000C701880F991FAC014152584F7A01FA01FE
:108F000080819181820F931FA9014C0D5D1D41301D
:108F1000584090F000E018E0021B130BA801B501C7
:108F20000E948D27A601401B510BB501600F711FD8
:108F3000F7018081918102C0A601B5010E948D27B1
:108F4000CC0DDD1D4D2F64E270E0892D0E94303084
:108F50004C2F65E270E0892DDF91CF911F910F9129
:108F6000FF90EF90DF90CF90BF90AF909F900C94C8
:108F70003030FF920F931F93CF93DF93F82EC0E012
:108F8000D0E08F2D0E9444278C01892B21F08F2D5A
:108F90000E944427EC01C017D10799F7CE01DF9159
:108FA000CF911F910F91FF9008955F926F927F92E2
:108FB0008F929F92AF92BF92CF92DF92EF92FF92E9
:108FC0000F931F93CF93DF931F92CDB7DEB74C0162
:108FD0008FE599E00EDF811125C021C00F5F1F4F83
:108FE0008981F801E35AF64F8183282F2F7730E0EB
:108FF0002C9DA0012D9D500D3C9D500D1124A40EC3
:10900000B51E37E0CC0CDD1CEE1CFF1C3A95D1F7E9
:1090100087FF14C0CE010196ECDE8111DFCF80E026
:1090200090E085C070905F09198201E010E0A12CEA
:10903000B12CC12CD12C7601C394ECCF872D807F2D
:1090400055245394803309F0512C8FEF800FD401B5
:109050008C93552011F1C801815A964FCADE88239E
:10906000F1F2C801805A964FC4DE8823C1F20E5F28
:109070001F4FD401EC91F0E0E35AF64FE380F12C5E
:10908000FE2CEE248481E80EF11C80915F0981FFA3
:1090900008C0B2E0EB0EF11C04C080E0E12CF12C22
:1090A00001C082E0C82ED12CC01AD10A9EEF692ED1
:1090B00077247A94C601800F911F8A159B0560F56D
:1090C000CE01019696DE882309F4A9CF8091F60996
:1090D0009091F7090097A9F0552099F0F4012081AB
:1090E000A301421B51099A01200F311FE216F3061A
:1090F00040F4DC01ED91FC910190F081E02D69815B
:1091000019950038110528F48981F801E35AF64FC2
:1091100082830F5F1F4FCECF8091F6099091F709A0
:10912000892B21F40138110508F079CFC8010F907F
:10913000DF91CF911F910F91FF90EF90DF90CF9033
:10914000BF90AF909F908F907F906F905F900895A9
:10915000089580E090E008958F929F92AF92BF9221
:10916000CF92DF92EF92FF920F931F93CF93DF93F3
:10917000CDB7DEB7A5970FB6F894DEBF0FBECDBF53
:109180005C018B017B01E40EF51ED7011C926DEF93
:1091900079E086EA98E00E948E11B50186EA98E0AF
:1091A0000E94D7126BEE74E086EA98E00E94D71214
:1091B000FE0131966F012091940B3091950B211592
:1091C000310511F42EE93BE0C601821B930B8A3F67
:1091D00091053CF468EF79E086EA98E00E94C712B6
:1091E000A5C019821A821B821C82FE01359680E17D
:1091F000DF011D928A95E9F748018E149F0441F022
:10920000F40161914F0186EA98E00E948711F5CF41
:1092100086EA98E00E949F12C8010E94BD0E7C0160
:109220006FE270E0C5010E94E066009741F0BC016A
:109230006F5F7F4F43E150E0C6010E94D166B601E7
:10924000CE0145960E94D907CE0145960E949D0603
:10925000882309F46BC0E114F10469F03CF4FEEFDB
:10926000EF16FFEFFF060CF061C056C021E0E216DA
:10927000F10471F151C06E018EE1C80ED11CE12CD8
:10928000F12C960101151105F1F0B3E0EB16F10494
:10929000D1F09FEFE91AF90AC8012CA33DA30E945F
:1092A000445B5C016CE270E0C8010E9498668C012E
:1092B0002CA13DA1892B11F00F5F1F4FD601AD925C
:1092C000BD926D01DFCF00E0A70160E070E02AC031
:1092D0000E94BC1400918E0B10918F0B2091900B6B
:1092E0003091910BDC01CB01801B910BA20BB30BD6
:1092F000853F9140A105B10540F000E020E030E05D
:1093000040E050E061E070E00DC06EEE74E086EA8F
:1093100098E00E94B7120AC000E020E030E040E090
:1093200050E0B701CE0145960E94F207A5960FB610
:10933000F894DEBF0FBECDBFDF91CF911F910F918B
:10934000FF90EF90DF90CF90BF90AF909F908F9065
:1093500008956BEA73E089EF94E00C94B22B1F93AD
:10936000CF93DF9363E17AE086EA98E00E948E1162
:10937000CCE2D5E01C2F1A5F499150E060E070E02C
:1093800020E186EA98E00E94C71161E17AE086EA6E
:1093900098E00E948E111C13EFCF86EA98E0DF91CF
:1093A000CF911F910C949F12AF92BF92CF92DF92F8
:1093B000EF92FF920F931F93CF93DF9300D000D0D3
:1093C000CDB7DEB761E07AE086EA98E00E948E11C0
:1093D0008E010D5F1F4F7E0187E0E80EF11C5801E2
:1093E00083EAC82E83E0D82EDA82C9821B821C82CF
:1093F0001D821E8280E590E00E94A23E44E050E083
:10940000B5018FE090E00E9463270E94A13EF80121
:1094100041918F0150E060E070E02AE086EA98E038
:109420000E94C7116FEF79E086EA98E00E948E11E2
:109430000E151F05C9F686EA98E00E949F1226962F
:109440000FB6F894DEBF0FBECDBFDF91CF911F9155
:109450000F91FF90EF90DF90CF90BF90AF90089565
:109460005F926F927F928F929F92AF92BF92CF92B4
:10947000DF92EF92FF920F931F93CF93DF93CDB7BD
:10948000DEB7E4970FB6F894DEBF0FBECDBF5C0128
:109490007B016A01890119A21AA21BA21CA2FE016A
:1094A000B5968CE0DF011D928A95E9F76FEE73E0C7
:1094B000CE0101960E94695BD5011296ED91FC9157
:1094C00013976081718140E250E0CE0101960E94C5
:1094D000B366B2E0EB16F104A1F054F4E114F10428
:1094E000B9F0EA94EF2809F076C06BEA73E00BC09C
:1094F00085E0E816F10429F099E0E916F10441F05D
:109500006AC06EEA73E0CE0181960E94AC6645C0E7
:109510000115110509F441C0612C712C82E1A82EBE
:1095200085E0B82E94E0592E7E01A1E3EA0EF11CED
:109530004601B1E08B1A91086C147D0474F5F801B2
:10954000808191810E5F1F4F9F938F93BF92AF9247
:109550001F925F92FF92EF920E94EB6640E150E013
:10956000B701CE0181960E94B3660FB6F894DEBFB4
:109570000FBECDBF6814790461F065E175E0C701E5
:109580000E94AC6640E150E0B701CE0181960E9496
:10959000B3669FEF691A790ACFCFBE016F5F7F4F25
:1095A00086EA98E00E94D71265EF79E086EA98E0B3
:1095B0000E948E11BE016F5D7F4F86EA98E00E9487
:1095C000B712BE016F5D7F4FCE0101960E94B22B94
:1095D00080E090E002C08FEF9FEFE4960FB6F89422
:1095E000DEBF0FBECDBFDF91CF911F910F91FF90D6
:1095F000EF90DF90CF90BF90AF909F908F907F9033
:109600006F905F900895EF92FF920F931F93CF9307
:10961000DF9300D000D0CDB7DEB78C017B0162E0D4
:1096200070E00E940607892B19F4E982FA8205C0CE
:109630008F2D880F880BF9828A83A981BA81BB2775
:1096400024E630E00E9436662FE330E040E050E050
:109650000E9459623A832983C8012B833C834D833E
:109660005E830E943207E82EF12CC8010E94E206B8
:109670002B813C814D815E816217730784079507BA
:1096800079F4672B682B692B09F44AC082E0E8164D
:10969000F10471F085E0E816F10409F041C008C05A
:1096A000232B242B252B41F182E0E816F104F9F459
:1096B00020E030E040E050E061E070E0C801D0DE42
:1096C0009E012F5F3F4F41E050E060E070E0C80135
:1096D000C7DE61E0C8010E941D0749815A81052E3D
:1096E000000C660B770BC8010E94AA0619C085E022
:1096F000E816F10429F7DCCF85E0E816F10481F0E3
:1097000082E0E816F10461F062E0C8010E941D07E2
:1097100020E030E040E050E062E070E0C801A0DE10
:1097200080E090E026960FB6F894DEBF0FBECDBF66
:10973000DF91CF911F910F91FF90EF900895AF921D
:10974000BF92CF92DF92EF92FF920F931F93CF932E
:10975000DF93CDB7DEB7C154D1090FB6F894DEBFA1
:109760000FBECDBFCB018A014EE459E46CE470E03A
:1097700049835A836B837C83FE0135962CE1DF019C
:109780001D922A95E9F74AAB5BAB6CAB7DABF196CA
:109790002CE0DF011D922A95E9F7AE014F5D5F4F86
:1097A00068E00E9413381AAABE016F5D7F4F809156
:1097B0004F05909150050E9491437C01009771F1F3
:1097C00062E274E00E949143FC01C184D284C1141E
:1097D000D104C9F041E150E0B601CE0181960E946A
:1097E000D166B60186EA98E00E94D71261E174E082
:1097F00086EA98E00E94D7124AE050E0B80186EA73
:1098000098E00E94A21263E174E0C7010E949143B4
:10981000DC011996ED90FC901A9708C063E37AE09A
:1098200086EA98E00E94C712E12CF12C0138BFEFC4
:109830001B0709F4C3C00535110509F4BFC064E274
:109840007AE0CE0101960E94695B40E250E0BE01E1
:109850006F5D7F4FCE0101960E94B3661F930F93F9
:1098600082E195E09F938F936E01E2E3CE0ED11CCF
:10987000DF92CF920E942867B601CE0101960E9426
:10988000B22B0F900F900F900F900F900F90E1144C
:10989000F10409F493C080914A0590914B0500971B
:1098A00009F48CC0B7010E9491437C01009709F430
:1098B00085C0DC0118968C91853009F07FC060E08E
:1098C000C7010E948443FC0181859285A385B485EC
:1098D0000597A105B10509F071C0C7010E94DD2AF5
:1098E000843008F46BC08430B1F50E941C276C01F1
:1098F000892B21F085E0D60118968C930E941C27B5
:109900005C01892B59F082E0F5018087012E000C63
:10991000220B330B01871287238734870E941C2771
:109920008C01892B59F082E0F801808788EC90E067
:10993000A0E0B0E081879287A387B487B501C60114
:109940000E94CF43B801C6010E94CF43B601C701B0
:109950000E94CF4333C064E0C7010E9484436C017E
:10996000009761F161E00E9484435C0160E0C60100
:109970000E948443012E000C220B330BDC0119964C
:109980000D931D932D933C931C97F5018185928532
:10999000A385B485892B8A2B8B2B39F4D7016D9144
:1099A0007C9187E195E00E94B22B88EC90E0A0E0EA
:1099B000B0E0F50181879287A387B487CF5BDF4F43
:1099C0000FB6F894DEBF0FBECDBFDF91CF911F91D0
:1099D0000F91FF90EF90DF90CF90BF90AF900895E0
:1099E0002F923F924F925F926F927F928F929F92AF
:1099F000AF92BF92CF92DF92EF92FF920F931F939D
:109A0000CF93DF9300D0CDB7DEB72DB63EB60E9420
:109A10007D2B982E882309F441C10E94BC146B0150
:109A20007C018091E5099091E609A091E709B09148
:109A3000E809A7019601281B390B4A0B5B0BDA01D9
:109A4000C90189399A43A105B105A8F48091E109BA
:109A50009091E209A091E309B091E409A701960170
:109A6000281B390B4A0B5B0BDA01C90189399A4370
:109A7000A105B105D0F12091E90980915D0990918E
:109A80005E09222379F02CEF3FEF3093F909209300
:109A9000F809DC01ED91FC910488F589E02D199518
:109AA000912CFCC020EC20935F0910926009DC012E
:109AB000ED91FC910280F381E02D42E050E06FE5F2
:109AC00079E01995C092E109D092E209E092E309A8
:109AD000F092E409C092E509D092E609E092E70924
:109AE000F092E80981E08093E90980915D09909105
:109AF0005E09DC01ED91FC910084F185E02D199562
:109B0000892B09F4CBC0CE0101964FDA8C01892B49
:109B100009F4C4C0C092E509D092E609E092E709D1
:109B2000F092E80970905F09872D807F803309F0FB
:109B30009AC0E091EA09F091EB09FB83EA83EF2BED
:109B400009F4ACC04DB65EB6A981B0E0CD01835A30
:109B5000964FFC01638170E0762F66278481680F41
:109B6000711DCB0101962DB73EB7281B390B0FB6DF
:109B7000F8943EBF0FBE2DBF4DB75EB74F5F5F4F2E
:109B80005A0120E030E02617370769F0C9018A0F33
:109B90009B1F835A964FFC018581FA018193AF0187
:109BA0002F5F3F4FF0CFC501820F931FFC01108242
:109BB000F72DF6708F2E42E0F4133EC0B9016A0F04
:109BC0007B1FAB01435A564FFA01858190E0982FD5
:109BD000882746813C01640E711C4BEF5FEF4A1BE6
:109BE0005B0B421B530B400F511F6C59764FC50145
:109BF000EA81FB81199580E480935F098092600976
:109C0000709261096092620980915D0990915E098C
:109C1000DC01ED91FC910280F381E02D44E050E005
:109C20006FE579E01995C092E109D092E209E092DE
:109C3000E309F092E40911C04DEF5FEF4A1B5B0BA3
:109C4000421B530B400F511F2A0F3B1FB9016E5986
:109C5000764FC501EA81FB8119950FB6F8945EBE77
:109C60000FBE4DBE1BC0803CA9F480ED80935F0900
:109C70001092600980915D0990915E09DC01ED917F
:109C8000FC910280F381E02D42E050E06FE579E045
:109C9000199504C0803D11F41092E909892D0FB681
:109CA000F8943EBE0FBE2DBE0F900F900F90DF9127
:109CB000CF911F910F91FF90EF90DF90CF90BF90C9
:109CC000AF909F908F907F906F905F904F903F905C
:109CD0002F900895CF93DF93CDB7DEB7C956D10942
:109CE0000FB6F894DEBF0FBECDBF789484B5826006
:109CF00084BD84B5816084BD85B5826085BD85B530
:109D0000816085BD80916E00816080936E001092AD
:109D10008100809181008260809381008091810028
:109D200081608093810080918000816080938000B9
:109D30008091B10084608093B1008091B000816017
:109D40008093B00080919100826080939100809117
:109D50009100816080939100809190008160809358
:109D600090008091A10082608093A1008091A10069
:109D700081608093A1008091A00081608093A00009
:109D80008091210182608093210180912101816075
:109D90008093210180912001816080932001809136
:109DA0007A00846080937A0080917A008260809348
:109DB0007A0080917A00816080937A0080917A00A5
:109DC000806880937A001092C10084E595E09093BA
:109DD00091058093900510922B0510922A0526E09C
:109DE00040E052EC61E070E086EA98E00E948C135B
:109DF0006AE173E086EA98E00E94C71286E0EAE131
:109E0000F2E0DE01119601900D928A95E1F76CE285
:109E1000C62E65E0D62EE12CF12C00E010E0C80142
:109E20000E942162D6018D936D0181508E3F18F4FE
:109E3000EE24E394F12C0F5F1F4F0630110579F7E4
:109E4000EF2879F461E073E086EA98E00E94C71297
:109E500086E0FE013196ACE2B5E001900D928A9564
:109E6000E1F77DDA60E070E080E090E00E9424435A
:109E700061E08DE00E94481426E040E855E260E091
:109E800070E089E098E00E948C1380ED9FE390934E
:109E90000F0B80930E0B85EE9FE39093110B809335
:109EA000100B81EE9FE39093130B8093120B64E1F0
:109EB00070E080E090E00E94841410925105E091DF
:109EC0003605F0913705309721F086EC9FE3908BB3
:109ED00087878CEA98E49093EB098093EA09809154
:109EE000520590915305892B59F488E392E00E9422
:109EF000C2598C010E94AF2F109353050093520555
:109F00008091520590915305009739F0FC01EA5C6D
:109F1000FD4F81E595E09183808362E17AE385ECF2
:109F200093E00E94EC2465E470E48AEC93E00E94E4
:109F3000EC2462E873E48FEC93E00E94EC2467E188
:109F400073E484ED93E00E94EC2469EE7FE388EDF6
:109F500093E00E94EC2468E17AE38CED93E00E94A8
:109F6000EC2463E870E481EE93E00E94EC24EE249C
:109F7000E394F12CA89586EA98E00E940810892BBA
:109F800009F493C086EA98E00E94E60F182F8A3001
:109F900031F08D3021F0883009F076C060C0E0915A
:109FA0009005F0919105108265EE73E086EA98E0E5
:109FB0000E94D7126DE074E084E595E00E94705B2A
:109FC0009A838983FE0133966F0101E010E0B02E81
:109FD000A12E6DE074E080E090E00E94705BD601FD
:109FE0008D939D936D010E31110539F40091320569
:109FF00010913305C980DA8008C00F5F1F4F892B8D
:10A0000031F7F4CFF8010481158101151105A1F094
:10A01000F80160817181C6010E94A366892B91F7C6
:10A02000D8011296ED91FC911397BE016F5F7F4F9F
:10A030008B2D9A2D199506C061E473E086EA98E0AD
:10A040000E94C71286EA98E00E949F1261E573E0C1
:10A0500086EA98E00E948E1184E595E010C068E0E1
:10A0600086EA98E00E948711809190059091910571
:10A07000F5E084359F0709F008F47DCF01979093B0
:10A0800091058093900577CF682F86EA98E00E942B
:10A090008711E0919005F0919105CF010196909381
:10A0A000910580939005108366CF0E94B3170297A5
:10A0B0004CF096DC8091520590915305009711F079
:10A0C0000E94301680915105882309F48BC280913B
:10A0D0004F0590915005892B09F484C20E94BC144D
:10A0E0000091940510919505209196053091970562
:10A0F000601771078207930708F474C20E94BC14AA
:10A100002B013C0180913E0590913F05009709F499
:10A1100057C2209192053091930560913C05709152
:10A120003D05261737070CF42CC10E94BC149B0177
:10A13000AC0128573C4E4F4F5F4FAA962CAF3DAF16
:10A140004EAF5FAFAA976EE773E086EA98E00E9491
:10A15000C712E0913605F0913705309739F4E09158
:10A160003405F091350580E090E00BC08FEF8387D8
:10A170001486DF0113963B961D92AE17BF07E1F7D9
:10A18000EECF20913C0530913D05821793070CF0EE
:10A1900081C0208131812E7F219331930196F1CFAF
:10A1A00060913C0570913D05A3E0660F771FAA956D
:10A1B000E1F720913A0530913B05620F731F0E9431
:10A1C000A22018160CF022C6C0903C05D0903D0588
:10A1D000B4E1CB16D1040CF019C60E94BC14AA96A7
:10A1E0002CAD3DAD4EAD5FADAA97621773078407E6
:10A1F000950708F00BC6A0903A05B0903B054601C4
:10A2000033E0880C991C3A95E1F78A0C9B1C67E0B7
:10A21000C4010E94AA1FD40117969C9189133AC0C9
:10A2200000E010E00C151D05ECF548E050E0B4012D
:10A23000C5010E946D66B8E0AB0EB11C892BC9F553
:10A24000000F111FE0913405F0913505E00FF11F6B
:10A250008081918181609183808367E773E086EAE2
:10A2600098E00E948E1180913C0590913D0523E07D
:10A27000880F991F2A95E1F720913A0530913B0507
:10A28000820F931F0E943E2E60E773E086EA98E0FB
:10A290000E94C7128091360590913705009709F00A
:10A2A0007FCFB4C580913E0590913F05892B21F465
:10A2B000F1CF0F5F1F4FB6CF80913C0590913D05C8
:10A2C000880F991F2091340530913505F901E80F69
:10A2D000F91F21E030E0318320836BE673E086EAEA
:10A2E00098E00E948E1160913C0570913D054AE016
:10A2F00050E086EA98E00E94561264E673E086EA2F
:10A3000098E00E948E1180913C0590913D0513E0EC
:10A31000880F991F1A95E1F720913A0530913B0576
:10A32000820F931F0E943E2E86EA98E00E949F12A1
:10A3300060913C0570913D0503E0660F771F0A951B
:10A34000E1F780913A0590913B05680F791FDB0199
:10A350008C91883261F480913E0590913F050E9476
:10A36000BC2D80913605909137050E947520809113
:10A370003C0590913D05019690933D0580933C05E9
:10A3800089CF00913A0510913B05A901F3E0440FF4
:10A39000551FFA95E1F7040F151FD8014C9148326B
:10A3A00009F003C1AE01435C5F4FB8010E94DE219A
:10A3B000882379F16DADB8E06B9FB00111242EAD0B
:10A3C00030E0322F2227330F330F330F262B372B5A
:10A3D000F8018081803101F525966FAD259770E0F9
:10A3E00024968FAD2497AB01481B5109CA0196955D
:10A3F000982F8827979587950E9414666051710958
:10A40000207F53E0220F331F5A95E1F7620F731F2D
:10A4100004C060E874EE01C0B901613854EE7507FC
:10A420006CF0072E000C880B990B0E94986320E0BB
:10A4300030E040E05CE30E944C6404C060E070E007
:10A440008EEF92EC0E946563E0913805F09139053A
:10A450003097A1F00091920510919305980193E037
:10A46000220F331F9A95E1F7A0913A05B0913B0571
:10A470002A0F3B1FAB01B901C80119950091920544
:10A480001091930583E0000F111F8A95E1F78091E9
:10A490003A0590913B05080F191FC0903E05D090DA
:10A4A0003F05D8018C91803149F0B801C6010E9466
:10A4B000EF21B82E882309F46CC002C0BCE0BB2E8B
:10A4C000F601858196810E944A20882309F461C0A3
:10A4D000B801D60115968D919C9116970E945A212C
:10A4E000F601408164E4858196810E947F20D60137
:10A4F00012968C91882309F44CC0E7EFEB0DE33002
:10A5000040F4F0E0EE0FFF1FE05EFD4F2080318051
:10A5100004C07EEE272E72E0372E0115110599F149
:10A52000F6018381882379F1808181112CC00E94FA
:10A53000BC144B015C019101330C440B550BAA96E2
:10A540002CAF3DAF4EAF5FAFAA97AE01435C5F4FFC
:10A55000B801C6010E9485218DAD81111AC00E94EB
:10A56000BC14DC01CB01AA962CAD3DAD4EAD5FAD68
:10A57000AA97821B930BA40BB50B88159905AA0506
:10A58000BB0518F306C0B101330C880B990B0E9470
:10A590008414809192059091930501969093930570
:10A5A0008093920564EC79E00DC02F5F3F4F3093AC
:10A5B00093052093920580ED97E00E94146602C0F7
:10A5C0006FEF7FEFCB01770FAA0BBB0B480E591E25
:10A5D0006A1E7B1E409294055092950560929605E6
:10A5E000709297050E94BC1480914005909141059E
:10A5F000A0914205B09143050E94050F80914C0542
:10A6000090914D05892B09F4DDC280914A05909106
:10A610004B05892B09F4D6C20E94BC140091980501
:10A620001091990520919A0530919B0506171707FF
:10A630002807390708F0C6C2D12C9AE0292E312C00
:10A6400023E1422E512C34E0A32EB12C4EE3842E74
:10A6500048E0942E0091460510914705011511051B
:10A6600009F4B0C2D110AEC2D80118968C918530D1
:10A6700009F091C260E0C8010E948443FC01818519
:10A680009285A385B48584309105A105B10529F093
:10A690000997A105B10509F07EC22AE232E06F9662
:10A6A0003FAF2EAF6F97A1961FAF0EAFA197CE0110
:10A6B000835A9F4F0E943F07A6968FADA69784307E
:10A6C00021F0893009F4A5C054C2809144059091CD
:10A6D0004505892B09F04DC2F0924505E0924405ED
:10A6E00060E070E0CE01835A9F4F0E9406073C0154
:10A6F00061E070E0CE01835A9F4F0E9406076C0113
:10A7000026E240E855E260E070E089E098E00E94CF
:10A710008C136092FC0989E098E09093FB09809388
:10A72000FA091092070B1092090B1092080BD092A5
:10A73000FE09C092FD09F092000AE092FF0983E051
:10A740000E940C28182F811118C00091010A109145
:10A75000020A6EE973E086EA98E00E948E1140E1F9
:10A7600050E0B80186EA98E00E94A212B801CE013A
:10A77000835A9F4F0E94034B0DC068E873E086EA3E
:10A7800098E00E948E1160E170E0812F0E94AC433E
:10A7900000E010E01092450510924405E091460556
:10A7A000F0914705828193814AE252E05EAF4DAF5E
:10A7B00021969FAF8EAF2197CE01CD960E943F0785
:10A7C0008091460590914705892B09F4D2C1CE01AD
:10A7D000CD960E949D06882309F4CBC126968FADA5
:10A7E0002697843009F0C5C160E070E0CE01CD96B7
:10A7F0000E9406078615970509F0BBC161E070E06D
:10A80000CE01CD960E9406078C159D0509F0B1C1B9
:10A8100014C38091440590914505892B09F0A9C185
:10A82000F0924505E09244050E941C278C01892B7B
:10A8300021F086E0D80118968C936FEE73E0CE017C
:10A84000CD9647D7A196EEADFFADA19760817181FE
:10A850004FE150E0CE01CD960E94B36668EE73E002
:10A86000CE01CD960E948D6626E040E855E260E07C
:10A8700070E089E098E00E948C1360E070E0CE0107
:10A88000835A9F4F0E9406078093FC0989E098E055
:10A890009093FB098093FA091092070B1092090B11
:10A8A0001092080BE4E3F8E0F093FE09E093FD0951
:10A8B0003092000A2092FF0983E00E940C28D82ED3
:10A8C00081117BC065EE73E086EA98E00E948E11EC
:10A8D00061E0C62E6AE0D62ED6016D917D916D01A4
:10A8E00040E150E086EA98E00E94561263EE73E081
:10A8F00086EA98E00E948E11B5E1CB16BAE0DB063D
:10A9000059F76091050A7091060A072E000C880B12
:10A91000990B0E94986320E030E048EC52E40E94DA
:10A92000FD629B01AC016EEE73E0C8010E94002C39
:10A930004091090A50910A0A60EF73E0C8010E9431
:10A94000D32760910B0A70910C0A072E000C880B1C
:10A95000990B0E94986320E030E048EC52E40E949A
:10A96000FD629B01AC0164EF73E0C8010E94002C02
:10A9700060910D0A70910E0A072E000C880B990B3E
:10A980000E94986320E030E040E251E40E94FD62C2
:10A990009B01AC0162EF73E0C8010E94002C409162
:10A9A000010A5091020A66EF73E0C8010E94D327A2
:10A9B00086EA98E00E949F120BC06DEC73E086EA75
:10A9C00098E00E948E1160E170E08D2D0E94AC43F2
:10A9D0008091010A83FF12C09092FE098092FD09C6
:10A9E000F092000AE092FF0983E00E940C28811196
:10A9F0000CC04091010A5091020A02C040E050E0B0
:10AA000069EF73E0C8010E94D32762E370E080E041
:10AA100090E00E9484145092FE094092FD09B09289
:10AA2000000AA092FF0983E00E940C28D82E811111
:10AA300083C063EC73E086EA98E00E948E1151E0D7
:10AA4000C52E5AE0D52EF601619171916F014AE051
:10AA500050E086EA98E00E94561261EC73E086EAC4
:10AA600098E00E948E11F9E0CF16FAE0DF0659F760
:10AA70006091010A7091020A61157105C9F0072EF3
:10AA8000000C880B990B0E9498632DEE3EE94CE375
:10AA90005EE30E944C6422E538EB42E152E40E94FE
:10AAA00094629B01AC0168ED73E0C8010E94002C28
:10AAB0006091030A7091040A072E000C880B990B11
:10AAC0000E9498632DEE3EE94CE35EE30E944C64E5
:10AAD00022E538EB42E152E40E9494629B01AC0112
:10AAE0006CEE73E0C8010E94002C6091070A70911F
:10AAF000080A16161706A4F4072E000C880B990BEB
:10AB00000E94986320E030E040E251E40E94FD6240
:10AB10009B01AC016DEF73E0C8010E94002C07C0DF
:10AB200040E050E06DEF73E0C8010E94D32786EA51
:10AB300098E00E949F120BC06BEA73E086EA98E0EF
:10AB40000E948E1160E170E08D2D0E94AC43C8011F
:10AB50000E944A2C6C01BC01CE01CD960E94B22B02
:10AB6000C601A5D4C8010E94882C109245051092F8
:10AB700044050E94BC14DC01CB018053984FAF4FB9
:10AB8000BF4F8093980590939905A0939A05B09331
:10AB90009B05DD24D394E0914605F0914705828121
:10ABA00093819093470580934605892B09F052CDF8
:10ABB000E0914A05F0914B05868197819093470576
:10ABC0008093460500914A0510914B05011511052A
:10ABD00009F47BC00E94BC1480909C0590909D0558
:10ABE000A0909E05B0909F0586169706A806B90608
:10ABF00008F06BC0D80116960D911C91179701159E
:10AC0000110509F43FC0F80180858530A9F560E0A1
:10AC1000C8010E948443FC0181859285A385B48587
:10AC20000597A105B10541F5C8010E94DD2A8530CF
:10AC300018F161E0C8010E948443FC01318462E0A4
:10AC4000C8010E948443DC011996AD90BC901A970C
:10AC500063E0C8010E948443FC018184928464E023
:10AC6000C8010E9484436C01892B31F0C6010E9407
:10AC7000DD2A823008F0FEC0D80112960D911C9199
:10AC80001397BDCF0E94BC14DC01CB0188579C4EAA
:10AC9000AF4FBF4F80939C0590939D05A0939E0559
:10ACA000B0939F05BE01635C7F4F8091940B9091A0
:10ACB000950B009711F48EE99BE0681B790B4AE035
:10ACC00050E086EA98E00E94A21200914805109197
:10ACD00049050115110509F496C00E94BC14809025
:10ACE000A0059090A105A090A205B090A30586169E
:10ACF0009706A806B90608F086C0F801C680D78076
:10AD000083E0282EC114D10409F46EC0D601189630
:10AD10008C91863009F062C061EC73E0C6010E943C
:10AD20009143009719F0FC01018501C000E0D601B4
:10AD30008D919C91A9D4182F68E074E0C6010E94FF
:10AD400091435C01892B49F56AE074E086EA98E05A
:10AD50000E94D712412F50E060E070E02AE086EABE
:10AD600098E00E94C7116FE074E086EA98E00E94C4
:10AD7000D7126AE070E0802F0E94AC4340E050E0C0
:10AD800068E074E0C6010E94D32768E074E0C60161
:10AD90000E9491435C01892B09F11123F9F007FF0F
:10ADA00017C160E0812F0E944814812F0E94F11387
:10ADB00033243394019709F017C1632C712CF501EA
:10ADC0008485082E000C990B6816790609F49FC13A
:10ADD0008385882309F40AC181508387D60112969E
:10ADE000CD90DC9013978ECF0E94BC14DC01CB0178
:10ADF000C296A11DB11D8093A0059093A105A093BB
:10AE0000A205B093A3050E94AE10B4C865E573E037
:10AE100086EA98E00E948E1160913C0570913D0594
:10AE20004AE050E086EA98E00E94A2121092930550
:10AE30001092920560E47FE1C5CBB801CE01CD96BA
:10AE40000E94034BE0914605F09147058281938172
:10AE50009093470580934605892B09F08ACEE091AF
:10AE60004A05F0914B058681978190934705809321
:10AE700046057FCE60E0C6010E948443DC0119963E
:10AE80004D905D906D907C901C9761E0C6010E9492
:10AE90008443FC012185328543855485D8016D9119
:10AEA0007C91211531054105510559F486EA98E058
:10AEB0000E94D71266E274E086EA98E00E94C71208
:10AEC00013C02150310941095109DC0119962D9314
:10AED0003D934D935C931C97232B242B252B21F41E
:10AEE00081E094E00E94B22BA8965FAE4EAEA89788
:10AEF000F8016081718186EA98E00E94D71260E2D1
:10AF000074E086EA98E00E948E114AE050E0B501B4
:10AF100086EA98E00E94561266E174E086EA98E0BC
:10AF20000E948E114AE050E0B20186EA98E00E9449
:10AF3000561260E174E086EA98E00E948E114AE0C1
:10AF400050E0B40186EA98E00E94561261E0832D39
:10AF50000E944814F2E08F16910489F025E08216D1
:10AF6000910469F061E0C6010E948443FC0181857F
:10AF70009285A385B485892B8A2B8B2B59F460E0AD
:10AF8000832D0E9419146BE074E086EA98E00E9419
:10AF9000C71272CEB2E04B0E511C4A145B043CF453
:10AFA00061E0832D0E94191467E074E0EECFA8964B
:10AFB0002EAD3FADA8972A153B053CF060E0832DF0
:10AFC0000E94191462E074E0E0CF6EEF73E0DDCF11
:10AFD00062E0812F0E944814812F0E94F1133324D4
:10AFE0003394892B09F4E9CE312CE7CE412F50E080
:10AFF00060E070E02AE086EA98E00E94C71161E113
:10B0000074E086EA98E00E94D7124AE050E0B3016B
:10B0100086EA98E00E94A21263E174E0C6010E94F1
:10B0200091432C0168E174E0C6010E9491434C01F8
:10B030006DE174E0C6010E9491438C0162E274E00C
:10B04000C6010E949143FC01892BF1F06114710447
:10B0500041F08114910419F46BEA73E011C0D4013A
:10B0600007C00115110519F46EEA73E009C0D80193
:10B0700019966D917C911A97DB018C91882321F0B0
:10B08000818592850E94B22B41145104E1F1F201B5
:10B0900061857285CE01CD960E94D907CE01CD96ED
:10B0A0000E949D06882379F1672869F08114910434
:10B0B00041F401E020E030E040E050E061E070E089
:10B0C0001EC0D4010CC00115110541F401E020E0BF
:10B0D00030E040E050E062E070E011C0D801199625
:10B0E0008D919C911A97FC012081222361F00E948E
:10B0F000BD0E01E020E030E040E050E0BC01CE01B8
:10B10000CD960E94F207D5011C963C9267CEF501C0
:10B11000238664CE0F931F93E4E1FBE083EA93E080
:10B12000918380831282138214821582E9E0F8E011
:10B130001382128248EE53E060E070E0448355834E
:10B14000668377832DE133E031832083A5EDB0E082
:10B15000B587A487A4EDB0E0B787A687A0EDB0E0DF
:10B16000B18BA08BA1EDB0E0B38BA28BA2EDB0E0D0
:10B17000B58BA48BA6EDB0E0B78BA68B118E128E8B
:10B18000138E148EE6EAF8E013821282448355830C
:10B19000668377833183208325EC30E035872487ED
:10B1A00024EC30E03787268720EC30E0318B208B91
:10B1B00021EC30E0338B228B22EC30E0358B248B7A
:10B1C00026EC30E0378B268B118E128E138E148E68
:10B1D000EAE1FBE02FEF20831282118214861386AE
:10B1E0000FEF1FEF98010783108721873287E7E26F
:10B1F000FBE0918380831282138214821582E3E440
:10B20000F9E01382128244835583668377832FE2A9
:10B2100033E031832083EDE2FBE09183808312826F
:10B22000138214821582E3E3FBE091838083128210
:10B23000138214821582E9E3FBE0918380831282FA
:10B24000138214821582EFE3FBE0918380831282E4
:10B25000138214821582E5E4FBE0918380831282DD
:10B26000138214821582EBE4FBE0918380831282C7
:10B27000138214821582E1E5FBE0918380831282C0
:10B28000138214821582EFE4F9E0918380831282A5
:10B29000138214821582E7E5F9E09183808312829C
:10B2A000138214821582E7E5FBE09183808312828A
:10B2B000138214821582EDE5FBE091838083128274
:10B2C000138214821582E3E6FBE09183808312826D
:10B2D000138214821582E6E7FBE091838083128259
:10B2E00013821482158210920F0B10920E0B109283
:10B2F000110B1092100B1092130B1092120BE9E627
:10B30000FBE01382128244835583668377832DE7A3
:10B3100033E03183208324E024879093ED098093E8
:10B32000EC091092EE091092EF091092F0091092B8
:10B33000F1092FEF3FEF3093F9092093F809F093CB
:10B340005E09E0935D091092F7091092F609ECE7A7
:10B35000FBE0918380831282138214821582E2E8DB
:10B36000FBE0918380831282138214821582E8E8C5
:10B37000FBE09183808312821382148215821F91D5
:10B380000F910895CF93DF938230910510F482E0FE
:10B3900090E0E091960BF091970B20E030E0C0E058
:10B3A000D0E0309711F14081518148175907C0F022
:10B3B0004817590761F482819381209719F09B8384
:10B3C0008A832BC09093970B8093960B26C02115F0
:10B3D000310519F04217530718F49A01BE01DF0135
:10B3E000EF010280F381E02DDCCF2115310509F159
:10B3F000281B390B2430310590F412968D919C91C5
:10B4000013976115710521F0FB019383828304C0BA
:10B410009093970B8093960BFD01329644C0FD01EB
:10B42000E20FF31F81939193225031092D933C93A6
:10B430003AC02091940B3091950B232B41F420912D
:10B440000A0230910B023093950B2093940B2091BC
:10B450000802309109022115310541F42DB73EB79C
:10B4600040910C0250910D02241B350BE091940B7E
:10B47000F091950BE217F307A0F42E1B3F0B281752
:10B48000390778F0AC014E5F5F4F2417350748F05D
:10B490004E0F5F1F5093950B4093940B81939193A4
:10B4A00002C0E0E0F0E0CF01DF91CF9108950F936B
:10B4B0001F93CF93DF93009709F48CC0FC01329760
:10B4C000138212820091960B1091970B01151105B2
:10B4D00081F420813181820F931F2091940B309150
:10B4E000950B2817390779F5F093950BE093940B9A
:10B4F00071C0D80140E050E0AE17BF0750F412967B
:10B500002D913C911397AD012115310509F1D90118
:10B51000F3CF9D01DA013383228360817181860F2D
:10B52000971F8217930769F4EC0128813981260F50
:10B53000371F2E5F3F4F318320838A819B81938306
:10B540008283452B29F4F093970BE093960B42C02E
:10B550001396FC93EE931297ED01499159919E0138
:10B56000240F351FE217F30771F480819181840F56
:10B57000951F029611969C938E93828193811396C8
:10B580009C938E931297E0E0F0E0D80112968D9193
:10B590009C911397009719F0F8018C01F6CF8D91CB
:10B5A0009C9198012E5F3F4F820F931F2091940B27
:10B5B0003091950B2817390769F4309729F41092C8
:10B5C000970B1092960B02C0138212821093950B68
:10B5D0000093940BDF91CF911F910F9108958F925B
:10B5E0009F92AF92BF92CF92DF92EF92FF92CF9352
:10B5F000DF93EC01688179818A819B8161157105F6
:10B600008105910521F464E279ED8BE597E02DE168
:10B6100033EF41E050E04DD749015A019B01AC01A5
:10B62000A7EAB1E462D76B017C01ACEEB4EFA501EF
:10B63000940167D7DC01CB018C0D9D1DAE1DBF1D94
:10B64000B7FF03C00197A109B04888839983AA83F3
:10B65000BB83BC01CD019F77DF91CF91FF90EF902D
:10B66000DF90CF90BF90AF909F908F900895B7CF0D
:10B670008EE092E0B4CF60930E0270930F0280933D
:10B680001002909311020895FC0188279927E894ED
:10B6900021912032E9F3293010F02E30C8F32B32FB
:10B6A00039F02D3231F4689403C044D0820F911DDB
:10B6B000219120532A30C8F31EF4909581959F4F15
:10B6C00008959111E4C5803219F089508550D0F762
:10B6D0000895FB01DC0105900D920020E1F708952B
:10B6E00042E95BE000C0FA01A191B081009719F432
:10B6F0001097E1F0CD01DC01CD010D90002011F497
:10B70000C00113C0FB012191222319F02015D9F7A4
:10B71000F3CFFB012191201519F41E92119606C05A
:10B720002223C1F70D900020A1F7D001FA01A193C7
:10B73000B08308957AE0979F902D879F802D910D7B
:10B7400011240895FC01238127FF0FC0E8E9FBE0E5
:10B75000208131812817390711F411821082329625
:10B760002BE0EE39F207A1F7A2DE80E090E0089529
:10B770000F931F93CF93DF93009731F461157105F9
:10B7800019F480E090E039C08B01EC016EE070E0CC
:10B7900081E090E062D5FC01892B99F380E88383F6
:10B7A0000115110571F01387028781E88383809169
:10B7B000980B9091990B892B21F4F093990BE093BE
:10B7C000980B2097C9F0D187C087838182608383DB
:10B7D00080919A0B90919B0B892B71F4F0939B0BAA
:10B7E000E0939A0B80919C0B90919D0B892B21F4F7
:10B7F000F0939D0BE0939C0BCF01DF91CF911F91B4
:10B800000F910895CF93DF93EC012B8120FF33C07C
:10B8100026FF0AC02F7B2B838E819F8101969F83F9
:10B820008E838A8190E029C022FF0FC0E881F981D0
:10B830008081082E000C990B009719F420622B834D
:10B840001AC03196F983E8830EC0EA85FB85199505
:10B8500097FF09C02B81019611F080E201C080E1C1
:10B86000822B8B8308C02E813F812F5F3F4F3F8308
:10B870002E83992702C08FEF9FEFDF91CF9108951C
:10B880000F931F93CF93DF93CDB7DEB7088519854C
:10B89000F801838188608383AE01445F5F4F6A85CE
:10B8A0007B85C80125D0F8012381277F2383DF9181
:10B8B000CF911F910F9108950F931F93CF93DF9313
:10B8C000CDB7DEB708851985F80183818860838349
:10B8D000AE01445F5F4F6A857B85C8019ED3F80146
:10B8E0002381277F2383DF91CF911F910F910895AB
:10B8F0002F923F924F925F926F927F928F929F9280
:10B90000AF92BF92CF92DF92EF92FF920F931F936D
:10B91000CF93DF93CDB7DEB72C970FB6F894DEBF89
:10B920000FBECDBF7C016B018A01FC01178216821C
:10B93000838181FFB0C1CE0101964C01F701938153
:10B94000F60193FD859193FF81916F01882309F49E
:10B950009EC1853239F493FD859193FF81916F01EA
:10B96000853221F4B70190E0BDD4E8CF512C312CC1
:10B9700020E02032A0F48B3269F030F4803259F0AC
:10B98000833269F420612CC08D3239F0803339F470
:10B99000216026C02260246023C0286021C027FDCA
:10B9A00027C030ED380F3A3078F426FF06C0FAE0B1
:10B9B0005F9E300D1124532E13C08AE0389E300D47
:10B9C0001124332E20620CC08E3221F426FD5FC17B
:10B9D000206406C08C3611F4206802C0883641F419
:10B9E000F60193FD859193FF81916F018111C1CF84
:10B9F000982F9F7D9554933028F40C5F1F4FFFE3E1
:10BA0000F9830DC0833631F0833771F0833509F047
:10BA100057C021C0F801808189830E5F1F4F4424E5
:10BA20004394512C540114C03801F2E06F0E711C84
:10BA3000F801A080B18026FF03C0652D70E002C030
:10BA40006FEF7FEFC5012C8742D42C0183012C8539
:10BA50002F77222E16C03801F2E06F0E711CF8010C
:10BA6000A080B18026FF03C0652D70E002C06FEF9B
:10BA70007FEFC5012C8719D42C012C852068222E3C
:10BA8000830123FC19C0832D90E048165906A0F4C9
:10BA9000B70180E290E026D43A94F5CFF50127FC77
:10BAA000859127FE81915F01B70190E01BD4311091
:10BAB0003A94F1E04F1A51084114510479F7DEC06D
:10BAC000843611F0893631F5F80127FF07C060810F
:10BAD0007181828193810C5F1F4F08C060817181E9
:10BAE000072E000C880B990B0E5F1F4F2F76722EBE
:10BAF00097FF09C090958095709561957F4F8F4F06
:10BB00009F4F2068722E2AE030E0A4013CD4A82E7A
:10BB1000A81843C0853729F42F7EB22E2AE030E0E2
:10BB200025C0F22FF97FBF2E8F36C1F018F488356B
:10BB300079F0ADC0803719F0883721F0A8C02F2FD9
:10BB40002061B22EB4FE0DC08B2D8460B82E09C0CA
:10BB500024FF0AC09F2F9660B92E06C028E030E06F
:10BB600005C020E130E002C020E132E0F801B7FE7C
:10BB700007C060817181828193810C5F1F4F06C075
:10BB80006081718180E090E00E5F1F4FA401FBD3C4
:10BB9000A82EA818FB2DFF777F2E76FE0BC0372D21
:10BBA0003E7FA51450F474FE0AC072FC08C0372D05
:10BBB0003E7E05C0BA2C372D03C0BA2C01C0B52C6F
:10BBC00034FF0DC0FE01EA0DF11D8081803311F4B8
:10BBD000397E09C032FF06C0B394B39404C0832FEA
:10BBE000867809F0B39433FD12C030FF06C05A2C9A
:10BBF000B31418F4530C5B18B32CB31460F4B701EE
:10BC000080E290E03C876ED3B3943C85F6CFB314CA
:10BC100010F43B1801C0312C34FF11C0B70180E390
:10BC200090E03C875FD33C8532FF16C031FD03C0F6
:10BC300088E790E002C088E590E0B7010CC0832F50
:10BC4000867851F031FF02C08BE201C080E237FDFF
:10BC50008DE2B70190E046D3A51430F4B70180E33C
:10BC600090E040D35A94F8CFAA94F401EA0DF11D64
:10BC70008081B70190E036D3A110F6CF332009F4CC
:10BC80005DCEB70180E290E02DD33A94F7CFF70173
:10BC90008681978102C08FEF9FEF2C960FB6F894A4
:10BCA000DEBF0FBECDBFDF91CF911F910F91FF90EF
:10BCB000EF90DF90CF90BF90AF909F908F907F904C
:10BCC0006F905F904F903F902F90089520FD09C096
:10BCD000FC0123FD05C022FF02C0738362835183F0
:10BCE0004083089544FD10C046FD10C0DB01FC01F7
:10BCF000AA0FBB1FEE1FFF1F1094D1F76A0F7B1F07
:10BD00008E1F9F1F31E003C033E001C034E0660F97
:10BD1000771F881F991F3150D1F7620F711D811D48
:10BD2000911D08950F931F93CF93DF938C01C8014A
:10BD300069DDEC0197FD06C0C4DC892BC1F7B801B1
:10BD4000CE0108D3CE01DF91CF911F910F910895BD
:10BD50008F929F92AF92BF92CF92DF92EF92FF921B
:10BD60000F931F93CF93DF931F92CDB7DEB78C0154
:10BD7000C62E7A01298346DDAC01552729814B3235
:10BD8000510521F04D32510561F42068CA94C1106B
:10BD900002C080E06FC0C801298334DD298197FD8E
:10BDA000F8CF322F3D7FD32E322F307339F58033C9
:10BDB00029F5BB24BA94BC0C09F449C0C8012983F5
:10BDC00021DD298197FD43C0382F3F7D383561F44F
:10BDD0008D2D8264D82ECA94CA94CC20C1F1C8019A
:10BDE00011DD97FF0BC033C026FF04C02D2D22604C
:10BDF000D22E03C03D2D3261D32ECB2C812C912C21
:10BE0000540120ED280F283078F0D4FE03C0B8018B
:10BE1000A1D21AC02A3040F0D6FEF9CF2F7D3FEED6
:10BE2000320F3630A0F727504D2DC501B4015ADF2F
:10BE30004B015C018D2D8260D82ECA94CC2051F02C
:10BE4000C801E0DC97FFDDCFD1FC04C0A2CF812C7C
:10BE5000912C5401D7FE08C0B094A0949094809483
:10BE6000811C911CA11CB11C2D2DB501A401C70181
:10BE70002DDF81E00F90DF91CF911F910F91FF9007
:10BE8000EF90DF90CF90BF90AF909F908F900895EC
:10BE90006F927F928F929F92AF92BF92CF92DF92DA
:10BEA000EF92FF920F931F93CF93DF93CDB7DEB73F
:10BEB000A1970FB6F894DEBF0FBECDBF5C017A012B
:10BEC000CE0101966C0180E2F60111928A95E9F7A4
:10BED000F501838040E050E0912C712C70E0A1E0EE
:10BEE000B0E0F90183FC859183FE81918F01982F49
:10BEF0009F01811103C080E090E07AC08E3519F473
:10BF00004115510549F1E72FF0E0E417F5073CF43E
:10BF10008D3559F18D3219F4772001F103C071107C
:10BF200001C0982E892F8695869586958601080FE3
:10BF3000111D892F87703D0101C0660C8A95EAF7B3
:10BF4000F801808186298083991559F0991510F49C
:10BF50009F5FE8CF9150E6CF71E004C077247394DF
:10BF600001C0712C4F5F5F4FBCCF772019F08E81DD
:10BF700080628E83711103C09924939416C0F601D8
:10BF80009E012F5D3F4F808180958193E217F307DB
:10BF9000D1F7F2CFE114F10429F0F7018083C70152
:10BFA00001967C016150912CE9F0C50169A32ADC5E
:10BFB00069A197FD15C0282F269526952695F6018F
:10BFC000E20FF11D208130E0AC014770552702C01F
:10BFD000359527954A95E2F720FDDCCFB501BAD11A
:10BFE000911089CFE114F10411F0F7011082C8011A
:10BFF000A1960FB6F894DEBF0FBECDBFDF91CF91F3
:10C000001F910F91FF90EF90DF90CF90BF90AF9076
:10C010009F908F907F906F9008954F925F927F9244
:10C020008F929F92AF92BF92CF92DF92EF92FF9248
:10C030000F931F93CF93DF931F92CDB7DEB76C01A1
:10C040002B015A01FC0117821682712CF601F38034
:10C05000F201F3FC8591F3FE8191382F2F018823A3
:10C0600009F4E5C090E039832CDB3981892B19F084
:10C07000C60158DEEBCF353241F4F201F3FC3591C5
:10C08000F3FE31912F01353259F4C6013983BADB01
:10C09000398197FDCAC03817C9F2B6015BD1C7C054
:10C0A0003A3239F4F3FC3591F3FE31912F0151E02E
:10C0B00001C050E0420110E020ED230F2A3088F447
:10C0C0005260612F70E080E090E040E259830ADE28
:10C0D000162FF401F3FC3591F3FE31914F01598194
:10C0E000EBCF052F232F240151FF03C0111102C0F4
:10C0F0009EC01FEF383619F03C3659F011C0F401DC
:10C10000F3FC2591F3FE21912F01283649F4052FE8
:10C1100008600460F201F3FC2591F3FE21912F01E8
:10C12000222309F484C0622F70E086E492E0298320
:10C13000B1D02981892B09F47AC000FD07C0F5012F
:10C14000E080F180C50102965C0102C0E12CF12C77
:10C150002E3649F4F6014681578160E070E0202FC9
:10C16000C701B4DD73CF233689F401FF11E0C601A6
:10C1700049DB97FD5AC0E114F10429F0F7018083EF
:10C18000C70101967C01115091F74BC02B3551F43A
:10C190009201A701612FC6017BDE2C01892B09F0DA
:10C1A00040C03AC0C6012983BDDD298197FD3DC04D
:10C1B0002F3641F128F4243619F1293631F124C003
:10C1C000233769F02537E1F01FC0E114F10429F0AD
:10C1D000F7018082C70101967C01115059F0C60118
:10C1E00011DB4C0197FD06C06CDA892B71F3B601A7
:10C1F000C401B0D0E114F104A1F0F701108211C024
:10C20000006203C0006101C00064202FA701612FFC
:10C21000C6019EDD811105C0F6018381807329F47A
:10C2200006C000FD13CF739411CF772019F0872D2E
:10C2300090E002C08FEF9FEF0F90DF91CF911F91A1
:10C240000F91FF90EF90DF90CF90BF90AF909F90B5
:10C250008F907F905F904F9008950F931F93CF938F
:10C26000DF93869F8001879F100D969F100D1124EC
:10C27000C80188D8EC01009721F0A80160E070E0C7
:10C280001FD0CE01DF91CF911F910F910895992773
:10C2900088270895FC010590061621F00020D9F7A3
:10C2A000C00108953197CF010895FC0105906150B8
:10C2B00070400110D8F7809590958E0F9F1F0895BC
:10C2C000DC0101C06D9341505040E0F70895FC013E
:10C2D0006150704001900110D8F7809590958E0FB5
:10C2E0009F1F08950F931F93CF93DF93FB0123812B
:10C2F00021FD03C08FEF9FEF28C022FF16C04681AB
:10C300005781248135814217530744F4A081B181BC
:10C310009D012F5F3F4F318320838C93268137818E
:10C320002F5F3F4F3783268310C0EB01092F182F53
:10C330000084F185E02D1995892BE1F68E819F818E
:10C3400001969F838E83812F902FDF91CF911F9134
:10C350000F910895FB01238120FF12C026FD10C01C
:10C360008F3F3FEF930761F082832F7D206423830B
:10C3700026813781215031093783268399270895F3
:10C380008FEF9FEF0895FA01AA27283051F120314D
:10C3900081F1E8946F936E7F6E5F7F4F8F4F9F4F59
:10C3A000AF4FB1E03ED0B4E03CD0670F781F891F9B
:10C3B0009A1FA11D680F791F8A1F911DA11D6A0F69
:10C3C000711D811D911DA11D20D009F468943F911C
:10C3D0002AE0269F11243019305D3193DEF6CF011B
:10C3E0000895462F4770405D4193B3E00FD0C9F7E1
:10C3F000F6CF462F4F70405D4A3318F0495D31FD4E
:10C400004052419302D0A9F7EACFB4E0A6959795A0
:10C41000879577956795BA95C9F700976105710576
:10C4200008959B01AC010A2E0694579547953795C0
:10C430002795BA95C9F7620F731F841F951FA01D1A
:10C440000895F999FECF92BD81BDF89A992780B5DC
:10C450000895262FF999FECF1FBA92BD81BD20BD48
:10C460000FB6F894FA9AF99A0FBE01960895A1E2D0
:10C470001A2EAA1BBB1BFD010DC0AA1FBB1FEE1F5E
:10C48000FF1FA217B307E407F50720F0A21BB30BA9
:10C49000E40BF50B661F771F881F991F1A9469F725
:10C4A00060957095809590959B01AC01BD01CF0181
:10C4B0000895052E97FB16F400940FD057FD05D074
:10C4C000D6DF07FC02D046F408C050954095309561
:10C4D00021953F4F4F4F5F4F0895909580957095F0
:10C4E00061957F4F8F4F9F4F08950FD0A59F900D5F
:10C4F000B49F900DA49F800D911D11240895B7FF46
:10C50000F4CFF3DF821B930B0895A29FB001B39F7A
:10C51000C001A39F700D811D1124911DB29F700D4C
:10C52000811D1124911D08955058BB27AA270ED0B4
:10C5300075C166D130F06BD120F031F49F3F11F41A
:10C540001EF45BC10EF4E095E7FB51C1E92F77D1F2
:10C5500080F3BA17620773078407950718F071F420
:10C560009EF58FC10EF4E0950B2EBA2FA02D0B0176
:10C57000B90190010C01CA01A0011124FF27591B28
:10C5800099F0593F50F4503E68F11A16F040A22F2E
:10C59000232F342F4427585FF3CF4695379527959F
:10C5A000A795F0405395C9F77EF41F16BA0B620B9E
:10C5B000730B840BBAF09150A1F0FF0FBB1F661FE5
:10C5C000771F881FC2F70EC0BA0F621F731F841F28
:10C5D00048F4879577956795B795F7959E3F08F04E
:10C5E000B3CF9395880F08F09927EE0F979587950D
:10C5F0000895D9D008F481E008950CD00FC107D177
:10C6000040F0FED030F021F45F3F19F0F0C051113E
:10C6100039C1F3C014D198F39923C9F35523B1F369
:10C62000951B550BBB27AA2762177307840738F0A1
:10C630009F5F5F4F220F331F441FAA1FA9F333D000
:10C640000E2E3AF0E0E830D091505040E695001CB4
:10C65000CAF729D0FE2F27D0660F771F881FBB1F70
:10C66000261737074807AB07B0E809F0BB0B802D4A
:10C67000BF01FF2793585F4F2AF09E3F510568F096
:10C68000B6C000C15F3FECF3983EDCF3869577952A
:10C690006795B795F7959F5FC9F7880F911D969598
:10C6A000879597F90895E1E0660F771F881FBB1FF4
:10C6B000621773078407BA0720F0621B730B840BA1
:10C6C000BA0BEE1F88F7E095089504D06894B11175
:10C6D000D9C00895BCD088F09F5790F0B92F992702
:10C6E000B751A0F0D1F0660F771F881F991F1AF07D
:10C6F000BA95C9F712C0B13081F0C3D0B1E0089546
:10C70000C0C0672F782F8827B85F39F0B93FCCF3C6
:10C71000869577956795B395D9F73EF49095809572
:10C72000709561957F4F8F4F9F4F0895E89409C092
:10C7300097FB3EF490958095709561957F4F8F4F54
:10C740009F4F9923A9F0F92F96E9BB279395F6956A
:10C75000879577956795B795F111F8CFFAF4BB0FE8
:10C7600011F460FF1BC06F5F7F4F8F4F9F4F16C04C
:10C77000882311F096E911C0772321F09EE8872FD6
:10C78000762F05C0662371F096E8862F70E060E092
:10C790002AF09A95660F771F881FDAF7880F96950B
:10C7A000879597F90895990F0008550FAA0BE0E8AF
:10C7B000FEEF16161706E807F907C0F01216130663
:10C7C000E407F50798F0621B730B840B950B39F4A3
:10C7D0000A2661F0232B242B252B21F408950A2609
:10C7E00009F4A140A6958FEF811D811D089597F949
:10C7F0009F6780E870E060E008959FEF80EC089507
:10C8000000240A941616170618060906089500242F
:10C810000A9412161306140605060895092E0394A9
:10C82000000C11F4882352F0BB0F40F4BF2B11F41D
:10C8300060FF04C06F5F7F4F8F4F9F4F089557FD7C
:10C840009058440F551F59F05F3F71F04795880F7E
:10C8500097FB991F61F09F3F79F087950895121615
:10C8600013061406551FF2CF4695F1DF08C01616C1
:10C8700017061806991FF1CF869571056105089472
:10C880000895E894BB2766277727CB0197F9089589
:10C890008ADF08F48FEF08950BD0C0CFB1DF28F006
:10C8A000B6DF18F0952309F0A2CFA7CF1124EACF65
:10C8B000C6DFA0F3959FD1F3950F50E0551F629FFF
:10C8C000F001729FBB27F00DB11D639FAA27F00DE9
:10C8D000B11DAA1F649F6627B00DA11D661F829F10
:10C8E0002227B00DA11D621F739FB00DA11D621FF5
:10C8F000839FA00D611D221F749F3327A00D611D12
:10C90000231F849F600D211D822F762F6A2F1124F3
:10C910009F5750408AF0E1F088234AF0EE0FFF1F46
:10C92000BB1F661F771F881F91505040A9F79E3F7D
:10C93000510570F05CCFA6CF5F3FECF3983EDCF37F
:10C94000869577956795B795F795E7959F5FC1F7BA
:10C95000FE2B880F911D9695879597F90895FA01FA
:10C96000EE0FFF1F30962105310599F16115710514
:10C9700061F48038BFE39B0749F1689490388105E2
:10C9800061F08038BFEF9B0741F0992342F5FF3FEC
:10C99000E1053105210511F1E8940894E795D901E5
:10C9A000AA2329F4AB2FBE2FF85FD0F310C0FF5F8E
:10C9B00070F4A695E0F7F73950F019F0FF3A38F423
:10C9C0009F779F930CD00F9007FC905808953EF0EE
:10C9D00014CF60E070E080E89FE308954FE79F7711
:10C9E0005F934F933F932F939ED02F913F914F9101
:10C9F0005F9152DF05C019F40EF0F9CE42CFFDCEA3
:10CA000026DFC8F39638C0F707F80F92E8942BE3B7
:10CA10003AEA48EB5FE74EDF0F920F920F924DB765
:10CA20005EB70F92C0D0E4ECF1E016D04F915F9169
:10CA3000EF91FF91E595EE1FFF1F49F0FE57E0686B
:10CA40004427EE0F441FFA95E1F74195550B32D07C
:10CA50000F9007FE26C00895DF93CF931F930F9387
:10CA6000FF92EF92DF927B018C01689405C0DA2E71
:10CA7000EF011EDFFE01E894A591259135914591C6
:10CA80005591AEF3EF0162DDFE019701A801DA9442
:10CA900079F7DF90EF90FF900F911F91CF91DF9189
:10CAA00008959B01AC0160E070E080E89FE3A5CDB4
:10CAB0009ECEACC0CCDEE8F39923D9F3940F511D80
:10CAC000BBF39150504094F059F0882332F0660F38
:10CAD000771F881F91505040C1F79E3F510544F782
:10CAE000880F911D9695879597F908955F3FACF053
:10CAF000983E9CF0BB27869577956795B79508F487
:10CB0000B1609395C1F7BB0F58F711F460FFE8CF00
:10CB10006F5F7F4F8F4F9F4FE3CFB4CE0EF076C045
:10CB20006CCE689464CE93DEC8F39923D1F3C6F338
:10CB3000DF93CF931F930F93FF92C92FDD27882395
:10CB40002AF02197660F771F881FDAF720E030E080
:10CB500040E85FEB9FE3883920F0803E30F021967B
:10CB60008F77E3DCECEEF1E003C0DFDCE9E1F2E03B
:10CB700073DF8B01BE01EC01FB2E6F5771097595B8
:10CB8000771F880B990BD4DD28E132E741E35FE39F
:10CB90008FDEAF2D9801AE01FF900F911F91CF91C5
:10CBA000DF91D4DC3BCEFA01DC01AA0FBB1F9B0155
:10CBB000AC01BF5728F422273327442750781FC0E1
:10CBC000B75188F4AB2F0024469537952795011C63
:10CBD000A395D2F3002069F0220F331F441FB395B1
:10CBE000DAF30DD0A1CC61307105A0E88A07B9460F
:10CBF00030F49B01AC016627772788279078309620
:10CC000021F0208331834283538308959F3F31F085
:10CC1000915020F4879577956795B795880F911D6A
:10CC20009695879597F9089597FB072E16F400942B
:10CC300006D077FD08D020D007FC05D03EF49095B3
:10CC400081959F4F0895709561957F4F0895EE0FE0
:10CC5000FF1F881F8BBF0790F691E02D199469275D
:10CC60009627692778278727782708954EDCB7FF0E
:10CC70000895821B930B0895AA1BBB1B51E107C0AB
:10CC8000AA1FBB1FA617B70710F0A61BB70B881F5C
:10CC9000991F5A95A9F780959095BC01CD010895EB
:10CCA00081E090E0F89425C10F931F93CF93DF9319
:10CCB0008C01FC0101900020E9F7CF01801B910B52
:10CCC0000E94C259EC01009711F0B80145D0CE0185
:10CCD000DF91CF911F910F910895FB01DC0104C0FA
:10CCE0008D910190801921F441505040C8F7881B64
:10CCF000990B0895FB01DC018D9181341CF08B357B
:10CD00000CF4805E619161341CF06B350CF4605E54
:10CD1000861B611189F3990B0895FB01DC010D90CD
:10CD20000020E9F7119701900D920020E1F7089596
:10CD3000FC018191861721F08823D9F7992708955E
:10CD40003197CF010895FB01DC018D91019080198D
:10CD50000110D9F3990B0895FB01DC0101900D92AC
:10CD60000020E1F70895FB01DC010D900020E9F7B8
:10CD700011974150504028F0019000200D92C9F7C2
:10CD800008951C920895FB01DC014150504030F0A1
:10CD90008D910190801919F40020B9F7881B990B27
:10CDA0000895FB01DC014150504048F001900D9284
:10CDB0000020C9F701C01D9241505040E0F708958E
:10CDC000FC0181E090E00190061609F4CF010020FB
:10CDD000D1F7019708950F931F93CF93DF93CDB7AA
:10CDE000DEB72E970FB6F894DEBF0FBECDBF0E890B
:10CDF0001F89888D998D26E02C831A83098397FFDC
:10CE000002C080E090E801979E838D83AE01445E6E
:10CE10005F4F6A8D7B8DCE0101960E94785C4D81BB
:10CE20005E8157FD0AC02F813885421753070CF4E5
:10CE30009A01F801E20FF31F10822E960FB6F894B4
:10CE4000DEBF0FBECDBFDF91CF911F910F9108952F
:10CE50000F931F93CF93DF93CDB7DEB72E970FB607
:10CE6000F894DEBF0FBECDBF0E891F8986E08C838C
:10CE70001A8309838FEF9FE79E838D83AE01465E01
:10CE80005F4F688D798DCE0101960E94785C2F816D
:10CE90003885F801E20FF31F10822E960FB6F89432
:10CEA000DEBF0FBECDBFDF91CF911F910F910895CF
:10CEB000CF93DF93CDB7DEB72E970FB6F894DEBFD2
:10CEC0000FBECDBF85E08C838C899D899A83898331
:10CED000AE01485E5F4F6E897F89CE0101969DD875
:10CEE0002E960FB6F894DEBF0FBECDBFDF91CF9167
:06CEF0000895F894FFCF45
:10CEF60003100001200000C000009E0B800001000E
:10CF060000000000000000000000DEADBEEFFE00E5
:10CF16005E00BC00770100000000F2074172742D2C
:10CF26004E6574000000044D515454040000000086
:10CF36006222930FA9485322A1227F22AF221D23EA
:10CF4600582300000000DA22930FA9485322242315
:10CF56009F24AF221D235823000000006A2E122FA3
:10CF6600A9484438802E0A3963385F2F86394A2FFC
:10CF7600A230C92F6030B92EEC38982E882E842E18
:10CF860030313233343536373839414243444546F9
:10CF96000001005E0000006C617A79686F6D652E95
:10CFA6007275000000000000000000000000000094
:10CFB60000000000000000000000006124930FA99B
:10CFC600485322F2227224AF221D23582300000068
:10CFD60000EB3DA53EA948B42E293E103E8C2F15E8
:10CFE6003F313EB52E0C31E930AC2E0D3E0B3EA145
:10CFF6002E013E00000000DA22930FA94853222496
:10D00600238F24AF221D23582300000000471093CE
:10D016000FD70F8D100810E60FFA0F00000000471B
:10D026001D181DA948EC1C101DFC1CED1C00000061
:10D036000085118511A948851185118511851185F0
:10D046001185118511851185118511000000008556
:10D0560011930FA948A84885118511851100000074
:10D06600008511930FA948A84800000000EB3DA5D4
:10D076003EA948B42E293E103E8C2F153F313EB5B1
:10D086002E0C31E930AC2E0D3E0B3EA12E013E009A
:10D096000000005C120000000085114F4E004F4654
:10D0A60046005245535400544F47474C45004841AB
:10D0B6004C54003B0068656C700073617665006CCB
:10D0C6006F61640067657400736574006B696C6CEE
:10D0D60000726571000D0A005F737461740056007A
:10D0E60052504D004900737700666C740070777279
:10D0F600002F616C61726D005300496E3A20002F5B
:10D10600003D006974656D0073636D640072636D44
:10D116006400656D6974002F6D79686F6D652F69A0
:10D126006E2F230031772054696D656F7574005238
:10D1360065736574206572726F720020636F6D701F
:10D146005F6964210022002525253278006E756C02
:10D156006C00747275650066616C7365002D002E37
:10D166000057495A6E657400646D7800646D78697D
:10D176006E006974656D73006D6F64627573006D22
:10D18600717474006F770025783A25783A25783AD5
:10D1960025783A25783A257825D181002F7265734E
:10D1A600702F23002F7265712F636F6E660031003A
:10D1B6002F253032782D253032782D253032782DB6
:10D1C600253032782D253032782D253032782E6371
:10D1D6006F6E6669672E6A736F6E005D20006F6EF4
:10D1E60020536B6970706564002F6D79686F6D658B
:10D1F6002F6F75742F526573746F726553746174F3
:10D2060065002564002C002F616C61726D6F666687
:02D21600000016
:00000001FF
